:100000000C94F6090C94500A0C94500A0C94500A63
:100010000C94500A0C94500A0C94500A0C94500AF8
:100020000C94500A0C94581E0C94500A0C94500ACC
:100030000C94CF380C94500A0C94500A0C94500A2B
:100040000C94500A0C94500A0C947B1A0C94500A8D
:100050000C94AC100C94500A0C9476100C94500A2A
:100060000C9466200C94500A0C9417340C94500A8B
:100070000C94939D0C94500A0C94D1920C94500AB9
:100080000C94500A0C94500A0C94500A8F2094201F
:100090009920A220B920D020E020F0205E21B623B4
:1000A000D0207A228B22A022BF22DC222723732396
:1000B00026260A27AD2726285E280E29C829312A98
:1000C000AC2ADE2A4A2B782BA52B052C5E2CC32CC0
:1000D0000E2D582DBC2D3E723C73C173DE7215740B
:1000E00045747D720D730681AA812F828A82DB821C
:1000F0004483888DC683FA83FA83FA83FA83FA836A
:10010000FA83FA83FA83FA832784A2843F8564857D
:10011000A785FF859586A0870388038803880388C1
:100120000388038803880388038833885188768886
:10013000D2880E8965899289328A888D898A898ACE
:10014000898A898A898A898A898A898A909B939BE4
:10015000939B939B9C9B9F9BA29BB49BB19B0A0DE3
:100160003D3D3D3D3D3D3D3D3D3D3D3D3D3D3D3DBF
:100170003D3D3D3D3D3D3D3D3D3D3D3D3D3D3D3DAF
:100180003D3D3D000A0D426174743A002025642013
:1001900043656C6C732000204C6F77207761726E22
:1001A000696E673A2025642E25645600202041752B
:1001B000746F2D43483A2025642E25645600202074
:1001C0004175746F6C616E64696E673A2025642EA8
:1001D000256456000A0D466C69676874436F6E7437
:1001E000726F6C206E6F7420737570706F727465AF
:1001F0006421000A0D466F756E6420424C2D4374D5
:10020000726C3A20002564000A0D0A0D2121204D50
:10021000495353494E4720424C2D4354524C3A20A7
:100220002564202121000A0D43616C6962726174AA
:10023000696E672070726573737572652073656E81
:10024000736F722E2E004F4B0A0D000A0D466C691B
:100250006768742D74696D65202575206D696E2041
:10026000546F74616C3A2575206D696E00416E673C
:100270006C654E69636B20202020202020416E6732
:100280006C65526F6C6C202020202020204163631D
:100290004E69636B202020202020202020416363B2
:1002A000526F6C6C20202020202020202059617764
:1002B0004779726F202020202020202020416C745C
:1002C0006974756465205B302E316D5D2041636318
:1002D0005A20202020202020202020202047617329
:1002E00020202020202020202020202020436F6D4F
:1002F000706173732056616C7565202020566F6C99
:1003000074616765205B302E31565D202052656335
:100310006569766572204C6576656C202047797238
:100320006F20436F6D70617373202020204D6F74B8
:100330006F7220312020202020202020204D6F743B
:100340006F7220322020202020202020204D6F742A
:100350006F7220332020202020202020204D6F7419
:100360006F722034202020202020202020313620B1
:100370002020202020202020202020202031372055
:100380002020202020202020202020202031382044
:100390002020202020202020202020202031392033
:1003A0002020202020202020202020202053657283
:1003B000766F2020202020202020202020486F76CB
:1003C00065726761732020202020202020437572F1
:1003D00072656E74205B302E31415D202043617068
:1003E0006163697479205B6D41685D2020486569AF
:1003F00067687420536574706F696E74203235209D
:1004000020202020202020202020202020323620C4
:1004100020202020202020202020202020436F6D1D
:100420007061737320536574706F696E74493243E1
:100430002D4572726F7220202020202020424C20F7
:100440004C696D69742020202020202020475053C3
:100450005F4E69636B2020202020202020475053CE
:100460005F526F6C6C202020202020202021212131
:1004700020494E434F4D50415449424C4520212183
:1004800021002E005B25695D005B25695D002B2046
:100490004D696B726F4B6F70746572202B004857FB
:1004A0003A5625642E25642053573A25642E25306C
:1004B00032642563200053657474696E673A25645D
:1004C000202573004D69786572204572726F722124
:1004D000004552522532643A004861726477617275
:1004E00065204572726F7220313A25642021210007
:1004F0004D697373696E6720424C2D4374726C3A78
:10050000256420212100493243204552524F522177
:10051000212100424C2D53656C667465737420452F
:1005200072723A253264004865696768743A20201F
:1005300025356900536574706F696E743A253569A5
:100540000050726573737572653A253569004F66A0
:10055000667365743A2020253569002841290025F5
:1005600069006163742E2062656172696E67004E76
:1005700069636B3A20202020202025356900526FC6
:100580006C6C3A20202020202025356900436F6DB7
:10059000706173733A202020253569004B25693A34
:1005A00025346920204B25693A25346920004E699D
:1005B0003A2534692020526F3A2534692000477368
:1005C0003A253469202047693A25346920005031A2
:1005D0003A253469202050323A25346920005033BE
:1005E0003A253469202050343A253469200047796F
:1005F000726F202D2053656E736F72004E69636BAE
:100600002025346920282533692E25782900526F4A
:100610006C6C2025346920282533692E2578290023
:100620005961772020253469202825336929004124
:100630004343202D2053656E736F72004E69636BC8
:100640002025346920282533692900526F6C6C20DD
:10065000253469202825336929005A2020202025A7
:10066000346920282533692900566F6C74616765E9
:100670003A2020202533692E2531695600437572B2
:1006800072656E743A2020202533692E2531694128
:1006900000506F7765723A2020202020253469575A
:1006A000004469736368617267653A202535696D36
:1006B00041680052656365697665720052432D5149
:1006C00075616C6974793A202534690052432D4371
:1006D00068616E6E656C733A25346900556E6465A9
:1006E00072766F6C74616765732020005761726E5B
:1006F0003A202532642E25645600486F6D653A20F5
:100700002532642E256456004C616E643A202532F1
:10071000642E25645600506F746925693A2020259F
:10072000336900506F746925693A202025336900C8
:10073000466C696768742D54696D65202000546F9C
:1007400074616C3A2535756D696E004163743A20A9
:10075000202535756D696E002872657365742900F2
:10076000436F6D70617373004D61676E65743A20FD
:100770002020253569004779726F3A2020202020FB
:1007800025356900536574706F696E743A2025359C
:100790006900536572766F202000536574706F692D
:1007A0006E74202025336900506F736974696F6E11
:1007B0003A202533690052616E67653A2533692D09
:1007C00025336900424C2D4374726C204572726F60
:1007D0007273200025336420253364202533642080
:1007E0002533642000424C2054656D70657261743D
:1007F0007572650025336420253364202533642019
:100800002533642000424C2043757272656E74007B
:1008100028696E20302E314129002533642025338C
:100820006420253364202533642000424C2D43741A
:10083000726C20666F756E64200020256320202076
:1008400025632020202563202020256320002025EB
:10085000632020202563202020256320202025637D
:1008600020002025632020202D2020202D20202046
:100870002D20003130003131003132000A0D2D2D94
:100880003E204861726477617265205665727369B3
:100890006F6E2042797465204368616E67656420DD
:1008A0003C2D2D000A0D47656E65726174696E6797
:1008B0002064656661756C7420506172616D657449
:1008C000657220536574202564000A0D5573696EA6
:1008D0006720506172616D65746572205365742084
:1008E0002564000A0D47656E65726174696E672044
:1008F00064656661756C74204D6978657220546119
:10090000626C65000A0D4D697865722D436F6E66E5
:1009100069673A202725732720282575204D6F7495
:100920006F727329000A0D414343206E6F74206378
:10093000616C69627261746564210D0A0000008F48
:10094000001E01AD013B02CA025803E60374040213
:10095000058F051B06A7063307BE074808D2085BAC
:1009600009E3096B0AF20A780BFD0B810C040D8672
:100970000D070E870E060F840F00107B10F5106E0A
:1009800011E5115B12CF124213B31323149214FE1C
:10099000146A15D3153B16A11605176717C8172734
:1009A000188318DE1837198E19E319361A871AD6E4
:1009B0001A231B6E1BB61BFD1B411C831CC31C0092
:1009C0001D3C1D751DAB1DE01D121E421E6F1E9AA3
:1009D0001EC31EE91E0D1F2E1F4D1F691F841F9B66
:1009E0001FB01FC31FD31FE11FEC1FF51FFB1FFF0D
:1009F0001F00200000050005000401060108000694
:100A000001020004000400070007000700070007B8
:100A1000000700070003010301050017010F01068D
:100A20000009010A0119010501050119011A010F47
:100A30000101000900060006004E6F204572726F2A
:100A4000722020202020202020004E6F7420636F11
:100A50006D70617469626C652020004D4B334D618F
:100A600067206E6F7420636F6D7061004E6F20465B
:100A70004320636F6D6D756E6963617400436F6DC4
:100A80007061737320636F6D6D756E69630047509D
:100A90005320636F6D6D756E69636174696F006378
:100AA0006F6D706173732076616C75652020200016
:100AB0005243205369676E616C206C6F7374202001
:100AC00000464320737069207278206572726F72DD
:100AD00020004E6F204E4320636F6D6D756E69630D
:100AE0006174004643204E69636B204779726F2022
:100AF00020202000464320526F6C6C204779726F93
:100B00002020202000464320596177204779726FCA
:100B10002020202020004643204E69636B20414363
:100B200043202020202000464320526F6C6C20413F
:100B300043432020202020004643205A2D41434398
:100B400020202020202020200050726573737572B1
:100B5000652073656E736F722000493243204643EF
:100B60002D3E424C2D4374726C2000426C204D6926
:100B70007373696E67202020202020004D697865FE
:100B800072204572726F7220202020200043617213
:100B90006566726565204572726F7220200047504D
:100BA0005320466978206C6F737420202020004DFC
:100BB00061676E6574204572726F7220202020007C
:100BC0004D6F746F7220726573746172742020208F
:100BD00000424C204C696D69746174696F6E20200D
:100BE00020004750532052616E676520202020204E
:100BF0002020004E6F2053442D436172642020203A
:100C00002020200053442D4C6F6767696E67206574
:100C100072726F7200466C79696E672072616E67DE
:100C20006521202020004D617820416C7469747525
:100C3000646521202020004E6F20475053206669B4
:100C40007820202020202000636F6D706173732056
:100C50006E6F742063616C2E00424C2D53656C6680
:100C6000746573742020202020006E6F20657874D6
:100C70002E20636F6D706173732000636F6D706100
:100C800073732073656E736F722020005365742038
:100C9000203A002021212020204C414E44494E473B
:100CA000202020202121202000202121204C6950BB
:100CB0006F20766F6C7461676520212120200020F1
:100CC000202020204D696B726F4B6F70746572200D
:100CD0002020202000202020202020202020202034
:100CE00020202020202020202020002020253269C4
:100CF0002E2531695620200020202532692E2531ED
:100D00006956202000414C543A2534696D202563F2
:100D100000414C543A2534696D202000414C543A2E
:100D20002D2D2D2D200020202532693A25303269C5
:100D300020200020202532693A2530326920200009
:100D40004449523A202533642563004300200020A3
:100D500020253569202000202025356920200049E4
:100D60003A2532692E2531694120003A003A003A8D
:100D7000002D2D2D2D2D2D2D2D2D2B2D2D2D2D2DD2
:100D80002D2D2D2D2D2D002D2D2D2D2D2D2D2D2DC0
:100D90002D2D2D2D2D2D2D2D2D2D2D2D003A0053AA
:100DA00041543A2532642000444953543A2533646F
:100DB0006D004420003344002121004D41473A2575
:100DC000337525252000484D3A25336425632025B9
:100DD0006300696E636C3A253264256328253269A5
:100DE0002900202020202532756D2F733A202048BD
:100DF0004D3A2533642563202563004552523A203D
:100E00002532642021004552523A20002121204CF5
:100E100069506F20766F6C74616765202121002016
:100E20007777772E4D696B726F4B6F707465722E8A
:100E30006465202000202532693A2530326920205F
:100E40002532692E25316956202534696D416800A7
:100E5000202532693A2530326920202532692E2535
:100E6000316956202534696D4168004449523A255C
:100E70003364256300414C543A2534696D00414C7C
:100E8000543A2534696D00414C543A2D2D2D2D20B6
:100E900000256300484D3A253364256320204449EA
:100EA00053543A2533646D202563005057523A2538
:100EB00032692E25316941202825695729200043B0
:100EC00046002020004750533A2532756D2F73207D
:100ED0005341543A256420002020334420004E4FD3
:100EE000464958004447505320002020204E6F2090
:100EF0004E6176694374726C2020202020202000EF
:100F00002532692E2569202532692E256920253252
:100F1000692E2569202532692E256941002533690E
:100F20002025336920253369202533692563430053
:100F30002532692E2569202532692E256941002533
:100F400032692E2569202532692E256920253269CE
:100F50002E2569202532692E256941002533692017
:100F600025336925634320202020202020200025D0
:100F700033692025336920253369202533692563AA
:100F800043004552523A20253264202100455252F6
:100F90003A20002121204C69506F20766F6C7461DB
:100FA000676520212100207777772E4D696B726F5E
:100FB0004B6F707465722E646520200053657474E5
:100FC000696E673A257520257320004D696E3A25B4
:100FD00032692E253169562025732000414C543A40
:100FE00000504F54493A2533752000284F4E292090
:100FF0002000284F46462920004C494D49540056B0
:101000004152494F0044495341424C4544004346F4
:101010003A0044495341424C45440020284F4E2950
:10102000200020284F4646290020544541434800CF
:101030004750533A0044495341424C4544002846E6
:10104000524545290028484F4D452900284149442B
:1010500029200028484F4C4429002046533A257542
:1010600073656B2000484F4D4520414C543A002594
:10107000756D00484F4C4420004E693A2534692074
:10108000526F3A25346920433A2533690047733A51
:101090002534692059613A253469200050313A25B8
:1010A00034692050323A25346920333A25336900B7
:1010B00050343A2534692050353A25346920363A7F
:1010C00025336900434F55504C494E47204F464603
:1010D0002120004C4F4F50494E47212000484821C5
:1010E0002000434F4D50415353204F46462120008E
:1010F0004C6F616420576179706F696E747300285A
:1011000052656C617469766520506F736974696F9C
:101110006E7329004163746976652057503A253211
:10112000642F256420004E6F205750732061637434
:101130006976652020202020002532692E2531691E
:101140005620002573002020200025326920202011
:10115000004C6F6164206C6973743A004C6F616479
:10116000206C6973743A202D2D20004E6F2053445B
:101170002D436172642020200028536574202D3E89
:10118000204C6F6164290020202020202020202076
:101190002020202000214E6F204750532D46697893
:1011A0002120004C6F616420576179706F696E7403
:1011B000730028466978656420506F736974696F9D
:1011C0006E7329004163746976652057503A253261
:1011D000642F256420004E6F205750732061637484
:1011E00069766520202020002532692E2531695638
:1011F0002000257300202020002532642028464945
:101200005829004C6F6164206C6973743A004C6F0C
:101210006164206C6973743A202D2D20004E6F207C
:1012200053442D43617264202020002853657420AC
:101230002D3E204C6F61642900202020202020209A
:1012400020202020202000004F505152535453564C
:101250005748005859005A554546474841004942A9
:101260004A4A0000000000000000000000444C4D0D
:1012700000000000004E0000004B00430A0D77778D
:10128000772E4D696B726F4B6F707465722E64654B
:101290002028632920486953797374656D7320474A
:1012A0006D6248000A0D74686520757365206F666D
:1012B000207468697320736F667477617265206942
:1012C00073206F6E6C79207065726D6974746564DB
:1012D000200A0D6F6E206F726967696E616C204D18
:1012E000696B726F4B6F707465722D4861726477B1
:1012F000617265005573657200486F54542056340E
:10130000004143542044534C004A657469005370B3
:10131000656B7472756D0050504D000A0D52656317
:1013200065697665723A2000532E42757300756EBA
:101330006B6E6F776E2E205573696E672050504D1F
:101340002E2E2E006E6F7420737570706F72746520
:101350006420627920686172647761726521000A95
:101360000D202D204C4942204E4F5420434F4D50CC
:10137000415449424C452021212121000A0D0A0DEA
:10138000212120426F6F746C6F61646572206E6FF3
:101390007420636F6D70617469626C6520746F2076
:1013A0004861726477617265203E20322E322021BE
:1013B000210A0D0A0D000A0D466C69676874436FB7
:1013C0006E74726F6C0A0D48617264776172653A6F
:1013D00025642E25640A0D536F6674776172653A31
:1013E0005625642E253032642563200011241FBE4B
:1013F000CFEFD0E4DEBFCDBF12E0A0E0B1E0E8E087
:10140000F1E401E00BBF02C007900D92A83EB107C6
:10141000D9F71DE0A8EEB2E001C01D92A432B107D9
:10142000E1F77AEAE2E0F0E081E28093570014917C
:1014300020EF37EF41E050E0C4EAD5E06FE0DA0199
:10144000C9012F5F3F4F4F4F5F4FABBFFC018791EB
:101450008993615067FFF3CF84EE8ABD8091AC051C
:1014600080937805893138F086E08093140187E015
:10147000809313017BEAE4EAF5E06EE0819178273E
:101480007095615067FFFACF8091B305781721F00E
:10149000173911F40000FECF0E94850B0C9483A035
:1014A0000C9400008EE591E09F938F938EE897E176
:1014B0009F938F93E091B705F091B80509950F9030
:1014C0000F900F900F90089580915C08E82FFF27F0
:1014D000EE0FFF1FE053F64F808191818D5E9F4F8D
:1014E00014F010920401808191818A5B9F4FCCF4AB
:1014F000809104018823A9F481E080930401809104
:10150000EB058F5F8093EB05853038F088EE93E034
:101510009093230380932203089566E970E00E946C
:10152000FD3B0895CF93DF93C82F882311F184E802
:1015300091E09F938F938EE897E19F938F93E09133
:10154000B705F091B8050995809126019091270182
:101550006BE270E00E94F69FCB018F5F80930001E9
:101560000F900F900F900F90873018F086E08093C7
:10157000000180917F08823328F590910001989FA7
:10158000802D112480930201CC23F1F068EC70E0EF
:10159000892F0E94FD3B8091000199279F938F9393
:1015A0008CE891E09F938F938EE897E19F938F93C0
:1015B000E091B705F091B80509958DB79EB70696ED
:1015C0008DBF02C0809302019091CA08923340F40B
:1015D00080910001899F802D11248093F20202C026
:1015E0009093F2023091CB08323340F480910001A5
:1015F000839F802D11248093F10202C03093F10269
:101600008091F20290910201981720F491509093EA
:10161000F2029F5F8091F102891720F09150909320
:10162000F1029F5F8091F2022091F102821728F06F
:10163000332319F021502093F202CC2309F462C025
:10164000892F6AE00E94D69F892F99279F938F93B5
:10165000809102010E94D69F99279F938F9387E9DB
:1016600091E09F938F93CEE8D7E1DF93CF93E09102
:10167000B705F091B80509958DB79EB708968DBF4F
:101680008091F1028823E9F06AE00E94D69F892FB9
:1016900099279F938F938091F1020E94D69F99275B
:1016A0009F938F938CEA91E09F938F93DF93CF93D7
:1016B000E091B705F091B80509958DB79EB70896EA
:1016C0008DBF8091F2028823E9F06AE00E94D69FE4
:1016D000892F99279F938F938091F2020E94D69F22
:1016E00099279F938F938EEB91E09F938F93DF9336
:1016F000CF93E091B705F091B80509958DB79EB7E6
:1017000008968DBFDF91CF910895CFEFD0E4DEBF73
:10171000CDBF88249924C1E07C2E14B815B88AE086
:101720008AB98FE58BB9B7EECB2EB3E0DB2E2EEC6A
:101730003FEFC20ED31ED7FEFACF6624199B08C016
:101740004C9B04C085E18093030108C086E101C081
:1017500089E18093030181E08093110481E887B9D6
:101760003E9A8FEF88B98BE184B981E085B9469ABA
:1017700084B7877F84BF8091600088618093600018
:101780001092600084EC99E09093230380932203ED
:1017900010925F0410925E041092D5091092D40941
:1017A000109261041092600410926304109262041B
:1017B00020910301243128F084EC94E0A0E0B0E013
:1017C00004C08BE095E0A0E0B0E0809343019093EB
:1017D0004401A0934501B09346012898293111F4A2
:1017E000299A01C029980E94CC1B0E949D1B0E942F
:1017F00096170E9496380E94881F81E00E94CB3382
:101800000E94E4700E949E7A86E00E94089C80916B
:101810000301893111F4299A01C0299878940E9412
:10182000B232809103018431E8F488E190E02CE049
:101830000FB6F894A895809360000FBE20936000C7
:1018400084ED91E09F938F938EE897E19F938F9320
:10185000E091B705F091B80509950F900F900F90A2
:101860000F90EECF8091710382608093710310928C
:1018700074030E94D04784EF91E00E94631B6C01C7
:101880008091710380FD05C0C6010E946C1B8823F6
:10189000B9F383EF91E09F938F93AEE8AA2EA7E16F
:1018A000BA2EBF92AF92E091B705F091B8050995B5
:1018B00080EA9FE00E94631B6C01C0E0D0E00F90C3
:1018C0000F900F900F9002E719E0FAEEEF2EF8E07C
:1018D000FF2E0E94D0478091710380FD05C0C60194
:1018E0000E946C1B8823B9F3F70180811816ACF4B1
:1018F0000BC00E94D0478091710380FD05C0C601D6
:101900000E946C1B8823B9F3C6010E946C1B8823BC
:1019100021F4F8018081882364F7F801808187FF32
:1019200019C02196DF93CF93219785E092E09F9392
:101930008F93BF92AF92E091B705F091B8050995EA
:101940008091EA028F5F8093EA022DB73EB72A5F4B
:101950003F4F2DBF219684E090E0E80EF91E085F0E
:101960001F4FCC30D10508F4B4CFC0E0D0E00FE673
:1019700019E0EAEEEE2EE8E0FE2EF801838187FD05
:101980001DC0F70180811816CCF42196DF93CF9308
:10199000219788E092E09F938F938EE897E19F9341
:1019A0008F93E091B705F091B805099582E0809397
:1019B00020032DB73EB72A5F3F4F2DBFF80183812B
:1019C00080788383219624E030E0E20EF31E085FE6
:1019D0001F4FCC30D10588F20E94520A90915A08CC
:1019E0008091EA02981728F48091D1058061809354
:1019F000D105993020F088E080933E0102C0909399
:101A00003E0186E292E09F938F93CEE8D7E1DF9389
:101A1000CF93E091B705F091B805099588EE93E072
:101A20000E94631B6C010E94C61F0F900F900F90C5
:101A30000F90C6010E946C1B8823D9F386E492E0C4
:101A40009F938F93DF93CF93E091B705F091B80503
:101A5000099580E00E94D73C289880ED97E090930C
:101A600023038093220385E58093ED058EE090E0CB
:101A70000E94D2309927182F00278FE090E00E9413
:101A8000D230080F111D1093F0020093EF028AE08C
:101A900090E00E94D2309927182F00278BE090E029
:101AA0000E94D230080F111D1093EE020093ED0238
:101AB0000F900F900F900F900F5F1F4F39F0809194
:101AC000EF029091F0028F5F9F4F41F41092F0026D
:101AD0001092EF021092EE021092ED028091ED0250
:101AE0009091EE029F938F938091EF029091F0027C
:101AF0009F938F938BE492E09F938F93DF93CF9389
:101B0000E091B705F091B80509950E949E2588E8F7
:101B100093E190933D0180933C01C1E0C093EC05BB
:101B20008C2F0E94920A809182080E94549B0E94EE
:101B3000520A80ED97E00E94631B6C018AEF90E0EF
:101B40000E94631B83E08093B4071092E9028091A6
:101B5000CE082DB73EB7285F3F4F2DBF84FF02C090
:101B6000C093F30212BC11BC8091F502882311F0DE
:101B70004798FECF80912603882309F4A6C280915E
:101B80001801882309F4A1C2F8948091260381509A
:101B90008093260378948091EB05882319F00E94A6
:101BA000640A02C00E94964B0E94D04728988091F8
:101BB0005204882331F08091520481508093520462
:101BC0000EC080916F00806280936F001092D109E7
:101BD0001092D0098091D10588608093D1058091C1
:101BE0003C0190913D01019790933D0180933C0110
:101BF00080913C0190913D01892B21F080917203ED
:101C00008823C9F180913C0190913D01892BD9F441
:101C10000E94F53385E090E090933D0180933C0174
:101C20008091EE079091EF0701969093EF078093D4
:101C3000EE078091D10581608093D1058091B50731
:101C400082608093B50780910B0190910C018F5FAA
:101C50009F4F91F480915104882371F088EA91E6B6
:101C6000909323038093220380E890E090930C01EB
:101C700080930B0101C028980E94069D8091260345
:101C8000882309F020C280917305882319F00E94EF
:101C9000088E19C280912103882311F40E940571D6
:101CA00080911101882311F00E94261C0E94E017E8
:101CB0000E940113C6010E946C1B882309F4FFC116
:101CC00084E190E0C80ED91E0E94E41B8091820836
:101CD000863019F40E94B28004C0843011F40E944E
:101CE000D88E80911104882331F18091FB07909167
:101CF000FC078C52914074F08091C4079091C50705
:101D000080509240C4F48091FB079091FC0783556A
:101D100093408CF0639432E3361570F48091510453
:101D2000882331F08091D00580628093D00504C073
:101D300080933D0401C0662480917203882329F4B6
:101D40008091540B8E3150F405C08091D105826092
:101D50008093D1058091B50782600FC080912203E6
:101D600090912303892B59F480913C0190913D017E
:101D7000079728F08091B5078D7F8093B5078091F4
:101D8000F302882361F080915204873940F0109269
:101D9000F30288E893E190932303809322038091D8
:101DA0000601882321F08150809306012EC0809384
:101DB000F705109225041092240410922304109227
:101DC000220410922104109220048091520488234E
:101DD000E1F480910B0190910C018F5F9F4FA9F46A
:101DE0002091F302223089F088E99AE3909323034B
:101DF0008093220380E09CE090930C0180930B0180
:101E0000222319F082E08093F3028091A501893C9E
:101E100070F081508093A5018091D1058B7F8093D4
:101E2000D1058091D40581608093D40551C0809103
:101E3000D60A8823F9F08091D10584608093D1057A
:101E400089E08093330580910B0190910C018F5FA5
:101E50009F4F81F480915104882361F088E99AE3CF
:101E6000909323038093220380E098EA90930C01DF
:101E700080930B01109225051092240510922305E2
:101E800010922205109221051092C90A8FEF8093BB
:101E90003E0B1092080B1092070B10920A0B109237
:101EA000090B8FEF9FEF9093060B8093050B109219
:101EB0004104109242041092430410924404109280
:101EC00045048091D4058E7F8093D4051092A5019E
:101ED00060910201262F33278091260190912701DE
:101EE00028173907F4F0809119048062809319044F
:101EF00080910B0190910C018F5F9F4F91F4809125
:101F00002601909127010B9764F080E797E1909369
:101F100023038093220380E093E090930C0180934D
:101F20000B0112BC11BC8091F4028F5F8093F4020C
:101F3000813309F07BC01092F40280915905882307
:101F400019F08150809359058091190481FF0AC0CE
:101F50008091EB029091EC0201969093EC028093B9
:101F6000EB0204C05AEA852E55E0952E80911A04A2
:101F700090911B048050944008F049C02091FD07C7
:101F80003091FE074091FF075091000880911E019B
:101F900090911F01A0912001B091210128173907CC
:101FA0004A075B0764F48091FD079091FE07A091BA
:101FB000FF07B09100080596A11DB11D20C020911A
:101FC000FD073091FE074091FF0750910008809176
:101FD0001E0190911F01A0912001B0912101821753
:101FE0009307A407B5079CF48091FD079091FE0725
:101FF000A091FF07B09100080597A109B10980934E
:10200000FD079093FE07A093FF07B0930008862F6B
:102010009927019620912601309127018217930775
:102020002CF4809119048F7D809319040894811CED
:10203000911C82E788168BE0980609F040C088243E
:1020400099242091EF023091F0022F5F3F4F30939F
:10205000F0022093EF028091ED029091EE02019642
:102060009093EE028093ED02832F9927682F8EE0E4
:1020700090E00E94DA308091EF029091F00290702F
:10208000682F8FE090E00E94DA308091ED0290910D
:10209000EE02892F9927682F8AE090E00E94DA30BB
:1020A0008091ED029091EE029070682F8BE090E0AD
:1020B0000E94DA3084E190E00E94631B6C010E9470
:1020C00040760E94D67A71107A94772039F40E9473
:1020D0000476882319F08CE0782E46CD8091210378
:1020E000882309F041CD0E9405713ECD1F920F92C9
:1020F0000FB60F9211248F939F93EF93FF938091CC
:1021000008018823E1F480910F0390911003019658
:102110009093100380930F03FC01E852F94FE08184
:10212000ED3019F08C3D910539F4109210031092A6
:102130000F0381E080930801E093C60004C0109271
:10214000100310920F03FF91EF919F918F910F90C9
:102150000FBE0F901F9018951F920F920FB60F92FF
:1021600011242F933F934F935F936F937F938F939C
:102170009F93AF93BF93CF93EF93FF9390E08091A2
:10218000F502813029F48091C6008093CE00D1C041
:102190008091F502823029F48091C6008093FA057F
:1021A000C8C08091C60080930703509115035C3D21
:1021B00010F090931603809107038D3009F06AC0E8
:1021C00080911603823009F065C090931603852F25
:1021D000992786509A4FFC01329740812091110334
:1021E00030911203241B3109DC0111978C91281BBB
:1021F0003109C9019F70909312038093110346E047
:10220000969587954A95E1F7982F935C90931303E1
:102210002F733070235C209314038081981729F466
:102220008C91281711F491E006C090E0809104038E
:102230008F5F8093040380910603882309F079C09F
:10224000992309F476C081E080930603580F5093D8
:1022500003035150E52FFF27E650FA4F8DE08083AE
:102260008091FC05823509F064C0C0915104CC23F3
:1022700009F05FC00E949E2588E190E02CE00FB637
:10228000F894A895809360000FBE20936000C093DF
:1022900020034FC020911603822F9927813091058A
:1022A000F9F0823091051CF4892B21F040C002978F
:1022B00011F13DC080910703833239F48091060308
:1022C000882319F481E0809316038091070380939B
:1022D000FA0581E08093150380910703992722C0B6
:1022E0002F5F20931603E52FFF27E650FA4F8091CA
:1022F0000703808309C0E52FFF27E650FA4F80913E
:10230000070380835C3D20F45F5F5093150302C098
:1023100010921603209107038091110390911203EC
:10232000820F911D909312038093110302C01092AB
:102330001603FF91EF91CF91BF91AF919F918F9134
:102340007F916F915F914F913F912F910F900FBEB1
:102350000F901F901895AC01A0E0B0E09D01A81768
:10236000B90748F4E8EDF6E08191280F311D119688
:10237000A417B507C8F33F70FD01E852F94FC90132
:1023800056E0969587955A95E1F7835C8083119680
:10239000FD01E852F94F2F733070822F835C8083E8
:1023A000A752B94F8DE08C93109208018091D80606
:1023B0008093C6000895A0E0B0E0E1EEF1E10C9456
:1023C0004FA02C859D850E85BB2483E28093D80683
:1023D0009F599093D9062093DA0633E0E32EF12C2F
:1023E000002309F49EC0CF84D888BE016D5E7F4F64
:1023F000A989BA890150109709F493C01097B9F0D0
:10240000F601EB0DF11DB3949081119791F4002327
:1024100049F1FB016E5F7F4FDB01C080D1806E5FB1
:102420007F4F0D90BC91A02DBB24015002C090E0C5
:1024300019C01097B9F0F601EB0DF11DB39440816E
:10244000119791F4002341F1FB016E5F7F4FDB0197
:10245000C080D1806E5F7F4F0D90BC91A02DBB24BA
:10246000015002C040E018C01097B1F0F601EB0D2A
:10247000F11DB3941081119781F4002371F0FB01D9
:102480003296DB01CD90DC90BF016E5F7F4FA08163
:10249000B181BB24015001C010E0F701E852F94FAF
:1024A000892F86958695835C80830894E11CF11CB6
:1024B000F701E852F94F892F99278370907024E033
:1024C000880F991F2A95E1F755279A0194E03695D0
:1024D00027959A95E1F7822B835C80830894E11C11
:1024E000F11CF701E852F94F4F705070440F551F1F
:1024F000440F551F812F992726E0969587952A9599
:10250000E1F7842B835C80830894E11CF11CF701C4
:10251000E852F94F1F73135C10830894E11CF11CFF
:102520006ACFC7010E94AB11E9E00C946BA0A3E055
:102530007A2F409103034650442309F458C0E72FF3
:10254000FF27E650FA4F80818D537F5FE72FFF27EB
:10255000E650FA4F20812D537F5FE72FFF27E6508B
:10256000FA4F30813D537F5FE72FFF27E650FA4F48
:1025700060816D537F5F9927880F991F880F991F7E
:10258000522F52955F70582B822F99278F70907021
:10259000F4E0880F991FFA95E1F7232F26952695E9
:1025A000282B832F992783709070E6E0880F991F5E
:1025B000EA95E1F7682B41504F3FC9F0EA2FFF271A
:1025C000E650FA4F5083AF5F41504F3F81F0EA2F02
:1025D000FF27E650FA4F2083AF5F41504F3F39F05D
:1025E000EA2FFF27E650FA4F6083AF5FA5CF8DEF4C
:1025F00095E09093020380930103A350A0930003FE
:102600000895A2E0B0E0E7E0F3E10C9455A08091DA
:102610000603882309F47EC40E9497128091FB056B
:10262000823609F0E4C28091FC0599278037910534
:1026300009F4AFC081379105C4F48A36910509F4D5
:1026400041C28B36910544F48B34910571F1863685
:10265000910509F46AC1CBC28D36910509F469C0B0
:102660008E36910509F44DC0C2C28437910541F1FF
:10267000853791054CF48137910509F491C0833772
:10268000910509F4EAC0B3C28737910509F4DCC1AA
:10269000883791052CF48537910509F498C1A7C2B4
:1026A0008937910509F47DC1A2C2E0910103F0913F
:1026B000020380819181909392018093910197C24E
:1026C00080910303A0910103B0910203853140F092
:1026D00080E1E5EDF5E00D9001928A95E1F70DC0FE
:1026E0008D919D910D90BC91A02D8093D5059093D7
:1026F000D605A093D705B093D80580EF8093FE024E
:102700004BC0809108018823E1F38DE490E09F9312
:102710008F938DED98E09F938F9381E08F938F93AC
:102720008EE48F930E94DB118DB79EB707968DBF05
:102730005EC2A0910103B09102031C91113081F49B
:102740008DE4EDEDF8E00D9001928A95E1F70E949D
:10275000ED3119838091D1058F7E8093D10501C021
:102760001982809108018823E1F381E090E09F9332
:102770008F93CE0101969F938F9381E08F938F93D8
:102780008DE48F930E94DB11ADB7BEB71796ADBF36
:102790002EC281E0809309038FEF8093060127C248
:1027A000809151048823E1F5E0910103F091020347
:1027B000E0818E2F8A508A3058F48983882311F45F
:1027C00081E003C0863010F085E0898361E00EC0AF
:1027D0008E2F84518A3070F48983882311F481E02C
:1027E00003C0863010F085E0898360E089810E9413
:1027F0006F3212C0E983EF3F19F40E94503289838F
:102800008981882311F481E003C0863010F085E0CF
:10281000898389810E94F03080E00E94920A03C07F
:102820000E9450328983809108018823E1F381E876
:1028300090E09F938F938BE598E09F938F9381E037
:1028400090E09F938F93CE0101969F938F9382E0A8
:102850008F9381E08F9381E52DC120910103309109
:102860000203D9018C918150853008F045C0F901EF
:102870008181823609F040C0809151048823E1F5BE
:102880002F5F3F4F81E8EBE5F8E0D9010D90019211
:102890008A95E1F7F90182910E945D3180919C084F
:1028A0009927AA27BB27BC01CD0124EC39E040E0E1
:1028B00050E00E94B79FDC01CB0180938901909387
:1028C0008A01A0938B01B0938C0180919D08992778
:1028D000AA27BB27BC01CD010E94B79FDC01CB0119
:1028E0008093850190938601A0938701B09388011E
:1028F0000E945032898301C0198280910801882387
:10290000E1F381E090E09F938F93CE0101969F9336
:102910008F9381E08F938F9383E58F930E94DB11D8
:102920008DB79EB707968DBF2BC080915104882329
:1029300009F05DC1E0910103F0910203E0818E2F67
:102940008150853018F48E2F0E94F0300E94503252
:102950008983809108018823E1F381E090E09F93CF
:102960008F93CE0101969F938F9381E08F938F93E6
:1029700086E48F930E94DB11ADB7BEB71796ADBF4B
:1029800010915104112341F46EE670E089810E9498
:10299000FD3B812F0E94920A809182080E94549BE5
:1029A00026C119822981A0910103B0910203E0EDB3
:1029B000F9E08D91992787FD909593A382A3822FAB
:1029C0008F5F8983282F32968C3098F310C1E09165
:1029D0000103F091020380810E94EC378A838823EF
:1029E00019F481E0898301C019828091080188234C
:1029F000E1F388E090E09F938F9387E699E09F93BF
:102A00008F9321E030E03F932F93809101039091C9
:102A100002039F938F933F932F93CE0102969F9330
:102A20008F933F932F93CE01820F931F9F938F938A
:102A300084E08F9381E08F9385E58F930E94DB1173
:102A4000EDB7FEB773963CC080910003893008F45F
:102A5000CEC020910103309102032F5F3F4F88E0E9
:102A6000A7E6B9E0F90101900D928A95E1F7D90145
:102A70008E910E943F378A83882319F481E08983ED
:102A800001C01982809108018823E1F321E030E040
:102A90003F932F93CE0102969F938F933F932F9353
:102AA000CE01820F931F9F938F9382E08F9381E0DB
:102AB0008F9387E58F930E94DB11EDB7FEB73B96AE
:102AC000EDBF95C080915104882309F090C00E9409
:102AD0000B9B8983823019F0843009F088C020E490
:102AE00030E0F8948091C1008F738093C100809191
:102AF000C9008F738093C9008091C100877E809345
:102B0000C1008091C900877E8093C9008091C80070
:102B100087FF03C08091CE00F9CF8091C00087FF6E
:102B200003C08091C600F9CFE0910103F091020348
:102B3000E081E13021F482E08093F5022EC0E4369A
:102B400011F421E830E081E08093F502832F99278A
:102B50008093CD002093CC008091CD008093C50060
:102B60008091CC008093C4008091CA008F7D8093B7
:102B7000CA008091CA008F7E8093CA008091C900EC
:102B80008B7F8093C9008091CA0084608093CA00C3
:102B90008091CA0082608093CA008091CA00877FBA
:102BA0008093CA008091C200877F8093C200809189
:102BB000C9008E7F8093C9008091C1008861809395
:102BC000C1008091C90088618093C9008091C100D3
:102BD00080688093C1008091C90080688093C9009B
:102BE00010926E0010926F00109270007894809195
:102BF000FC0599278436910509F421C18536910594
:102C0000C4F48136910509F4D5C08236910544F4A7
:102C10008F33910539F18B34910509F4C0C072C12D
:102C20008236910509F4D3C08336910509F4E2C0D8
:102C300069C18C36910509F450C18D3691054CF46B
:102C40008736910509F45BC18836910509F415C1F1
:102C500059C18437910509F467C08637910509F495
:102C60004AC150C12091FB052C5629832C3008F015
:102C700049C1822F9927BC01660F771F660F771F06
:102C8000680F791F655D764F4091010350910203F3
:102C900085E0DB01FA0101900D928A95E1F7DB01F5
:102CA0008C9180FF0BC080911703909118030097BF
:102CB00029F001979093180380931703822F992787
:102CC000FC01EE0FFF1FEE0FFF1FE80FF91FE55D80
:102CD000F64F808182FF26C08091170390911803E0
:102CE000892BC9F4299A10927404109275041092D9
:102CF000760410927704109270041092710410926E
:102D000072041092730410927C0410927D0410924D
:102D10007E0410927F0484EF91E0909318038093D7
:102D20001703F0C02998EEC080910303A09101031E
:102D3000B0910203803140F080E1E5EDF5E00D90C7
:102D400001928A95E1F70DC08D919D910D90BC91F6
:102D5000A02D8093D5059093D605A093D705B09369
:102D6000D805809108018823E1F31F928091050125
:102D70008F9384E58F930E94DB118AEF8093FE028C
:102D80008FEF8093060180EA9FE00E94631B90937F
:102D9000F7028093F6020F900F900F90B3C0E0916E
:102DA0000103F091020380819181909392018093BD
:102DB0009101A8C0E0910103F0910203808180930A
:102DC0000701803298F08FE1809307010FC0A09136
:102DD0000103B09102038BE0EDEEF5E00D9001925E
:102DE0008A95E1F78091F6058093F6078FEF80933F
:102DF000060188C08091FA029091FB02892B89F428
:102E0000E0910103F0910203E081EE2351F08AE0AA
:102E1000E89FC00111240E94631B9093C805809312
:102E2000C705E0910103F091020390818AE0989F29
:102E3000C00111249093FB028093FA0215C08FEF1A
:102E400080930601E0910103F091020390818AE0F2
:102E5000989FC00111249093FD028093FC02892B5E
:102E600019F081E080930B0380EA9FE00E94631BCE
:102E70009093F7028093F60245C08FEF809306018E
:102E8000E0910103F0910203908197FD08C082E078
:102E9000809308031092F9021092F8021AC09095DC
:102EA00080916A03892B80936A0391818AE0989FBD
:102EB000C00111249093F9028093F80284E080937A
:102EC000080380EA9FE00E94631B9093F7028093BF
:102ED000F60281E080930C0315C08FEF809306010A
:102EE000E0910103F0910203808180936B0381E004
:102EF00080930D0307C081E080930A0303C081E043
:102F000080930E03109206031092020310920103A5
:102F100010920003E3E0CE5F0C9471A0982F809193
:102F2000C00085FFFCCF9093C60008950F931F93B8
:102F300088E18093C1008091C00082608093C000CE
:102F40008091C10080688093C1008091C10080643D
:102F50008093C10000E010E00093C5008AE290E099
:102F60008093C4008091FC029091FD020E94631B3B
:102F70009093CA058093C9058CED90E00E94631B75
:102F80009093F9058093F80582E08093CB0584E067
:102F90008093CC051092CF058BE08093CD051092E5
:102FA000CE051092D305809103018093D205109332
:102FB000020300930103109200031F910F910895E3
:102FC000A0E1B0E0E6EEF7E10C9454A08091080196
:102FD000882309F48CC28091F6029091F7020E9436
:102FE0006C1B882361F01092F9021092F802109283
:102FF000FD021092FC021092FB021092FA028091E4
:10300000F8029091F902892B41F08091D6069091B7
:10301000D7060E946C1B882329F480910C03882317
:1030200009F460C080910801882309F45BC0809195
:1030300008030AE018E08430A8F00E94B42580E577
:1030400090E09F938F931F930F9381E08F938F93C3
:1030500088E48F930E94DB112DB73EB7295F3F4F65
:103060002DBF34C010926C038DE694E09F938F9334
:1030700087EA95E29F938F93E091B705F091B805A9
:10308000099584E190E09F938F931F930F9381E0C4
:1030900090E09F938F9388E093E09F938F9382E0DB
:1030A0008F9381E08F9388E48F930E94DB1180914E
:1030B0000803982F8F5F809308032DB73EB7215FD9
:1030C0003F4F2DBF943010F0109208038091F8020A
:1030D0009091F9020E94631B9093D7068093D606C5
:1030E00010920C0380910D03882351F18091080107
:1030F000882331F10E94B42580E590E09F938F935F
:103100008AE098E09F938F9321E030E03F932F93E4
:1031100088E291E09F938F933F932F938BE693E008
:103120009F938F9383E08F9381E08F938CE48F93B1
:103130000E94DB1110920D038DB79EB70F968DBFC5
:1031400080910A038823D1F0809108018823B1F08F
:103150008AE090E09F938F938BEC95E09F938F9301
:1031600081E08F938F9386E58F930E94DB111092FD
:103170000A032DB73EB7295F3F4F2DBF80910E0345
:103180008823D9F0809108018823B9F08BE090E082
:103190009F938F938DEE95E09F938F9381E08F9314
:1031A000809105018F9387E48F930E94DB11109229
:1031B0000E038DB79EB707968DBF8091FC0290914C
:1031C000FD02892B41F08091C9059091CA050E94AA
:1031D0006C1B882321F480910B03882341F180919B
:1031E0000801882321F10E94073B82E490E09F932D
:1031F0008F9384EB97E09F938F9381E08F938F93CE
:1032000084E48F930E94DB1110920B032DB73EB71D
:10321000295F3F4F2DBF8091FC029091FD020097E6
:1032200031F00E94631B9093CA058093C905809179
:10323000FA029091FB02892B09F497C08091C7058F
:103240009091C8050E946C1B882309F48EC0809160
:103250000801882309F489C08091DC0A9091DD0A75
:103260009093BA058093B9058091DE0A9091DF0AA8
:103270009093BC058093BB052091BE0A3091BF0A94
:103280004091C00A5091C10ADA01C901F3E0880FE8
:10329000991FAA1FBB1FFA95D1F7820F931FA41F76
:1032A000B51F820F931FA41FB51F209143013091BA
:1032B00044014091450150914601BC01CD010E945D
:1032C0002BA03093BE052093BD058091740490918E
:1032D0007504A0917604B0917704E9E0B595A795BF
:1032E00097958795EA95D1F78093BF0580917004F3
:1032F00090917104A0917204B091730479E0B59536
:10330000A795979587957A95D1F78093C005809179
:103310007C0490917D04A0917E04B0917F0469E0CB
:10332000B595A795979587956A95D1F78093C1052F
:103330008EE090E09F938F9389EB95E09F938F931E
:1033400081E08F938F9383E48F930E94DB118091B0
:10335000FA029091FB020E94631B9093C805809330
:10336000C7058DB79EB707968DBF809107018F3F28
:1033700079F1992754E0880F991F5A95E1F78359FD
:103380009D4F40E150E0BC01CE0101960E94019E9C
:1033900080E190E09F938F93CE0101969F938F934E
:1033A00081E090E09F938F9387E091E09F938F93CC
:1033B00082E08F9381E08F9381E48F930E94DB11F1
:1033C0008FEF809307012DB73EB7255F3F4F2DBF8D
:1033D0008091F6078823C9F0809108018823A9F01D
:1033E00081E090E09F938F9386EF97E09F938F9378
:1033F00081E08F938F9382E48F930E94DB11109270
:10340000F6078DB79EB707968DBF80910903882375
:10341000D1F0809108018823B1F086E490E09F9379
:103420008F9380ED99E09F938F9381E08F938F939B
:1034300080E58F930E94DB11109209032DB73EB7F0
:10344000295F3F4F2DBF8091F8059091F9050E94AB
:103450006C1B882309F44BC080910801882309F470
:1034600046C08091A501882361F58091DC0A909186
:10347000DD0A9093E6058093E5058091DE0A909140
:10348000DF0A9093E8058093E70580912E048093EE
:10349000E90580912D048093EA0588E090E09F93F0
:1034A0008F9385EE95E09F938F9381E08F9383E0D8
:1034B0008F938BE68F930E94DB118DB79EB7079693
:1034C0008DBF8091EB05853018F086E08093EB0589
:1034D00080911F03882319F083E690E002C087EEF5
:1034E00093E00E94631B9093F9058093F805E4E054
:1034F000C05F0C9470A01F920F920FB60F92112410
:103500002F933F935F936F937F938F939F93AF938B
:10351000BF93EF93FF9380912103882329F080913B
:10352000210381508093210380914805882319F05D
:10353000815080934805809129038150809329030D
:103540008F3F09F051C089E08093290380912703C0
:1035500090912803019690932803809327038091EC
:1035600012018F5F817080931201882349F480914A
:103570002603843028F4809126038F5F80932603EE
:10358000349903C081E080931F03809122039091BE
:103590002303892B11F180912203909123030B9730
:1035A00050F080912203909123030A979093230374
:1035B0008093220304C0109223031092220380916F
:1035C00022039091230320910B0130910C0182235F
:1035D0009323892B41F0479A07C08FEF9FEF909379
:1035E0000C0180930B01479880911F03882309F4F5
:1035F0005AC02091A501222309F055C08091AE0A3E
:1036000083FF51C086B19927FC01E071F07084FFFF
:1036100013C0809124039091250301969093250374
:10362000809324038091240390912503895E934025
:10363000D0F120931F0337C080912403909125037C
:10364000892B69F180912403909125038A5691403A
:1036500030F5809124039091250369E270E00E9487
:10366000E29F8091240390912503860F971F9093EA
:1036700025038093240380912403909125030B97C5
:1036800050F080912403909125030A979093920122
:103690008093910104C0F0939201E0939101109204
:1036A000250310922403FF91EF91BF91AF919F9159
:1036B0008F917F916F915F913F912F910F900FBEEE
:1036C0000F901F9018952091270330912803280F01
:1036D000391FC901019608952091270330912803CD
:1036E000821B930B892F992786958074907008957B
:1036F000CF93DF930E94631BEC01CE010E946C1BF1
:103700008823D9F3DF91CF910895CF93DF930E945F
:10371000631BEC0109C080911801882329F0909364
:1037200018018FEC80937A00CE010E946C1B982FB9
:10373000882389F3DF91CF9108959FB7F8945F981C
:103740003E9A469A8091B0008F708093B00080912D
:10375000B00083608093B0008091B1008B73809340
:10376000B1008091B1008B608093B1001092B200E3
:103770008FEF8093B3008091B00080688093B00099
:10378000809170008A7F80937000809170008260C9
:10379000809370009FBF08958AE090E00E94631BB1
:1037A0009093F8078093F70782E085BD83EB84BD93
:1037B0008FEF88BD84EB87BD86E086BD80916E006B
:1037C000816080936E0008958091CD0820917001F2
:1037D00082FF30C090918B088CE3989FB001112438
:1037E00090918A0880E5989FA0011124922F90580B
:1037F00097FD9D5F9595959586E09802C0011124EF
:103800002091090130910A01281B390B30930A01DC
:1038100020930901421753072CF050930A0140935B
:10382000090108952617370784F070930A01609301
:1038300009010895822F992736E0880F991F3A953C
:10384000E1F790930A01809309010895EF92FF92A6
:103850000F931F93CF93DF9380919208E82FFF2758
:10386000E75BFE4F9681C08180911101813009F0A4
:1038700021C18091CF0887FF05C0C0E0D0E0E0E023
:10388000F0E046C0892F992787FD9095A92FB92F81
:103890002091AC043091AD044091AE045091AF043E
:1038A000BC01CD010E94B79F97FF04C061587F4FB4
:1038B0008F4F9F4F7B018C0187E015950795F794FB
:1038C000E7948A95D1F78C2F992787FD9095A92F9A
:1038D000B92F2091A4043091A5044091A6045091E1
:1038E000A704BC01CD010E94B79F97FF04C0615897
:1038F0007F4F8F4F9F4FB7E0959587957795679549
:10390000BA95D1F7F801E701C61BD70BE80BF90B05
:1039100020912C0530912D05C901A3E0880F991F36
:10392000AA95E1F7821B930BAA2797FDA095BA2FC2
:10393000C81BD90BEA0BFB0B80916E019927AA27B4
:10394000BB27BC01CD019E01AF010E94B79F97FF2D
:1039500004C061507E4F8F4F9F4FFC01EB0179E017
:10396000F595E795D795C7957A95D1F71091CD083C
:103970006091090170910A0112FF05C07093100156
:1039800060930F0118C040910F0150911001809178
:103990009108282F3327CB01841B950BB9010E9476
:1039A000F69F80910F0190911001860F971F9093C1
:1039B000100180930F0110FF14C080910F019091AE
:1039C000100197FD0F9664E0959587956A95E1F74C
:1039D000AA2797FDA095BA2FC80FD91FEA1FFB1F72
:1039E00015C080910F019091100197FD0F9654E042
:1039F000959587955A95E1F7AA2797FDA095BA2F37
:103A00008C1B9D0BAE0BBF0BFD01EC012091C5087B
:103A1000222321F1332780911B0390911C03829F65
:103A2000A001839F500D929F500D1124CA01AA2717
:103A300097FDA095BA2F8C0F9D1FAE1FBF1F2F5F44
:103A40003F4F442737FD4095542FBC01CD010E94C4
:103A50002BA030931C0320931B0304C0D0931C03A2
:103A6000C0931B0380918A08282F3327220F331F0E
:103A7000220F331F80911B0390911C038217930721
:103A80007CF080918B08282F3327220F331F220FC1
:103A9000331F80911B0390911C032817390724F4CE
:103AA00030931C0320931B03809111018F5F80933F
:103AB0001101F9C0892F992787FD9095A92FB92F5A
:103AC0002091A4043091A5044091A6045091A7042C
:103AD000BC01CD010E94B79F97FF04C061587F4F82
:103AE0008F4F9F4F7B018C0187E015950795F794C9
:103AF000E7948A95D1F78C2F992787FD9095A92F68
:103B0000B92F2091AC043091AD044091AE04509196
:103B1000AF04BC01CD010E94B79F9B01AC0197FF90
:103B200004C021583F4F4F4F5F4FC7E05595479511
:103B300037952795CA95D1F72E0D3F1D401F511F70
:103B400080916D019927AA27BB27BC01CD010E9456
:103B5000B79F97FF04C061507E4F8F4F9F4FFC016E
:103B6000EB01B9E0F595E795D795C795BA95D1F7EB
:103B700080916F019927A6E0880F991FAA95E1F718
:103B800040910D0150910E01209191083327841B23
:103B9000950BB9010E94F69F80910D0190910E0145
:103BA000860F971F90930E0180930D018091CD0891
:103BB00081FF14C080910D0190910E0197FD0F9629
:103BC00074E0959587957A95E1F7AA2797FDA095DA
:103BD000BA2FC80FD91FEA1FFB1F15C080910D0116
:103BE00090910E0197FD0F9664E0959587956A95E3
:103BF000E1F7AA2797FDA095BA2F8C1B9D0BAE0B62
:103C0000BF0BFD01EC012091C608222321F13327CF
:103C10008091190390911A03829FA001839F500DF8
:103C2000929F500D1124CA01AA2797FDA095BA2F83
:103C30008C0F9D1FAE1FBF1F2F5F3F4F442737FDC7
:103C40004095542FBC01CD010E942BA030931A0344
:103C50002093190304C0D0931A03C09319038091D1
:103C60008E08282F3327220F331F220F331F8091F6
:103C7000190390911A03821793077CF080918F08A3
:103C8000282F3327220F331F220F331F8091190350
:103C900090911A032817390724F430931A032093BC
:103CA000190310921101E6E0CDB7DEB70C946EA0B7
:103CB0001F920F920FB60F9211242F933F934F93A1
:103CC0005F938F939F93EF93FF9380912A038823B1
:103CD00009F0DDC08091B00086FF9FC08091B000E8
:103CE0008F7B8093B000E0912D0320919008EE230C
:103CF000D9F433278DED96E0289FA001299F500D20
:103D0000389F500D1124CA0120912B0330912C03B0
:103D1000821B930B90931E0380931D0310922C0320
:103D200010922B03469AB0C02E1738F48AE090E028
:103D300090931E0380931D03A7C089EA93E090939C
:103D40001E0380931D038E2F992783309105D9F090
:103D50008430910534F48130910549F0029761F087
:103D600020C08430910591F0059799F01AC0809198
:103D70001B0390911C0304C08091190390911A03B6
:103D800087559E4F1DC08091890A05C08091620AA7
:103D900002C08091920A9927880F991F880F991F56
:103DA000EFCFFF27EE0FFF1FE053F64F2081318149
:103DB000220F331F80911D0390911E03820F931FCA
:103DC00090931E0380931D0380911D0390911E0309
:103DD00055E08D3D950718F08CED95E005C08757AF
:103DE000914030F487E791E090931E0380931D0388
:103DF00020911D0330911E032C5B304030931E0335
:103E000020931D0380912B0390912C03820F931F0D
:103E100090932C0380932B0337C08091B000806473
:103E20008093B0008CEB90E090931E0380931D0371
:103E300080912B0390912C0384549F4F90932C03DB
:103E400080932B0380912003882321F080915204DA
:103E5000882321F480912003823011F4469801C018
:103E6000469A80912D038F5F80932D03282F33274F
:103E70008091900899270196821793072CF481E08E
:103E80008093110110922D0381E080932A032091E9
:103E90001D0330911E0341E02F37340730F08FEFC0
:103EA0008093B3002F5F30400FC02F3F3105C9F022
:103EB000C0F0A9014F5F50404F37510550F480E8E2
:103EC0008093B3002058304030931E0320931D038D
:103ED00012C08FEF8093B30050931E0340931D03D5
:103EE0000AC080911D038093B30010921E031092AC
:103EF0001D0310922A03FF91EF919F918F915F9183
:103F00004F913F912F910F900FBE0F901F901895DA
:103F100010927C008FEC80937A00089580911104B8
:103F2000609116017091170120913A03882379F06E
:103F3000CB01AA27BB27332727FD3095432F532FCB
:103F4000BC01CD010E94B79FDC01CB0116C084E00B
:103F5000660F771F8A95E1F7CB01AA27BB27332786
:103F600027FD3095432F532FBC01CD010E94B79FF1
:103F7000DC01CB010497A109B1098093320390932E
:103F80003303A0933403B09335030895CF93DF93A5
:103F900010923A030E948E1F83E090E00E94D2307C
:103FA000C82FDD27C03FD10508F42A96C7BD8C2F46
:103FB000809588BD86E990E00E94851B80911C0158
:103FC00090911D018152934010F0C0EFD0E0C630B7
:103FD000D10510F1C7BD8C2F809588BD84E690E097
:103FE0000E94851B82E894E09F938F938EE897E16F
:103FF0009F938F93E091B705F091B8050995809153
:104000001C0190911D010F900F900F900F90815205
:10401000934010F42197DBCFC09307086C2F83E007
:1040200090E00E94DA308091680880FF0AC0809199
:1040300007088A508C3D28F08091D00580648093D9
:10404000D00580E180931501809111048823E9F067
:1040500080910301873150F4CC38D105B0F480EA67
:1040600090E08C1B9D0B6AE170E009C0CA3AD10553
:1040700060F48CEB90E08C1B9D0B63E170E00E9480
:10408000E29FCB01805F8093150180911501282F5D
:10409000332780911C0190911D01829FA001839F75
:1040A000500D929F500D1124CA01AA27BB2780935F
:1040B0001E0190931F01A0932001B09321018CE277
:1040C00091E00E94851BDF91CF9108951F920F927E
:1040D0000FB60F921124EF92FF920F931F932F931D
:1040E0003F934F935F936F937F938F939F93AF9380
:1040F000BF93CF93DF93EF93FF9380915203282FC9
:104100003327442755278F5F80935203F9012231CB
:10411000310508F0ECC4EA5BFF4F0C947DA0809160
:1041200078009091790046C0809178009091790054
:10413000EBC1809178009091790090935603809321
:104140005503FBC18091B6049091B704209178008B
:1041500030917900821B930B9093FA078093F907B3
:104160008091F9079091FA079093600380935F0321
:1041700003C280917800909179002091B804309129
:10418000B904821B930B90930608809305088091D5
:104190000508909106089093620380936103A9C477
:1041A0008091590390915A032091780030917900C1
:1041B000820F931F90935A038093590381E09AC40E
:1041C00080915703909158032091780030917900A5
:1041D000820F931F909358038093570384E08AC4FF
:1041E0008091CE0883FF26C08091260190912701FF
:1041F0009C01220F331F280F391F409178005091E6
:1042000079008BE090E0489FB001499F700D589F66
:10421000700D1124CB016EE170E00E94E29F260F29
:10422000371F36952795369527953093270120938C
:10423000260142C08091680390916903892B91F413
:104240002091780030917900C90153E0880F991FBF
:104250005A95E1F7820F931F820F931F9093690382
:10426000809368032091780030917900C90143E080
:10427000880F991F4A95E1F7820F931F820F931FB2
:1042800020916803309169038217930718F02E5F1D
:104290003F4F02C02250304030936903209368039F
:1042A00080916803909169036FE170E00E94E29F42
:1042B000709327016093260185E01CC480917800EB
:1042C000909179009093FC078093FB078091FB0706
:1042D0009091FC074091B2045091B304841B950B5C
:1042E0006091B104262F332727FD3095821B930B55
:1042F0009093400380933F0380911104882309F039
:1043000071C080913F039091400302977CF172E06D
:104310004E3E57070CF0A7C0209153033091540331
:104320002B5F3F4F3093540320935303255030406D
:1043300080911A0490911B04845F914030F4215FB6
:104340003F4F309354032093530380915303909134
:104350005403853691050CF486C04F5F5F4F509330
:10436000B3044093B2048456904037C080913F0319
:10437000909140038F5F9F4F0CF075C082E04732F1
:1043800058070CF470C0209153033091540325500A
:10439000304030935403209353032B5F3F4F809161
:1043A0001A0490911B04845F914030F42F503040E8
:1043B00030935403209353038091530390915403FB
:1043C0007FEF8C3997070CF04EC04150504050930E
:1043D000B3044093B2048C599F4F9093540380933D
:1043E000530341C080917E0A90917F0A8F5C9F4168
:1043F000D4F180913F03909140030297ACF020915B
:10440000530330915403C901019690935403809350
:104410005303895893413CF166301CF46F5F6093FD
:10442000B104275833411BC080913F039091400352
:104430008F5F9F4FC4F42091530330915403C901FF
:104440000197909354038093530388579C4E5CF4D8
:104450006B3F1CF061506093B10429573C4E309380
:1044600054032093530380913F03909140039C0198
:10447000442737FD4095542F80916C0490916D0432
:10448000A0916E04B0916F04820F931FA41FB51FFB
:1044900080936C0490936D04A0936E04B0936F04AA
:1044A00020916C0430916D0440916E0450916F0422
:1044B00057FF04C021503C4F4F4F5F4F9AE0559536
:1044C0004795379527959A95D1F780916C049091EF
:1044D0006D04A0916E04B0916F04821B930BA40B2A
:1044E000B50B80936C0490936D04A0936E04B0930D
:1044F0006F04F7C080915703909158032091780082
:1045000030917900820F931F909358038093570343
:1045100010925103F1C2209178003091790080917E
:10452000550390915603280F391F8FEF97E0821B98
:10453000930B909346038093450380911401DAC254
:104540008091B6049091B704209178003091790061
:10455000821B930B9093FA078093F9078091F907D8
:104560009091FA0720915F0330916003820F931FAF
:10457000909344038093430380911301BBC28091C5
:104580007800909179002091B8043091B904821B91
:10459000930B9093060880930508809105089091ED
:1045A00006082091610330916203820F931F90935C
:1045B0004203809341039DC22091590330915A03D5
:1045C0008091780090917900280F391F220F331FB6
:1045D000220F331F30935A0320935903C90137FD2B
:1045E000079603E0959587950A95E1F790934A031E
:1045F0008093490380915B0390915C03820F931F2A
:1046000097FD01969595879590935C0380935B0346
:104610002091C2043091C304821B930B9093250117
:104620008093240120914F03309150038091240105
:1046300090912501280F391F37FF02C02F5F3F4F90
:10464000359527953093500320934F03B7CD209194
:104650005703309158038091780090917900280F8A
:10466000391F220F331F220F331F3093580320931B
:104670005703C90137FD0796A3E095958795AA953D
:10468000E1F7909348038093470380915D039091F5
:104690005E03820F931F97FD0196959587959093E2
:1046A0005E0380935D032091C0043091C104821B9E
:1046B000930B909323018093220120914D0330911D
:1046C0004E038091220190912301280F391F37FF5B
:1046D00002C02F5F3F4F3595279530934E032093AF
:1046E0004D0383E007C280911104882309F180E023
:1046F0000E948C999B01AC0120503F4F4F4F5F4F60
:1047000057FF06C09B01AC0121503D4F4F4F5F4FFB
:1047100079E055954795379527957A95D1F7209368
:104720002E0330932F03409330035093310310C076
:1047300080914C0490914D04A0914E04B0914F048F
:1047400080932E0390932F03A0933003B0933103F3
:104750001092520381E0809318018091360390916A
:104760003703019690933703809336038091780046
:104770009091790090931D0180931C018091110408
:10478000882309F472C080911C0190911D017C0165
:10479000002711278091320390913303A0913403B5
:1047A000B0913503E81AF90A0A0B1B0BE092630378
:1047B000F0926403009365031093660380911501E2
:1047C000282F33274427552780911E0190911F01E0
:1047D000A0912001B0912101BC01CD010E942BA02C
:1047E00080911E0190911F01A0912001B0912101A3
:1047F000821B930BA40BB50B80931E0190931F019A
:10480000A0932001B093210180911E0190911F017E
:10481000A0912001B09121018E0D9F1DA01FB11FFD
:1048200080931E0190931F01A0932001B09321015A
:104830008091FD079091FE07A091FF07B0910008BD
:1048400020911E0130911F014091200150912101C2
:10485000821B930BA40BB50B80934C0490934D04D7
:10486000A0934E04B0934F0444C180911C019091D9
:104870001D01AA27BB27C0916303D0916403E09177
:104880006503F0916603C80FD91FEA1FFB1FC09391
:104890006303D0936403E0936503F0936603809110
:1048A00067038F5F80936703803108F422C1809192
:1048B0001E0190911F01A0912001B09121019C0146
:1048C000AD0163E0220F331F441F551F6A95D1F7D6
:1048D000281B390B4A0B5B0B2C0F3D1F4E1F5F1F14
:1048E0008091320390913303A0913403B09135034A
:1048F000281B390B4A0B5B0B57FF04C0295F3F4F46
:104900004F4F5F4F03E055954795379527950A958B
:10491000D1F720931E0130931F0140932001509343
:104920002101C091FD07D091FE07E091FF07F091B2
:10493000000880911E0190911F01A0912001B0916B
:104940002101C81BD90BEA0BFB0BC0934C04D0937D
:104950004D04E0934E04F0934F0420913B033091BB
:104960003C0340913D0350913E0357FF04C0215F3B
:104970003F4F4F4F5F4F14E055954795379527951B
:104980001A95D1F780913B0390913C03A0913D0390
:10499000B0913E03821B930BA40BB50B80933B039A
:1049A00090933C03A0933D03B0933E0380913B035F
:1049B00090913C03A0913D03B0913E038C0F9D1F4D
:1049C000AE1FBF1F80933B0390933C03A0933D0316
:1049D000B0933E0380913B0390913C03A0913D0333
:1049E000B0913E03B7FF03C00F96A11DB11DC4E0F7
:1049F000B595A79597958795CA95D1F720914C04C1
:104A000030914D04281B390B64E0213036071CF02F
:104A100020E034E006C07CEF2030370714F420E0BB
:104A20003CEF809138039091390380913803909145
:104A3000390397FF03C0909581959F4FA901F3E03B
:104A4000440F551FFA95E1F78D5B9240C4F08091B9
:104A50003803909139039C01E4E0220F331FEA955B
:104A6000E1F7281B390B240F351F37FF02C0215FE8
:104A70003F4F74E0359527957A95E1F717C08091FF
:104A80003803909139039C0165E0220F331F6A952A
:104A9000E1F7281B390B240F351F37FF02C0215EB9
:104AA0003F4F45E0359527954A95E1F73093390317
:104AB000209338038091630390916403A091650370
:104AC000B0916603B7FF03C00196A11DB11DB59556
:104AD000A795979587958093630390936403A0931C
:104AE0006503B093660388E08093670302C0109269
:104AF000520382E0809351038091510380937C00A4
:104B000080915203882319F08FEC80937A00FF91F3
:104B1000EF91DF91CF91BF91AF919F918F917F9155
:104B20006F915F914F913F912F911F910F91FF9046
:104B3000EF900F900FBE0F901F90189590E2EAE053
:104B4000F8E08FE49193815087FFFCCF0895909116
:104B50006C03903540F4E92FFF27E65FF74F808321
:104B60009F5F90936C030895A0E0B0E0EAEBF5E25C
:104B70000C9450A020916A0320FF0AC080916B031F
:104B8000882311F0815002C08091280180936B032B
:104B900021FF0CC090916B0380912801981719F4A4
:104BA00010926B0303C09F5F90936B03822F992732
:104BB00080FF04C081FF02C010926B030E949E25FB
:104BC00080916B03282F332707EA15E2C091B705C0
:104BD000D091B8058A3098F481E180936C033F93BB
:104BE0002F9384E894E09F938F931F930F93FE017C
:104BF00009952DB73EB72A5F3F4F2DBF12C080E108
:104C000080936C033F932F9389E894E09F938F9355
:104C10001F930F93FE0109954DB75EB74A5F5F4F33
:104C20004DBF20916B03822F9927AA27BB27FC0138
:104C3000439710F00C94B82EE85AFF4F07EA15E29C
:104C4000C091B705D091B8050C947DA010926C036B
:104C50008EE894E09F938F9357EAE52E55E2F52E68
:104C60001F930F93FE01099584E180936C030F90CD
:104C70000F900F900F9081E690E09F938F9384E0C8
:104C800090E09F938F9382E090E09F938F93809129
:104C900003016AE00E94D69F892F99279F938F93E3
:104CA000809103010E94D69F99279F938F938EE94D
:104CB00094E09F938F931F930F93E091B705F0912A
:104CC000B805099588E280936C038DB79EB70E9660
:104CD0008DBF8EED98E09F938F938091010199276E
:104CE0009F938F9386EB94E09F938F931F930F93E3
:104CF000E091B705F091B80509958091D105992704
:104D0000EDB7FEB73896EDBFEC01C071D07084FFEF
:104D10000BC08CE380936C0384EC94E09F938F939F
:104D20001F930F930C94AE2E90913305992351F15C
:104D30008CE380936C03892F99279F938F9381ED48
:104D400094E09F938F93FF92EF92E091B705F091DB
:104D5000B8050995DF93CF939091330581E1989F32
:104D6000C0011124875C954F9F938F93FF92EF9220
:104D7000E091B705F091B80509952DB73EB7245FCE
:104D80003F4FFFC59091D005992371F08CE380933C
:104D90006C03892F99279F938F9389ED94E09F93BC
:104DA0008F93FF92EF927FC5909172039923B9F090
:104DB0008CE380936C03892F99279F938F9380EFC7
:104DC00094E09F938F93FF92EF92E091B705F0915B
:104DD000B80509958DB79EB706968DBFD2C780914D
:104DE0003C0190913D01069730F48CE380936C0375
:104DF00086E095E0AFC79091540B9E3108F0C1C793
:104E00008CE380936C03892F99279F938F9383E181
:104E100095E017C110926C0380914C0490914D0461
:104E2000A0914E04B0914F04BC01CD0125E030E0CB
:104E300040E050E00E942BA03F932F9387E295E043
:104E40009F938F931F930F93FE01099584E18093A5
:104E50006C032DB73EB72A5F3F4F2DBF80914804AA
:104E600090914904A0914A04B0914B04BC01CD013A
:104E700025E030E040E050E00E942BA03F932F93CC
:104E800084E395E09F938F931F930F93E091B70571
:104E9000F091B805099588E280936C034DB75EB731
:104EA0004A5F5F4F4DBF80911C0190911D019F9300
:104EB0008F9381E495E09F938F931F930F93E091DD
:104EC000B705F091B80509958CE380936C038DB715
:104ED0009EB706968DBF87B599279F938F938EE4D3
:104EE00095E09F938F931F930F93E091B705F091F7
:104EF000B8050995EDB7FEB73696EDBF8091110460
:104F0000882309F43EC789E380936C038BE595E021
:104F10009F938F931F930F93E091B705F091B8057E
:104F200009958DE480936C030F900F900F900F9074
:104F30008091150199279F938F938FE595E09F931B
:104F40008F931F930F93E091B705F091B8050995E2
:104F50002DB73EB72A5F3F4F14C510926C0382E60F
:104F600095E09F938F9347EAE42E45E2F42E1F933A
:104F70000F93FE01099584E180936C030F900F90CD
:104F80000F900F908091AC049091AD04A091AE046D
:104F9000B091AF04B7FF04C081509C4FAF4FBF4FDB
:104FA0003AE0B595A795979587953A95D1F7BF9330
:104FB000AF939F938F938FE695E09F938F93FF928C
:104FC000EF92E091B705F091B805099588E28093DA
:104FD0006C034DB75EB7485F5F4F4DBF8091A4042F
:104FE0009091A504A091A604B091A704B7FF04C0B6
:104FF00081509C4FAF4FBF4F2AE0B595A79597952D
:1050000087952A95D1F7BF93AF939F938F938EE7A0
:1050100095E09F938F93FF92EF92E091B705F09107
:10502000B80509958CE380936C038DB79EB70896FD
:105030008DBF80916A0A90916B0A9F938F938DE840
:1050400095E09F938F93FF92EF927CC291E0F92EAF
:10505000C1E0D0E002ED19E09F2D969584E1989F84
:10506000C001112480936C03F801828193819F9386
:105070008F932196DF93CF932197808191819F9386
:105080008F93DF93CF938CE995E09F938F9387EA7B
:1050900095E29F938F93E091B705F091B80509953C
:1050A0002DB73EB7245F3F4F2DBF32E0F30E22965F
:1050B0000C5F1F4F48E04F1578F663C610926C03E3
:1050C00080915D08E82FFF27EE0FFF1FE053F64F9A
:1050D000808191819F938F9380915C08E82FFF27B7
:1050E000EE0FFF1FE053F64F808191819F938F93C6
:1050F0008EEA95E09F938F931F930F93FE0109957E
:1051000084E180936C038DB79EB708968DBF809124
:105110005F08E82FFF27EE0FFF1FE053F64F808157
:1051200091819F938F9380915E08E82FFF27EE0F68
:10513000FF1FE053F64F8081918181589F4F9F93CD
:105140008F938EEB95E09F938F931F930F93E09136
:10515000B705F091B805099588E280936C03EDB727
:10516000FEB73896EDBF80916108E82FFF27EE0F5C
:10517000FF1FE053F64F8081918181589F4F9F938D
:105180008F9380916008E82FFF27EE0FFF1FE053F9
:10519000F64F8081918181589F4F9F938F938EEC22
:1051A00095E09F938F931F930F93E091B705F09134
:1051B000B80509958CE380936C032DB73EB7285F43
:1051C0003F4F2DBF80916308E82FFF27EE0FFF1F91
:1051D000E053F64F8081918181589F4F9F938F9329
:1051E00080916208E82FFF27EE0FFF1FE053F64F74
:1051F0008081918181589F4F9F938F938EED95E091
:105200009F938F931F930F93E091B705F091B8058B
:1052100009954DB75EB7485F5F4F4EC310926C0360
:105220008EEE95E09F938F9387EAE82E85E2F82E25
:105230001F930F93FE01099584E180936C030F90F7
:105240000F900F900F908091C2049091C3049C0125
:1052500097FF02C0215F3F4F207F821B930B97FD7A
:105260000196959587959F938F938091C204909115
:10527000C30497FD0F96B4E095958795BA95E1F72D
:105280009F938F932091C2043091C30437FF02C0D3
:10529000295F3F4FA3E035952795AA95E1F78091C7
:1052A000490390914A03821B930B9F938F938CEF3A
:1052B00095E09F938F93FF92EF92E091B705F09165
:1052C000B805099588E280936C038DB79EB70A965E
:1052D0008DBF8091C0049091C1049C0197FF02C0D2
:1052E000215F3F4F207F821B930B97FD0196959581
:1052F00087959F938F938091C0049091C10497FDEF
:105300000F96E4E095958795EA95E1F79F938F9343
:105310002091C0043091C10437FF02C0295F3F4F84
:1053200073E0359527957A95E1F780914703909141
:105330004803821B930B9F938F938EE096E09F937D
:105340008F93FF92EF92E091B705F091B805099520
:105350008CE380936C03EDB7FEB73A96EDBF809176
:10536000BE049091BF0497FD0196959587959F93F4
:105370008F938091BE049091BF042091450330919A
:105380004603821B930B9F938F9380E296E0ECC2BF
:1053900010926C038FE296E09F938F931F930F936D
:1053A000FE01099584E180936C030F900F900F909C
:1053B0000F908091B8049091B9049F938F9380913E
:1053C0004103909142039F938F938CE396E09F93C8
:1053D0008F931F930F93E091B705F091B80509954E
:1053E00088E280936C034DB75EB7485F5F4F4DBF57
:1053F0008091B6049091B7049F938F93809143035B
:10540000909144039F938F938BE496E09F938F93A7
:105410001F930F93E091B705F091B80509958CE3C0
:1054200080936C038DB79EB708968DBF8091B204B0
:105430009091B3049F938F9380913F039091400389
:105440009F938F938AE596E09F938F931F930F937B
:10545000E091B705F091B8050995EDB7FEB738961C
:1054600079C010926C0380912601909127016AE027
:1054700070E00E94F69F9F938F93809126019091F8
:1054800027016AE070E00E94F69F7F936F9389E6A0
:1054900096E09F938F931F930F93FE01099584E1EC
:1054A00080936C032DB73EB7285F3F4F2DBF80918F
:1054B0004E0B90914F0B6AE070E00E94E29F9F9329
:1054C0008F9380914E0B90914F0B6AE070E00E9499
:1054D000E29F7F936F938DE796E09F938F931F9347
:1054E0000F93E091B705F091B805099588E2809394
:1054F0006C034DB75EB7485F5F4F4DBF8091500B57
:105500009091510B9F938F9381E996E09F938F9396
:105510001F930F93E091B705F091B80509958CE3BF
:1055200080936C038DB79EB706968DBF8091520B0A
:105530009091530B9F938F9381EA96E09F938F9363
:105540001F930F93E091B705F091B8050995EDB75A
:10555000FEB73696EDBF15C410926C0383EB96E050
:105560009F938F931F930F93FE01099588E2809379
:105570006C030F900F900F900F9080915204992719
:105580009F938F938CEB96E09F938F931F930F9332
:10559000E091B705F091B80509958CE380936C0311
:1055A0002DB73EB72A5F3F4F2DBF8091CF09992776
:1055B00001979F938F938CEC96E071C110926C03CE
:1055C0008CED96E09F938F931F930F93FE010995A7
:1055D00084E180936C030F900F900F900F90809157
:1055E00002016AE00E94D69F892F99279F938F938B
:1055F000809102010E94D69F99279F938F938CEEF2
:1056000096E09F938F931F930F93E091B705F091CE
:10561000B805099588E280936C038DB79EB708960C
:105620008DBF8091F1026AE00E94D69F892F992751
:105630009F938F938091F1020E94D69F99279F9309
:105640008F938AEF96E09F938F931F930F93E09130
:10565000B705F091B80509958CE380936C03EDB71D
:10566000FEB73896EDBF8091F2026AE00E94D69FA5
:10567000892F99279F938F938091F2020E94D69F42
:1056800099279F938F9388E097E09F938F931F9321
:105690000F936EC153E5C52E54E0D52E20E030E0C7
:1056A000E90143E0F42EC0936C03F60181916F0190
:1056B00099279F938F9389010F5F1F4F1F930F931C
:1056C00086E197E09F938F9387EA95E29F938F936C
:1056D000E091B705F091B80509952DB73EB7285F61
:1056E0003F4F2DBFFA9464969801F7FEDCCF49C373
:1056F00097E5C92E94E0D92EC0E0D0E08E0183E07A
:10570000F82E00936C03F60181916F0199279F9306
:105710008F932596DF93CF9383E297E09F938F93A8
:1057200087EA95E29F938F93E091B705F091B805D2
:1057300009952DB73EB7285F3F4F2DBFFA940C5EF9
:105740001F4F2497F7FEDDCF1CC310926C0380E33C
:1057500097E09F938F931F930F93FE01099584E128
:1057600080936C030F900F900F900F908091ED023B
:105770009091EE029F938F938EE397E09F938F9388
:105780001F930F93E091B705F091B805099588E252
:1057900080936C034DB75EB74A5F5F4F4DBF8091FA
:1057A000EF029091F0029F938F938BE497E09F9389
:1057B0008F931F930F93E091B705F091B80509956A
:1057C00089E480936C038DB79EB706968DBF88E5FC
:1057D00097E09F938F931F930F93E091B705F091FC
:1057E000B805099580916A030F900F900F900F9064
:1057F00083FFC7C21092F0021092EF0260E070E0E7
:105800008EE090E00E94EB30BCC210926C0380E608
:1058100097E09F938F931F930F93FE01099584E167
:1058200080936C030F900F900F900F9080919101D7
:10583000909192019F938F9388E697E09F938F9327
:105840001F930F93E091B705F091B805099588E291
:1058500080936C03EDB7FEB73696EDBF80916A0A70
:1058600090916B0A9F938F9386E797E09F938F9316
:105870001F930F93E091B705F091B80509958CE35C
:1058800080936C032DB73EB72A5F3F4F2DBF8091A9
:105890006A0490916B049F938F9384E897E09F93A1
:1058A0008F931F930F93E091B705F091B805099579
:1058B0004DB75EB74A5F5F4F4DBF63C210926C0336
:1058C00082E997E09F938F93B7EAEB2EB5E2FB2E28
:1058D0001F930F93FE01099584E180936C030F9051
:1058E0000F900F900F908091700199279F938F9345
:1058F0008AE997E09F938F931F930F93E091B705E9
:10590000F091B805099588E280936C038DB79EB736
:1059100006968DBF80911B0390911C0397FD039603
:1059200095958795959587959F938F9388EA97E0AE
:105930009F938F93FF92EF92E091B705F091B80596
:1059400009958CE380936C03EDB7FEB73696EDBFF7
:1059500080918B0899279F938F9380918A0899272C
:105960009F938F9386EB97E09F938F93FF92EF9295
:10597000E091B705F091B80509952DB73EB7285FBE
:105980003F4F2DBFFEC110926C0384EC97E09F93B4
:105990008F93F7EACF2EF5E2DF2E1F930F93FE01D0
:1059A00009950F900F900F900F90CFE6D9E000E08F
:1059B00010E0E2E0FE2E802F8C5E80936C038B8DD6
:1059C00099278F7790709F938F938B8999278F77E3
:1059D00090709F938F938B8599278F7790709F936B
:1059E0008F938B8199278F7790709F938F9384EDFE
:1059F00097E09F938F93DF92CF92E091B705F0915C
:105A0000B80509954DB75EB7445F5F4F4DBFFA9437
:105A10000C5E1F4FA096F7FECECFB3C110926C0361
:105A200085EE97E09F938F9377EAC72E75E2D72E86
:105A30001F930F93FE0109950F900F900F900F90F9
:105A4000CFE6D9E000E010E062E0F62E802F8C5E19
:105A500080936C038F8D992787FD90959F938F93EB
:105A60008F89992787FD90959F938F938F8599278D
:105A700087FD90959F938F938F81992787FD9095B0
:105A80009F938F9384EF97E09F938F93DF92CF92B2
:105A9000E091B705F091B80509958DB79EB70C96C2
:105AA0008DBFFA940C5E1F4FA096F7FECFCF69C151
:105AB00010926C0385E098E09F938F9357EAC52E70
:105AC00055E2D52E1F930F93FE01099587E480932D
:105AD0006C030F900F900F900F9080E198E09F93D0
:105AE0008F931F930F93E091B705F091B805099537
:105AF000FF240F900F900F900F90C0E0D0E08E0128
:105B0000802F8C5E80936C038C2F8D5F0E94B57A02
:105B10009F938F938C2F8E5F0E94B57A9F938F9364
:105B20008C2F8F5F0E94B57A9F938F938C2F0E944A
:105B3000B57A9F938F938AE198E09F938F93DF923A
:105B4000CF92E091B705F091B80509959E012C5FC1
:105B50003F4F80915A089927EDB7FEB73C96EDBFAD
:105B6000281739070CF00DC1F3940C5E1F4FE901A3
:105B7000F2E0FF1528F605C110926C038BE298E065
:105B80009F938F9347EAE42E45E2F42E1F930F93E1
:105B9000FE01099584E180936C030F900F900F90A4
:105BA0000F9080918A09881F8827881F97E0899F16
:105BB000C00111248D969F938F9380918209881F35
:105BC0008827881F96E0899FC00111248D969F9396
:105BD0008F9380917A09881F8827881F95E0899F75
:105BE000C00111248D969F938F9380917209881F15
:105BF0008827881F9927880F991F880F991F8D96CE
:105C00009F938F938AE398E09F938F931F930F93B3
:105C1000E091B705F091B805099588E280936C038F
:105C20002DB73EB7245F3F4F2DBF8091AA09881F33
:105C30008827881F9BE0899FC00111248D969F9320
:105C40008F938091A209881F8827881F9AE0899FD7
:105C5000C00111248D969F938F9380919A09881F7C
:105C60008827881F99E0899FC00111248D969F93F2
:105C70008F9380919209881F8827881F992723E096
:105C8000880F991F2A95E1F78D969F938F938EE445
:105C900098E09F938F931F930F93E091B705F09136
:105CA000B80509958CE380936C034DB75EB7445FEC
:105CB0005F4F4DBF8091B209881F8827881F9CE0E5
:105CC000899FC00111248D969F938F9382E698E05F
:105CD0009F938F931F930F93E091B705F091B805B1
:105CE00009958091BA09EDB7FEB73696EDBF87FFEB
:105CF00012C080E480936C0383E798E09F938F93B6
:105D00001F930F93E091B705F091B80509950F9097
:105D10000F900F900F908091C20987FF12C084E40A
:105D200080936C0386E798E09F938F93FF92EF92A6
:105D3000E091B705F091B80509950F900F900F907D
:105D40000F908091CA0987FF1CC088E480936C0380
:105D500089E798E09F938F93FF92EF92E091B705C8
:105D6000F091B80509950F900F900F900F9009C012
:105D700080912801281719F42150209328011092AE
:105D80006B0310926A03E8E0CDB7DEB70C946CA009
:105D9000F999FECF92BD81BDF89A80B599270895F3
:105DA000F999FECF1FBA92BD81BD60BD0FB6F894C0
:105DB000FA9AF99A0FBE08954AEA20E030E02617D1
:105DC000370740F4FC018191480F2F5F3F4F2617A2
:105DD0003707C8F3842F99270895EAEA40E050E096
:105DE0004617570778F49C01F999FECF32BD21BDC3
:105DF000F89A80B5E80F4F5F5F4F2F5F3F4F461710
:105E0000570790F38E2F9927089581E080935E08BD
:105E100082E080935D0883E080935C0884E0809357
:105E20005F0885E08093600886E08093610887E0E2
:105E30008093620888E08093630889E08093640817
:105E40008AE0809365088BE0809366088CE08093FD
:105E50006708089582E680935B088CE0E0EDF8E047
:105E600011928A95E9F78AE080937B0810929F0847
:105E70008BE1809377088EE480939C0880939D0843
:105E800080E280939E081092CC088AE6809368088E
:105E900082E78093CE0880E58093CF0886E08093E8
:105EA00082081092BF081092BC0838E03093750841
:105EB00086EE8093760880E48093780885E080936E
:105EC0006B082EE12093690890911104992399F0B1
:105ED00084E180936C0888E280936A0820936E08BE
:105EE00081E080936F08109270088FE780937108AB
:105EF0002093C20810C08FE080936C0820936A083A
:105F000090936E0830936F0884E1809370089093AB
:105F100071089093C2088FE080936D081092C708B3
:105F20008CE08093C8081092840810928508109223
:105F30008608109287081092A1081092A208109269
:105F4000A3081092A40890E89093880842E3409335
:105F5000890872E07093CD0888E180938A0886EE04
:105F600080938B0883E0809390085DE750939308BB
:105F7000509394085093950890938C0865E560932E
:105F80008D0886E480938E088CED80938F088CE3D7
:105F900080939108109292089AEA9093A5088CEC4D
:105FA0008093A7081092A9089093AA0898E290936A
:105FB000A6089093A8081092AB08409396082AE58B
:105FC000209397084093980836E03093AC0884E615
:105FD0008093AD088093AE082093AF0888E7809344
:105FE000B0089093B4088BE48093B1086093B20832
:105FF0008093B3083093B50888E08093B608409347
:10600000B7088AE28093B80885EF8093B9088CE8D6
:106010008093BA087093BB081092BD081092BE0816
:1060200081E480938008209381081092C008109228
:10603000C10886E98093C3085093990884E380934C
:106040009A081092C4081092C5081092C6081092BF
:10605000C90881E280937F0880E28093CB088FE1BA
:106060008093CA0808950E942A2F8AE080937208BC
:1060700080E18093730826E0209374089AE590935A
:10608000790888E780937A0890937C0880937D084C
:1060900020937E0880E2809383088CE380939B08A2
:1060A0008BE48093A00886E491E6A3E7B4E78093AD
:1060B000D0089093D108A093D208B093D30861E898
:1060C00070E08BE598E00E94DC2E8093DC08089558
:1060D000CF93DF930E942A2F88E08093720830E1EB
:1060E0003093730826E02093740894E6909379081F
:1060F00088E780937A0890937C0880937D082093AA
:106100007E083093830886E480939B088093A008E0
:10611000A0EDB8E085E0E9E2F1E0ED01019009923F
:106120008A95E1F761E870E0CD01855790400E94C3
:10613000DC2E8093DC08DF91CF9108950E942A2FF6
:1061400026E0209372088AE08093730884E08093AD
:10615000740894E69093790888E780937A0890937E
:106160007C0880937D0820937E0880E180938308DB
:1061700086E480939B088093A00885E491E6A3E7DA
:10618000B9E78093D0089093D108A093D208B09338
:10619000D30861E870E08BE598E00E94DC2E8093E4
:1061A000DC080895F999FECF92BD81BDF89A80B5BB
:1061B00099270895F999FECF1FBA92BD81BD60BDA0
:1061C0000FB6F894FA9AF99A0FBE089568EC7EE239
:1061D0000E94459E089540ED5EE20E947F9E0895D4
:1061E000EF92FF920F931F93CF93C82F815085306A
:1061F00008F0C3E082E8C89F8001112482EEE82EF7
:106200008FEFF82EE00EF11E61E870E0C7010E94EA
:10621000ED2E682F98012D593F4F8FB39927AC0170
:106220004270507081FDF9CF32BD21BDF89A80B522
:10623000861711F0CA0123C08FB399279C012270E1
:10624000307081FDF9CFF2BCE1BCF89A80B582369E
:1062500011F0C90114C082E8C89FC00111244E97F3
:1062600028EC3EE242E850E0BC018BE598E00E9459
:10627000209E0E9431760E94269881E090E0CF9186
:106280001F910F91FF90EF900895282F863010F006
:1062900025E003C0882309F421E020930101F99946
:1062A000FECF1FBA82E090E092BD81BD20BD0FB647
:1062B000F894FA9AF99A0FBE0895CF93C82F809157
:1062C0005B08823609F051C0C63010F0C5E003C04B
:1062D000CC2309F44AC00E94F09C8091CF0882FF31
:1062E00007C080918008843618F080E5809380088C
:1062F00061E870E08BE598E00E94DC2E8093DC087A
:1063000082E8C89FC001112420ED3EE242E850E03F
:106310006BE578E04E970E945D9E20ED3EE24CE0FA
:1063200050E06CE578E080E590E00E945D9E6CE0D6
:1063300070E08CE598E00E94DC2E282FF999FECFC2
:106340001FBA8CE590E092BD81BD20BD0FB6F894D8
:10635000FA9AF99A0FBE8C2F0E9445310E9431762D
:106360000E94269881E090E002C080E090E0CF910A
:1063700008956DE470E088EE93E00E94ED2E482FC2
:106380008FB399279C012270307081FDF9CF85E38E
:1063900094E092BD81BDF89A80B5841779F48FB3EB
:1063A00099279C012270307081FDF9CF88EE93E02F
:1063B00092BD81BDF89A80B5813011F0C901089570
:1063C00028EC3EE24EE450E068EE73E08DED98E09C
:1063D0000E94209E81E090E008958091DD08813048
:1063E000A9F46DE470E08DED98E00E94DC2E8093BE
:1063F0002A0920ED3EE24EE450E06DED78E088EEB3
:1064000093E00E945D9E81E090E0089580E090E03E
:106410000895CF93DF9381E08093DD08EDEDF8E000
:106420008FE0158616861786108A8150349687FF6E
:10643000F8CF80E48093EA088093EB081092EC0890
:106440008093ED088093EE0890EC9093EF08109203
:10645000F0088093F1088093F2081092F30890936B
:10646000F4089093F5088093F6081092F70880934B
:10647000F8089093F908AEEDB8E08CE0EFE2F1E0B7
:10648000ED01019009928A95E1F76DE470E0CD018C
:1064900001970E94DC2E80932A09DF91CF91089505
:1064A000F999FECF82E090E092BD81BDF89A80B567
:1064B000282F863078F023E0322FF999FECF1FBACB
:1064C00082E090E092BD81BD30BD0FB6F894FA9A9B
:1064D000F99A0FBE20930101822F992708951F93E7
:1064E000CF93C82F162F863010F0C5E003C0882345
:1064F00009F4C1E08C2F99278230910541F0833057
:10650000910544F4019731F40E94333005C00E9494
:10651000683002C00E949E301123E1F06CE070E010
:1065200080E590E00E94ED2E282FF999FECF8CE5B2
:1065300090E092BD81BDF89A80B5821759F428EC9D
:106540003EE24CE050E060E570E08CE598E00E94AF
:10655000209E02C00E94052F8C2F0E945D31CF919A
:106560001F910895DF92EF92FF920F931F93CF93A5
:10657000FF24DF2CEF2C81E190E00E94D23090913B
:106580000301981791F1963169F481E190E00E943E
:10659000D230853139F44C9905C06F2D81E090E0FF
:1065A0000E94DA306091030181E190E00E94DA30CC
:1065B00088E190E028E00FB6F894A89580936000F9
:1065C0000FBE209360008CE798E09F938F938EE836
:1065D00097E19F938F93E091B705F091B8050995E6
:1065E0000F900F900F900F90FFCF81E090E00E94EE
:1065F000D230823611F031E0E32E6CE070E080E5BD
:1066000090E00E94ED2EC82FF999FECF8CE590E026
:1066100092BD81BDF89A80B58C1711F421E0D22E7D
:10662000C1E001E010E0EE2029F48C2F0E94F03050
:106630008823B9F591E0F92E1F930F9384EA98E02F
:106640009F938F938EE897E19F938F93E091B70587
:10665000F091B80509952DB73EB72A5F3F4F2DBF82
:106660000130110521F00230110521F006C00E9411
:10667000333005C00E94683002C00E949E30DD2089
:1066800059F028EC3EE24CE050E060E570E08CE52B
:1066900098E00E94209E02C00E94052F8C2F0E942D
:1066A0005D31CF5F0F5F1F4FC63008F4BCCFFF20B6
:1066B00019F083E00E9445310E945032C82F0E9499
:1066C000F0308C2F99279F938F938AEC98E09F93BB
:1066D0008F930EE817E11F930F93E091B705F091A8
:1066E000B805099581E090E00E94D2302DB73EB701
:1066F0002A5F3F4F2DBF8F3F21F00E94B931882381
:1067000099F483EE98E09F938F931F930F93E091FA
:10671000B705F091B80509950E9409320E94ED3144
:106720000F900F900F900F90EE2029F062E681E01D
:1067300090E00E94DA3010925A0890E0EAEEF8E019
:10674000CFE08081349618160CF49F5FC150C7FFCC
:10675000F8CF90935A08892F99279F938F938EEDA6
:1067600098E09F938F9384E099E09F938F931F937A
:106770000F93E091B705F091B80509950E94520A70
:106780008DB79EB708968DBFCF911F910F91FF9047
:10679000EF90DF900895982F2FB7F8943998389A92
:1067A00088B1836088B98091B9008C7F8093B900EB
:1067B0008AE28093B80010927703109275031092CA
:1067C0007403992379F0EFE6F9E08BE010821182EF
:1067D0001282138214821582168217828150389693
:1067E00087FFF4CF78942FBF08951092770384E940
:1067F0008093BC0080E88093BC001092BD00109292
:10680000BA001092BB001092B9001092B80010921A
:10681000730380E00E94CB331092BB0085E8809325
:10682000BC008091710382608093710308951F9270
:106830000F920FB60F9211242F933F936F937F9374
:106840008F939F93EF93FF9380917703282F3327A4
:106850008F5F809377032330310509F40DC1243015
:1068600031055CF42130310509F454C02230310582
:106870000CF091C0232B71F0DFC22530310509F4F3
:106880005CC1253031050CF40FC12630310509F407
:1068900019C2D2C281E08093730309C0809175034D
:1068A0008C3090F4809175038F5F80937503809195
:1068B0007503E82FFF27EE0FFF1FEE0FFF1FE352B8
:1068C000F74F8585181654F7809175036CE00E9488
:1068D000D69F9093750380917D038F5F80937D0396
:1068E00090913E01981770F410927D0310927003FE
:1068F00010926F0385E08093770380917403880F73
:106900008D5A04C080917503880F8E5A8093BB0006
:1069100085E810C180917503E82FFF2723E0EE0F73
:10692000FF1F2A95E1F7E159F64F81818093BB0063
:1069300085E88093BC0080917503E82FFF2793E0E2
:10694000EE0FFF1F9A95E1F7E159F64F808180FF26
:1069500091C080917503E82FFF2783E0EE0FFF1FA2
:106960008A95E1F7E159F64F8281882329F08091D9
:106970005A08873008F476C280916F0390917003B3
:10698000892B09F06FC280916D0390916E03892B62
:1069900009F068C26FC08091750321E030E002C049
:1069A000220F331F8A95E2F780916D0390916E0359
:1069B00028233923232B79F080917503E82FFF27B3
:1069C000EE0FFF1FEE0FFF1FEE0FFF1FE159F64FF7
:1069D00080E184830DC080917503E82FFF27EE0FBF
:1069E000FF1FEE0FFF1FEE0FFF1FE159F64F14823E
:1069F00080917503E82FFF2773E0EE0FFF1F7A9554
:106A0000E1F7E159F64F8481282F332763E0220F05
:106A1000331F6A95E1F780917503E82FFF27EE0F8A
:106A2000FF1FEE0FFF1FEE0FFF1FE159F64F828190
:106A30008770822B8093BB0085E88093BC002091F7
:106A4000750381E090E002C0880F991F2A95E2F754
:106A500020916F033091700382239323892B51F08F
:106A600087E699E090937B0380937A0388E0809394
:106A70007C03F8C184E0DDC1E0917A03F0917B03EF
:106A800081918093BB0085E88093BC00F0937B03E9
:106A9000E0937A0380917C03815080937C03882368
:106AA00009F4E0C183E0C5C18091B900803351F59C
:106AB00080917803882329F4809175038F5F8093F8
:106AC000780380917503E82FFF27EE0FFF1FEE0F6D
:106AD000FF1FEE0FFF1FE159F64F838199278F7734
:106AE00090708F37910574F480917503E82FFF271C
:106AF00033E0EE0FFF1F3A95E1F7E159F64F83813E
:106B00008F5F83831092770384E98093BC008AE0CF
:106B100090E090933D0180933C01809175038F5FDD
:106B20008093750310927703809171038E7F809319
:106B3000710385EA8093BC0095C18091B9008034CF
:106B4000C1F180917403E82FFF2723E0EE0FFF1FB0
:106B50002A95E1F7E159F64F83818F7783838091FE
:106B600074038F5F80937403809174038C30A0F062
:106B70001092740310926E0310926D03809179034A
:106B80008F5F809379038C3038F010927903809175
:106B900071038D7F80937103809171038160809375
:106BA00071031092770384E98093BC001092730301
:106BB00082C080917403E82FFF2793E0EE0FFF1F40
:106BC0009A95E1F7E159F64F83818068838380913C
:106BD0007403E82FFF2783E0EE0FFF1F8A95E1F78C
:106BE000E159F64F808180FF40C080917403E82F07
:106BF000FF27EE0FFF1FEE0FFF1FEE0FFF1FE159E4
:106C0000F64F848199270097D1F0409709F04AC048
:106C100087E699E090937B0380937A0388E08093E2
:106C20007C0380917403E82FFF27EE0FFF1FEE0F08
:106C3000FF1FEE0FFF1FE159F64F148233C0809102
:106C400074039927E3E0880F991FEA95E1F78C58C0
:106C5000964F90937B0380937A0390917403809175
:106C600079039817E1F483E01BC08091740399279E
:106C700073E0880F991F7A95E1F78C58964F90939F
:106C80007B0380937A038091710381FD06C090910C
:106C9000740380917903981711F482E001C081E0B8
:106CA00080937C0380917C03813011F485E801C0DE
:106CB00085EC8093BC0080917803809372031092DE
:106CC0007803D0C0E0917A03F0917B038091BB0000
:106CD000808380917A0390917B03019690937B034C
:106CE00080937A0380917C03815080937C0382306F
:106CF00010F085EC9BC0813011F485E897C080913D
:106D0000710381FF6BC08091190480FD67C0809181
:106D10007403E82FFF2763E0EE0FFF1F6A95E1F78A
:106D2000E159F64F868199278C7F9070883F9105B5
:106D300081F480917403E82FFF27EE0FFF1FEE0F01
:106D4000FF1FEE0FFF1FE159F64F808181608083A6
:106D50000DC080917403E82FFF27EE0FFF1FEE0F89
:106D6000FF1FEE0FFF1FE159F64F10828091740351
:106D7000E82FFF2733E0EE0FFF1F3A95E1F7E159C7
:106D8000F64F8681883F71F480917403E82FFF27C6
:106D900023E0EE0FFF1F2A95E1F7E159F64F8081BE
:106DA00086601BC080917403E82FFF2793E0EE0FED
:106DB000FF1F9A95E1F7E159F64F8681893F71F4FB
:106DC00080917403E82FFF2783E0EE0FFF1F8A9561
:106DD000E1F7E159F64F80818460808380917403EC
:106DE0008F5F80937403809174038C30A0F01092B5
:106DF000740310926E0310926D03809179038F5F7C
:106E0000809379038C3038F010927903809171036C
:106E10008D7F809371031092770384E98093BC0087
:106E2000809171038160809371031AC08093BC00CC
:106E300086E08093770316C01092770384E98093ED
:106E4000BC00809171038160809371038AE090E0BF
:106E500090933D0180933C0110927503109274034E
:106E600010927303FF91EF919F918F917F916F919A
:106E70003F912F910F900FBE0F901F9018951F9369
:106E8000CF93DF93182F80915104882321F48091B0
:106E9000FE02882319F081E090E09AC01D3008F0CE
:106EA00095C01123B1F0E12FFF2743E0EE0FFF1F44
:106EB0004A95E1F7E159F64F359780813596882359
:106EC0000CF084C03897808180FD03C083E090E09F
:106ED0007FC08091670999278B709070029719F095
:106EE00084E090E075C067E070E087E699E00E947A
:106EF000DC2E90916E09891719F085E090E068C04A
:106F000080ED97E00E94631BEC018091710380FD8E
:106F100005C0CE010E946C1B8823B9F3112319F41C
:106F20008FEF90E00BC0212F33272150304081E0BC
:106F300090E002C0880F991F2A95E2F790937003A2
:106F400080936F03A1E0B0E0EFE6F9E040E050E0AD
:106F50006BE0CD01042E02C0880F991F0A94E2F75E
:106F600020916F033091700382239323892B11F0BA
:106F70001182128261504F5F5F4F389667FFE9CFF1
:106F80001092750310927703809171038E7F809326
:106F9000710385EA8093BC008091710380FD05C078
:106FA000CE010E946C1B8823B9F380916F039091EE
:106FB0007003892B29F0CE010E946C1B882311F3EA
:106FC00080916F0390917003009711F082E090E040
:106FD000DF91CF911F9108950F931F93CF93DF936C
:106FE000982F80915104882321F48091FE028823F8
:106FF00019F081E090E095C09D30A0F4992319F438
:1070000086E090E08EC0C92FDD27FE0153E0EE0F31
:10701000FF1F5A95E1F7E159F64F35978081359674
:1070200087FD03C082E090E07CC03897808180FDBE
:1070300003C083E090E075C080ED97E00E94631B81
:107040008C018091710380FD05C0C8010E946C1BFA
:107050008823B9F3219721E030E0C90102C0880FED
:10706000991FCA95E2F790936E0380936D03D9013F
:10707000EFE6F9E040E050E06BE0CD01042E02C005
:10708000880F991F0A94E2F720916D0330916E03E7
:1070900082239323892B11F01182128261504F5F5A
:1070A0005F4F389667FFE9CF10927403109267091B
:1070B00010926E0910927703809171038E7F8093F6
:1070C000710385EA8093BC008091710380FD05C047
:1070D000C8010E946C1B8823B9F380916D039091C5
:1070E0006E03892B29F0C8010E946C1B882311F3C1
:1070F0008091670999278B709070029719F084E04E
:1071000090E00FC067E070E087E699E00E94DC2E17
:1071100090916E09891719F085E090E002C080E037
:1071200090E0DF91CF911F910F910895CF93DF935E
:1071300080E021E83FEFC6E1DAE0E0EDF9E0DF01D1
:10714000853020F411961C921E9202C03183208358
:107150001982188222968F5F12963296833280F3BC
:107160008FE790E090930F0A80930E0A81E89FEFDB
:1071700090930D0A80930C0A1092110A1092100A33
:107180001092BF041092BE041092C1041092C00469
:107190001092C3041092C204DF91CF9108951F9200
:1071A0000F920FB60F9211240F931F932F933F93BB
:1071B0004F935F936F937F938F939F93AF93BF93FF
:1071C000CF93DF93EF93FF938091CE0882FDC2C0EF
:1071D000409186005091870080917F0390918003B9
:1071E000481B590B809186009091870090938003F3
:1071F00080937F03CA018D549440A0918103B09184
:107200008203835F9A4158F4809181038093CF0970
:10721000149714F01092410181E090E096C0A131E2
:10722000B1050CF0DFC1CA018B5F9040845B9140D7
:1072300008F086C080913F0190914001481B590B96
:10724000E091C408EE2351F0FF27EE0FFF1FE0533B
:10725000F64F8081918184369105ECF4FD01EA0FAF
:10726000FB1FE053F64F80819181FA01E81BF90B77
:10727000CF01F7FF03C0909581959F4F06975CF46F
:1072800080915204883C20F480915204865F01C0B2
:1072900088EC80935204FD01EA0FFB1FE053F64F88
:1072A000808191819C01220F331F280F391F240FE9
:1072B000351F37FF02C02D5F3F4FE901D595C795B8
:1072C000D595C795CA0101968C179D0714F421978F
:1072D00006C041505040C417D5070CF42196809148
:1072E0005204833CE0F08D010A0F1B1FF801E053AC
:1072F000F64F808191819E01281B390BC90163E003
:1073000070E00E94F69FCB01880F991F860F971F90
:107310000A5E154FD80111969C938E9307C0AA0F51
:10732000BB1FAA5EB54F11961C921E92E09181037D
:10733000F0918203EE0FFF1FE053F64FD183C0831D
:1073400080918103909182030196909382038093B0
:10735000810348C14091860050918700809183034A
:1073600090918403481B590B80918600909187006F
:107370009093840380938303CA018D549440609159
:107380000D04835F9A4108F072C060937E03809180
:107390007E03843008F453C09091CF0980917E031E
:1073A000981709F04CC050910E045B3008F43FC0B0
:1073B0001092410110920D0440E05F31C0F0E42FC3
:1073C000FF27EE0FFF1F9F0127533C4FDF01A05304
:1073D000B64F8D919C91D9018D939C93DF01AA5E4C
:1073E000B54F8D919C91E551FC4F91838083E42FA3
:1073F000FF27EE0FFF1F9F012053364FDF01AB57D2
:10740000BC4F8D919C91D90111969C938E93DF0175
:10741000A955BC4F8D919C91EA5EF54F9183808375
:10742000842F8F5F482F813140F280930D0480912B
:107430000E048F3F79F08F5F80930E040BC0809114
:107440000E04853620F08AE080930E0402C010926C
:107450000E04289A81E080930D04809151048823C2
:1074600009F0C0C080917E038093CF09BBC0613119
:1074700008F098C0CA018B5F9040845B914008F08F
:1074800090C080913F0190914001481B590BE62F1D
:10749000FF27EE0FFF1FEB57FC4F80819181FA0110
:1074A000E81BF90BCF0105960B9720F5E091C40876
:1074B000EE2351F0FF27EE0FFF1FE053F64F8081C0
:1074C000918184369105B4F480910E048A3120F0C4
:1074D00080915204865F05C08B3028F08091520461
:1074E0008E5F8093520480915204893C18F088EC9E
:1074F00080935204E62FFF27EE0FFF1FEB57FC4F40
:10750000808191819C01220F331F280F391F240F86
:10751000351F37FF02C02D5F3F4FE901D595C79555
:10752000D595C795CA0101968C179D0714F421972C
:1075300006C041505040C417D5070CF421968091E5
:1075400052048E3BD8F0E62FFF27EE0FFF1FDF011E
:10755000AB57BC4F8D919C919E01281B390BC901E3
:1075600063E070E00E94F69FCB01880F991F860FA1
:10757000971FE955FC4F9183808308C0E62FFF27B2
:10758000EE0FFF1FE955FC4F1182108280910D0410
:10759000E82FFF27EE0FFF1FEB57FC4FD183C0836F
:1075A00001C0289A80910D04843120F48F5F80936C
:1075B0000D0418C08431B1F4289A8EE180930D0433
:1075C00020E1C6E1DAE0A9ECB3E0E0EDF9E08D916D
:1075D0009D91918380833296198218822296215040
:1075E00027FFF5CFFF91EF91DF91CF91BF91AF9141
:1075F0009F918F917F916F915F914F913F912F91CB
:107600001F910F910F900FBE0F901F9018958091B2
:10761000DC0A9091DD0A9093B7078093B6078091BA
:10762000DE0A9091DF0A9093B9078093B8078091A2
:10763000B20A9091B30A97FD039695958795959513
:1076400087959093BB078093BA078091C20A909167
:10765000C30A97FD03969595879595958795909381
:10766000BD078093BC078091BE049091BF04209118
:10767000450330914603821B930B9093BF07809381
:10768000BE0780914C0490914D04A0914E04B0919E
:107690004F04BC01CD012AE030E040E050E00E9400
:1076A0002BA03093C1072093C0078091FB079091D6
:1076B000FC079093C3078093C2078091910190913A
:1076C00092019093C7078093C607809126019091FD
:1076D00027019093C9078093C80780915204992786
:1076E0009093CB078093CA0780916A0A90916B0AA6
:1076F0009093CD078093CC07809170099927909340
:10770000CF078093CE078091780999279093D1076E
:107710008093D0078091800999279093D307809315
:10772000D2078091880999279093D5078093D40731
:1077300080911B0390911C039093DF078093DE07D9
:1077400080913604909137049093E1078093E0078D
:1077500080914E0B90914F0B9093E3078093E2073B
:107760008091520B9091530B9093E5078093E4071F
:107770008091480490914904A0914A04B0914B042F
:10778000BC01CD012AE030E040E050E00E942BA097
:107790003093E7072093E60780916A0490916B0489
:1077A0009093ED078093EC078091540B9927909369
:1077B000F1078093F007809124059091250590931F
:1077C000F3078093F207809122059091230590930F
:1077D000F5078093F4078091D005882321F48091E8
:1077E000D105882321F08091B507816003C0809185
:1077F000B5078E7F8093B5070895EF92FF921F9390
:10780000CF93DF93182F7B0180915104882371F56A
:1078100080910301893111F4299801C0299A1150EE
:107820001F3FE9F0F0922303E0922203E7018091E9
:10783000220390912303892B11F4209781F38091E7
:1078400026038823A1F310922603809122039091AE
:107850002303892B09F421970E94069DE8CF80918C
:107860000301893111F4299A01C02998DF91CF9140
:107870001F91FF90EF900895CF93DF9310927A00BD
:107880008091490390914A039093750A8093740AFA
:1078900080914703909148039093660A8093650A0C
:1078A00080914503909146039093B80A8093B70A5C
:1078B0002091410330914203C901880F991F880F1D
:1078C000991F820F931F820F931F9093B30A809387
:1078D000B20A2091430330914403C901880F991FD4
:1078E000880F991F820F931F820F931F9093C30AD3
:1078F0008093C20A8FEC80937A00A3E5B4E0C0E6DF
:10790000D8E097E08991E82FFF27EE0FFF1FE053A3
:10791000F64F0190F081E02DE158FF4F1E161F0633
:107920001CF0E0E0F0E005C0EF3FF10514F0EFEFF0
:10793000F0E08C91282F3327E217F30714F48150DD
:1079400004C02E173F0714F48F5F8C93915011964B
:1079500097FFD8CF80919C089927AA27BB27BC0105
:10796000CD0124EC39E040E050E00E94B79FDC01FB
:10797000CB018093890190938A01A0938B01B093EE
:107980008C0180919D089927AA27BB27BC01CD01B6
:107990000E94B79FDC01CB01809385019093860103
:1079A000A0938701B0938801DF91CF910895A0E063
:1079B000B0E0EDEDFCE30C944AA0782E91E0692E46
:1079C000CC24DD2456014601E6011092D005D09268
:1079D000B904C092B804D092B704C092B604D09251
:1079E000B304C092B2041092B104D092C304C09206
:1079F000C204D092C104C092C004D092BF04C0920D
:107A0000BE0410926B0110926A0110923A030E9418
:107A10003C3C84E690E00E94851B0E943C3C8091A7
:107A2000680880FF14C080911C0190911D01875B44
:107A3000934058F480911C0190911D018E5E9240FC
:107A400020F080913A03882311F00E94C61F009114
:107A50001C0110911D0187B58B5F87BD87B580958F
:107A600088BD8FE1E82E8AE090E00E94851B80911E
:107A7000450390914603C80ED91E80914903909109
:107A80004A03A80EB91E8091470390914803880EBF
:107A9000991E8091FB079091FC07C80FD91FEA94AB
:107AA000E7FEE1CF80911C0190911D01825F934020
:107AB00080F480911C0190911D01459750F08091B8
:107AC0001C0190911D01081B190B109317010093C5
:107AD000160187B5855087BD87B5809588BD95010E
:107AE000205F3F4F36952795369527953093C304F1
:107AF0002093C204C40140969695879596958795E4
:107B00009093C1048093C00440E150E0C40ED51EA0
:107B1000B5E0D694C794BA95E1F7D092BF04C0926D
:107B2000BE04C40FD51FA5E0D695C795AA95E1F769
:107B3000D093B304C093B2049093BD048093BC046B
:107B40003093BB042093BA0452E07516C9F58091B6
:107B5000B20A9091B30A97FF03C0909581959F4F09
:107B60006CE070E00E94F69F9B017093B9046093F3
:107B7000B8048091C20A9091C30A97FF03C0909500
:107B800081959F4F6CE070E00E94F69F7093B70460
:107B90006093B604B90184E090E00E94EB306091FC
:107BA000B6047091B70486E090E00E94EB306091DB
:107BB000B2047091B30488E090E00E94EB304FC0B3
:107BC00084E090E00E94E6309093B9048093B8047A
:107BD00086E090E00E94E6309C019093B704809389
:107BE000B6048091B8049091B9048150984018F47B
:107BF00021503840A0F185E299E09F938F938EE861
:107C000097E19F938F93E091B705F091B80509959F
:107C10008091B20A9091B30A97FF03C09095819525
:107C20009F4F6CE070E00E94F69F7093B9046093E0
:107C3000B8048091C20A9091C30A97FF03C090953F
:107C400081959F4F6CE070E00E94F69F7093B7049F
:107C50006093B60466240F900F900F900F9012BCA3
:107C600011BC1092750A1092740A1092660A109252
:107C7000650A1092B80A1092B70A88EC90E00E9448
:107C8000851B80914103909142039C01220F331F79
:107C9000220F331F280F391F280F391F3093B30AC3
:107CA0002093B20A80914303909144038C01000F0A
:107CB000111F000F111F080F191F080F191F109314
:107CC000C30A0093C20A80917708C82EDD24EE24EF
:107CD000FF24442737FD4095542FC701B6010E9469
:107CE000B79F4B015C016093AC047093AD0480932B
:107CF000AE049093AF049801442737FD4095542F6C
:107D0000C701B6010E94B79FDC01CB018093A40498
:107D10009093A504A093A604B093A70480928C042A
:107D200090928D04A0928E04B0928F04809384046C
:107D300090938504A0938604B093870410927C04EA
:107D400010927D0410927E0410927F0400919101A4
:107D50001091920110936B0400936A0484E690E002
:107D600090938E0180938D0182E390E090932303A2
:107D70008093220380919C089927AA27BB27BC01E6
:107D8000CD0124EC39E040E050E00E94B79FDC01D7
:107D9000CB018856954CAF4FBF4F8093890190938C
:107DA0008A01A0938B01B0938C0180919D08992743
:107DB000AA27BB27BC01CD010E94B79FDC01CB01E4
:107DC0008856954CAF4FBF4F8093850190938601A5
:107DD000A0938701B0938801109248011092470147
:107DE000C801AA2797FDA095BA2F20914301309191
:107DF00044014091450150914601BC01CD010E94D2
:107E0000B79FDC01CB018093BE0A9093BF0AA09379
:107E1000C00AB093C10A10926704109266040E94CF
:107E20003176772029F080911904846080931904B9
:107E30008FEF80933E0B10923F0B80E28093400BBC
:107E4000C3E5D4E0A0E6B8E077E0E72E8D91E82F17
:107E5000FF27EE0FFF1FE053F64F8081918181587D
:107E60008993EA94E7FEF2CF84E6809352048091EE
:107E70002003882311F0579A17C08091CD089927C5
:107E800080FF05C082FF03C080EE9EE202C080E05A
:107E900091E190930A018093090181E0809311019F
:107EA0000E94261C0E94261C8091AC049091AD0477
:107EB000A091AE04B091AF04E0904301F090440172
:107EC0000091450110914601BC01CD01A801970127
:107ED0000E942BA059016A018091A4049091A504ED
:107EE000A091A604B091A704BC01CD01A8019701FF
:107EF0000E942BA0B901C5010E9479908C010E94BB
:107F00008A7A9C0190937F0A80937E0A8091B204C2
:107F10009091B304AA2797FDA095BA2F6DE0880F22
:107F2000991FAA1FBB1F6A95D1F78050904FAF438E
:107F3000B040442737FD4095542FBC01CD010E942D
:107F40002BA0C90180509E4F9093B3048093B2043C
:107F5000053111050CF06624772081F08091110421
:107F6000882361F0C9018C5890408234910530F02B
:107F70008091D00580628093D00566248091C204F0
:107F80009091C30480569940815C9B4228F0809177
:107F9000D00581608093D0058091C0049091C10488
:107FA00080569940815C9B4228F08091D005826088
:107FB0008093D0058091BE049091BF048C52914073
:107FC0008957954028F08091D00584608093D00532
:107FD0008091B8049091B9048C529140835C914097
:107FE00028F08091D00588608093D0058091B604F8
:107FF0009091B7048C529140835C914028F080911D
:10800000D00580618093D0058091B2049091B30433
:10801000805092408355914028F08091D005806235
:108020008093D0058091D0058111662486E48093E9
:1080300080010E94269882E00E948C9980911E0106
:1080400090911F01A0912001B09121018093FD0723
:108050009093FE07A093FF07B09300081092390396
:108060001092380310923B0310923C0310923D0390
:1080700010923E0310926C0410926D0410926E04E4
:1080800010926F041092EF071092EE070E948E1F5D
:10809000862D9927EEE0CDB7DEB70C9466A0A3E15C
:1080A000B0E0E5E5F0E40C9446A08091BE04909128
:1080B000BF042091450330914603821B930B90939C
:1080C000B80A8093B70A80914F039091500397FDAF
:1080D00007969C0153E0359527955A95E1F7309323
:1080E000750A2093740A80914D0390914E0397FD79
:1080F000079643E0959587954A95E1F79093660A30
:108100008093650A3093810A2093800A9093780ABD
:108110008093770A8091B20A9091B30AAC01440F20
:10812000551F480F591F2091410330914203C90147
:10813000880F991F880F991F820F931F820F931F1B
:10814000480F591F57FF02C04D5F5F4F5595479528
:10815000559547955093B30A4093B20A8091C20A4D
:108160009091C30AAC01440F551F480F591F20912D
:10817000430330914403C901880F991F880F991F49
:10818000820F931F820F931F480F591F57FF02C082
:108190004D5F5F4F55954795559547955093C30A49
:1081A0004093C20A2091410330914203C901880FD4
:1081B000991F880F991F820F931F820F931F9C0195
:1081C000442737FD4095542F80919C0490919D0445
:1081D000A0919E04B0919F04820F931FA41FB51F0E
:1081E00080939C0490939D04A0939E04B0939F045D
:1081F0002091430330914403C901880F991F880FD0
:10820000991F820F931F820F931F9C01442737FDF4
:108210004095542F8091980490919904A0919A04CC
:10822000B0919B04820F931FA41FB51F80939804E5
:1082300090939904A0939A04B0939B0480918A0A26
:1082400090918B0A2091410330914203820F931F3A
:1082500090938B0A80938A0A8091BA0A9091BB0A04
:108260002091430330914403820F931F9093BB0AE4
:108270008093BA0A8091B4049091B50401969093CA
:10828000B5048093B4048091FB079091FC07209182
:10829000B2043091B304821B930B9C01442737FD39
:1082A0004095542F8091940490919504A091960448
:1082B000B0919704820F931FA41FB51F809394045D
:1082C00090939504A0939604B09397048FEC8093B9
:1082D0007A00109218012091840430918504409115
:1082E00086045091870429873A874B875C872954F5
:1082F0003B46414050402CF028E43BE641E050E052
:108300000DC089859A85AB85BC85885B9449AE4F45
:10831000BF4F4CF428EB34E94EEF5FEF2D833E83E3
:108320004F83588708C089859A85AB85BC858D8326
:108330009E83AF83B88720918C0430918D04409147
:108340008E0450918F042D873E874F87588B295478
:108350003B46414050402CF028E43BE641E050E0F1
:108360000DC08D859E85AF85B889885B9449AE4FD9
:10837000BF4F4CF428EB34E94EEF5FEF29833A838B
:108380004B835C8308C08D859E85AF85B8898983C2
:108390009A83AB83BC83A091B70AB091B80ABB8B18
:1083A000AA8BFD01CF01AA2797FDA095BA2FA09017
:1083B0007C04B0907D04C0907E04D0907F04A80E11
:1083C000B91ECA1EDB1EA0927C04B0927D04C0922E
:1083D0007E04D0927F04E090BE0AF090BF0A009124
:1083E000C00A1091C10AE80EF91E0A1F1B1FE09275
:1083F000BE0AF092BF0A0093C00A1093C10AF0911E
:108400003504F98BFF2309F098C180913404882347
:1084100009F093C18091AE0A86FF8FC18091650AF1
:108420009091660AAA2797FDA095BA2FBC01CD01AD
:1084300029813A814B815C810E94B79F9B01AC01ED
:1084400097FF04C02150384F4F4F5F4F6BE0559559
:108450004795379527956A95D1F780916A01682EDF
:10846000772488249924CA01B901A40193010E94A8
:10847000B79FDC01CB018093CE049093CF04A093EF
:10848000D004B093D104B7FF04C08150904FAF4FD8
:10849000BF4F1C012D013CE055944794379427941D
:1084A0003A95D1F72092CE043092CF044092D00476
:1084B0005092D1048091740A9091750AAA2797FD71
:1084C000A095BA2FBC01CD012D813E814F815885E9
:1084D0000E94B79F97FF04C06150784F8F4F9F4F06
:1084E0002BE095958795779567952A95D1F7A40107
:1084F00093010E94B79FDC01CB018093D20490933B
:10850000D304A093D404B093D504B7FF04C0815022
:10851000904FAF4FBF4F9C01AD018CE055954795F3
:10852000379527958A95D1F72093D2043093D304B9
:108530004093D4045093D5048091CE049091CF04FD
:1085400090935D0A80935C0A8091D2049091D30449
:108550009093610A8093600A2219330944095509EE
:108560002093D2043093D3044093D4045093D50481
:10857000E20EF31E041F151FE092BE0AF092BF0A1E
:108580000093C00A1093C10A809169018823B1F455
:1085900057FF04C02F5F3F4F4F4F5F4F5595479593
:1085A00037952795A21AB30AC40AD50AA0927C046B
:1085B000B0927D04C0927E04D0927F042A893B89C8
:1085C00079010027F7FC0095102F8091D20490913B
:1085D000D304A091D404B091D504E80EF91E0A1F6B
:1085E0001B1FC801B70129813A814B815C810E9420
:1085F000B79F9B01AC0197FF04C02150384F4F4FEC
:108600005F4FBBE05595479537952795BA95D1F7BC
:1086100080916B01A82EBB24CC24DD24CA01B901B2
:10862000A60195010E94B79FDC01CB018093C6048F
:108630009093C704A093C804B093C904B7FF04C0C3
:108640008150904FAF4FBF4F3C014D01ACE095942E
:10865000879477946794AA95D1F76092C604709234
:10866000C7048092C8049092C904C801B7012D8143
:108670003E814F8158850E94B79F97FF04C061508B
:10868000784F8F4F9F4FFBE095958795779567952E
:10869000FA95D1F7A60195010E94B79FDC01CB01A5
:1086A0008093CA049093CB04A093CC04B093CD04E0
:1086B000B7FF04C08150904FAF4FBF4FAC01BD0119
:1086C000ECE07595679557954795EA95D1F74093F6
:1086D000CA045093CB046093CC047093CD042A89D0
:1086E0003B8937FF03C0309521953F4F2134310539
:1086F000E4F1D401C30197FE07C0B095A095909511
:1087000081959F4FAF4FBF4F81389105A105B105AE
:1087100084F4DB01CA0177FF07C0B095A09590955E
:1087200081959F4FAF4FBF4F81389105A105B1058E
:10873000E4F081E08093680418C01092610A1092FE
:10874000600A10925D0A10925C0A1092CA0410929C
:10875000CB041092CC041092CD041092C604109257
:10876000C7041092C8041092C9048091CA04909161
:10877000CB04A091CC04B091CD04BC01CD0124E682
:1087800030E040E050E00E942BA0E090C604F09062
:10879000C704E21AF30AF092730AE092720A809117
:1087A000C6049091C704A091C804B091C904BC014B
:1087B000CD0124E630E040E050E00E942BA0DA0139
:1087C000C9012091CA043091CB048C01021B130B08
:1087D0001093680A0093670A8091430190914401C5
:1087E000A0914501B0914601BC01CD0128E631E0E0
:1087F00040E050E00E94B79F2091BE0A3091BF0A2E
:108800004091C00A5091C10A2617370748075907F7
:1088100064F0261B370B480B590B2093BE0A30938C
:10882000BF0A4093C00A5093C10A2091BE0A3091FA
:10883000BF0A4091C00A5091C10A57FF0CC0260FD1
:10884000371F481F591F2093BE0A3093BF0A409319
:10885000C00A5093C10A6091650A7091660A6E0D54
:108860007F1D9B01442737FD4095542F8091800444
:1088700090918104A0918204B0918304820F931F90
:10888000A41FB51F8093800490938104A093820459
:10889000B093830480913A0490913B04681B790B58
:1088A000CB01AA2797FDA095BA2F29853A854B853C
:1088B0005C85820F931FA41FB51F8093840490933F
:1088C0008504A0938604B0938704C0908501D0905E
:1088D0008601E0908701F0908801C816D906EA0663
:1088E000FB06C4F488EA91E6A0E0B0E08C199D098B
:1088F000AE09BF098093840490938504A0938604F5
:10890000B09387048093800490938104A0938204A1
:10891000B093830422273327A9012C193D094E095E
:108920005F098091840490918504A0918604B091A0
:10893000870482179307A407B507B4F4D701C601CB
:10894000885A9146A040B040809384049093850457
:10895000A0938604B093870480938004909381044D
:10896000A0938204B09383046091740A7091750A95
:10897000600F711F9B01442737FD4095542F809154
:10898000880490918904A0918A04B0918B04820F8D
:10899000931FA41FB51F8093880490938904A0930C
:1089A0008A04B0938B048091380490913904681B39
:1089B000790BCB01AA2797FDA095BA2F2D853E856F
:1089C0004F855889820F931FA41FB51F80938C0475
:1089D00090938D04A0938E04B0938F04E09089014E
:1089E000F0908A0100918B0110918C01E816F90634
:1089F0000A071B07C4F488EA91E6A0E0B0E08E19EC
:108A00009F09A00BB10B80938C0490938D04A093CD
:108A10008E04B0938F048093880490938904A0936C
:108A20008A04B0938B0422273327A9012E193F090A
:108A3000400B510B80918C0490918D04A0918E0479
:108A4000B0918F0482179307A407B507B4F4D80137
:108A5000C701885A9146A040B04080938C049093FF
:108A60008D04A0938E04B0938F0480938804909318
:108A70008904A0938A04B0938B0480917C04909124
:108A80007D04A0917E04B0917F0480939004909324
:108A90009104A0939204B093930480918C049091DC
:108AA0008D04A0918E04B0918F048093AC049093B8
:108AB000AD04A093AE04B093AF0480918404909170
:108AC0008504A0918604B09187048093A4049093B8
:108AD000A504A093A604B093A70480918804909164
:108AE0008904A0918A04B0918B048093A804909388
:108AF000A904A093AA04B093AB0480918004909140
:108B00008104A0918204B09183048093A004909387
:108B1000A104A093A204B093A30480912401909196
:108B2000250197FD079633E0959587953A95E1F7EE
:108B30009093750A8093740A809122019091230189
:108B400097FD079623E0959587952A95E1F79093F1
:108B5000660A8093650A8091490390914A030F97B2
:108B600034F488E19CEF9093750A8093740A8091A5
:108B7000490390914A03079734F480E398EF909368
:108B8000750A8093740A8091490390914A03815D2C
:108B9000974034F088EE93E09093750A8093740ABE
:108BA0008091490390914A03805E974034F080EDB4
:108BB00097E09093750A8093740A8091470390918F
:108BC00048030F9734F488E19CEF9093660A8093F2
:108BD000650A8091470390914803079734F480E336
:108BE00098EF9093660A8093650A8091470390916D
:108BF0004803815D974034F088EE93E09093660AD5
:108C00008093650A8091470390914803805E974066
:108C100034F080ED97E09093660A8093650A609146
:108C20007801662309F4AEC04091240150912501DA
:108C30008091D6049091D704481B590B5093DD04C2
:108C40004093DC042091240130912501280F391F25
:108C500037FF02C02F5F3F4F359527953093D704DC
:108C60002093D604413851051CF080E890E005C0FF
:108C700040585F4F34F480E89FEF9093DD04809379
:108C8000DC0440912201509123018091D8049091FD
:108C9000D904481B590B5093DB044093DA0420910C
:108CA000220130912301280F391F37FF02C02F5FA7
:108CB0003F4F359527953093D9042093D8044138F8
:108CC00051051CF080E890E005C040585F4F34F437
:108CD00080E89FEF9093DB048093DA04462F5527BA
:108CE0008091DC049091DD04849FB001859F700D1C
:108CF000949F700D11249B0177FF02C0215F3F4FAD
:108D0000B4E035952795BA95E1F78091740A909172
:108D1000750A820F931F9093750A8093740A80914D
:108D2000DA049091DB04849F9001859F300D949F1D
:108D3000300D1124A90137FF02C0215F3F4FA4E08D
:108D400035952795AA95E1F78091650A9091660A75
:108D5000820F931F9093660A8093650A8091240185
:108D600090912501860F971F9093250180932401F0
:108D70008091220190912301840F951F90932301EC
:108D8000809322010091770A1091780A80915C0A01
:108D900090915D0A101611065CF59C0197FF04C0C6
:108DA00022273327281B390BC901AA2797FDA09535
:108DB000BA2F20916901332744275527BC01CD01E3
:108DC0000E94B79F9B01AC0197FF04C0215C3F4FFD
:108DD0004F4F5F4FF6E05595479537952795FA9594
:108DE000D1F78091720A9091730A820F931F27C066
:108DF00097FF03C0909581959F4FAA2797FDA09557
:108E0000BA2F20916901332744275527BC01CD0192
:108E10000E94B79F9B01AC0197FF04C0215C3F4FAC
:108E20004F4F5F4FE6E05595479537952795EA9563
:108E3000D1F78091720A9091730A821B930B9093E1
:108E4000730A8093720AE090800AF090810A809100
:108E5000600A9091610A1E141F045CF59C0197FF43
:108E600004C022273327281B390BC901AA2797FDE5
:108E7000A095BA2F20916901332744275527BC01BB
:108E8000CD010E94B79F9B01AC0197FF04C0215CFC
:108E90003F4F4F4F5F4F76E0559547953795279554
:108EA0007A95D1F78091670A9091680A820F931F93
:108EB00027C097FF03C0909581959F4FAA2797FDE4
:108EC000A095BA2F20916901332744275527BC016B
:108ED000CD010E94B79F9B01AC0197FF04C0215CAC
:108EE0003F4F4F4F5F4F66E0559547953795279514
:108EF0006A95D1F78091670A9091680A821B930B5B
:108F00009093680A8093670A8091AE0A87FF44C0F5
:108F10003989332309F040C0809134048823E1F576
:108F200041E0E41641E0F4064CF08091740A90911F
:108F3000750A8E0D9F1D805091400DC050E0E516C2
:108F40005FEFF50664F48091740A9091750A8E0DB6
:108F50009F1D80509F4F9093750A8093740A81E003
:108F6000013018074CF08091650A9091660A800FD5
:108F7000911F805091400CC09FEF0030190764F49E
:108F80008091650A9091660A800F911F80509F4FD3
:108F90009093660A8093650AE2E1CD5E0C9462A02C
:108FA00080915104882329F5809119048C7F809346
:108FB0001904809118048F7D80931804A5EDB5E005
:108FC000EFE6F9E09BE08091FE02882309F48C93A0
:108FD0008D91818312829150389697FFF4CF8091C2
:108FE000FE02882359F08091FE0281508093FE0298
:108FF00005C08091190481608093190480917303E6
:10900000882319F010927303089580937703809159
:1090100071038E7F8093710385EA8093BC0008956D
:10902000882319F480E090E00895E82FFF27EE0FE1
:10903000FF1FE053F64F8081918181589F4F8F3FF2
:10904000910521F01CF08FEF90E004C097FF02C063
:1090500080E090E099270895CF93DF93A3E5B4E0F3
:10906000C0E6D8E057E08991E82FFF27EE0FFF1FF9
:10907000E053F64F0190F081E02DE158FF4FEF3FB4
:10908000F10521F01CF0EFEFF0E004C0F7FF02C0A3
:10909000E0E0F0E0893111F4EC931BC04C91242FF7
:1090A0003327E217F307A9F0CF01821B930B97FD3B
:1090B00003969595879595958795242F280F2C9342
:1090C000822F9927E817F90714F4215001C02F5F68
:1090D0002C935150119657FFC6CF80916A08883F54
:1090E00038F0EFEFF0E0E81BF109ED5AFB4F80811B
:1090F00080937D0180917D01882329F0843618F0CA
:1091000084E680937D0180916C08883F38F0EFEF12
:10911000F0E0E81BF109ED5AFB4F808180937C0160
:1091200080917C01882329F0843618F084E68093AE
:109130007C0180917908883F38F0EFEFF0E0E81B80
:10914000F109ED5AFB4F808180937701809177017F
:109150008B3010F48AE002C08F3F11F480937701C6
:109160008091A608883F38F0EFEFF0E0E81BF109A6
:10917000ED5AFB4F808180938C0A80918C0A863057
:1091800010F485E002C08F3F11F480938C0A809127
:10919000A808883F38F0EFEFF0E0E81BF109ED5A3E
:1091A000FB4F80818093B50A8091B50A863010F418
:1091B00085E002C08F3F11F48093B50A8091930837
:1091C000873F19F4429905C006C0863F31F4439B9E
:1091D00002C08CE815C086E413C0883F38F0EFEF7A
:1091E000F0E0E81BF109ED5AFB4F80818093890A7A
:1091F0008091890A893110F488E102C08F3F11F40F
:109200008093890A80919408873F19F4429905C098
:1092100006C0863F31F4439B02C08CE815C086E44B
:1092200013C0883F38F0EFEFF0E0E81BF109ED5A8A
:10923000FB4F80818093620A8091620A893110F429
:1092400088E102C08F3F11F48093620A80919508F3
:10925000883F38F0EFEFF0E0E81BF109ED5AFB4FE3
:1092600080818093920A8091920A893110F488E17A
:1092700002C08F3F11F48093920A80916B080E9484
:10928000104880932F0480916E08883F38F0EFEFEC
:10929000F0E0E81BF109ED5AFB4F808180937B01E0
:1092A00080917008883F38F0EFEFF0E0E81BF1099B
:1092B000ED5AFB4F80818093790180917808883F37
:1092C00038F0EFEFF0E0E81BF109ED5AFB4F808139
:1092D00080937A0180917A08883F38F0EFEFF0E0D0
:1092E000E81BF109ED5AFB4F808180937601809154
:1092F0007B08883F38F0EFEFF0E0E81BF109ED5A0A
:10930000FB4F80818093780180917C08883F38F002
:10931000EFEFF0E0E81BF109ED5AFB4F80818093FD
:10932000750180917D08883F38F0EFEFF0E0E81B91
:10933000F109ED5AFB4F808180937401809183087D
:10934000883F38F0EFEFF0E0E81BF109ED5AFB4FF2
:1093500080818093720180918408883F38F0EFEF1C
:10936000F0E0E81BF109ED5AFB4F808180932E0459
:1093700080918508883F38F0EFEFF0E0E81BF109B5
:10938000ED5AFB4F808180932D0480918608883FA1
:1093900038F0EFEFF0E0E81BF109ED5AFB4F808168
:1093A00080932C0480918708883F38F0EFEFF0E03D
:1093B000E81BF109ED5AFB4F808180932B048091CB
:1093C000A108883F38F0EFEFF0E0E81BF109ED5A13
:1093D000FB4F808180932A048091A208883F38F057
:1093E000EFEFF0E0E81BF109ED5AFB4F808180932D
:1093F00029048091A308883F38F0EFEFF0E0E81BE4
:10940000F109ED5AFB4F8081809328048091A408D4
:10941000883F38F0EFEFF0E0E81BF109ED5AFB4F21
:1094200080818093270480918808883F38F0EFEF8F
:10943000F0E0E81BF109ED5AFB4F80818093700149
:1094400080918C08883F38F0EFEFF0E0E81BF109DD
:10945000ED5AFB4F808180936F0180918908883F8E
:1094600038F0EFEFF0E0E81BF109ED5AFB4F808197
:1094700080936E0180918D08883F38F0EFEFF0E027
:10948000E81BF109ED5AFB4F808180936D018091BB
:109490009608883F38F0EFEFF0E0E81BF109ED5A4D
:1094A000FB4F808180936C0180919908883F38F050
:1094B000EFEFF0E0E81BF109ED5AFB4F808180935C
:1094C0006B0180919A08883F38F0EFEFF0E0E81BDD
:1094D000F109ED5AFB4F808180936A0180919B08CE
:1094E000883F38F0EFEFF0E0E81BF109ED5AFB4F51
:1094F0008081809369018091C308883F38F0EFEF45
:10950000F0E0E81BF109ED5AFB4F80818093710A6E
:1095100090912E05992321F08091710A981720F0DF
:109520008091710A882311F49093710A80916808E0
:109530008093AE0A8091CE088093910A8091A00812
:10954000883F38F0EFEFF0E0E81BF109ED5AFB4FF0
:109550008081809368018091BC08883F38F0EFEFEC
:10956000F0E0E81BF109ED5AFB4F80818093C50ABA
:1095700080917201282F33272F5F3F4F8CE398E2B1
:10958000B9010E94F69F70937F0160937E018091E4
:1095900076088093B60A809175088093790AE091E5
:1095A000BE08EE2309F449C081E080932604FF271A
:1095B000EE0FFF1FE053F64F80819181805C9F4F3B
:1095C00014F41092260480918001209126048217C1
:1095D00021F18330F8F43091AB01222351F08CED6E
:1095E00095E09093230380932203332369F48EE262
:1095F00009C088EC90E090932303809322033323E7
:1096000019F487E18093AB0185E080933C042093BB
:10961000800103C08150809380018091050B90915F
:10962000060B97FF0FC080912604882359F0809184
:10963000D00580688093D00505C0E09326048AE0B9
:10964000809380018091050B9091060B97FF1DC0C0
:10965000809151048823C9F0809126048823A9F0C1
:1096600080910B0190910C018F5F9F4F71F488E9FD
:109670009AE3909323038093220380E094EA9093EB
:109680000C0180930B0110922604809126048823FC
:1096900021F080911804816003C0809118048E7FAE
:1096A00080931804DF91CF910895809171088823E9
:1096B00001F5609136047091370477FF02C06D5F49
:1096C0007F4F7595679575956795409126015091E7
:1096D000270180910201282F3327649FC001659FD5
:1096E000900D749F900D1124B9010E94E29FCB014F
:1096F00001C0992790938401809383018091830115
:10970000909184018734910538F486E490E0909339
:1097100084018093830108958F3A910530F08FEA98
:1097200090E090938401809383010895A8E1B0E0D4
:10973000ECE9FBE40C9446A00E944F408091190490
:10974000992784719070892B91F58091CF0882FFC1
:1097500027C080913604909137040097F1F002E021
:1097600088359007D4F49C0197FF02C02D5F3F4FCE
:109770003595279535952795809180089927289FBD
:10978000A001299F500D389F500D1124CA0164E695
:1097900070E00E94F69FCB0106C08DE290E003C00E
:1097A0008091800899279093170480931604209144
:1097B00014043091150455E72033350759F41092FD
:1097C0005D0410925C048091790A992790931704A4
:1097D0008093160460915C0470915D047A836983C0
:1097E0008091790A99270A966817790714F49A8361
:1097F000898380915204843608F062C080911804F5
:1098000082FD5EC08091F2049091F304009731F0E4
:1098100001979093F3048093F2040BC010925104CB
:1098200090931B0480931A04809119048D7E809379
:109830001904289A80911A0490911B04895E934020
:10984000E0F18091540B8536C0F18091160490911F
:1098500017049A8389838091190480618093190485
:1098600080915C08A82FBB27AA0FBB1FFD01EA5EF1
:10987000F54F1182108280915D08282F3327220F27
:10988000331FC9018A5E954FFC0111821082A053DB
:10989000B64F11961C921E922053364FD901119645
:1098A0001C921E9280915F08E82FFF27EE0FFF1F8A
:1098B000E053F64F11821082B4C510925104B1C525
:1098C000809152048D3808F482C59091C70899237D
:1098D00009F445C08091C808882309F440C0E92FE5
:1098E000FF27EE0FFF1FE053F64F80819181C39752
:1098F000BCF080919501823361F48091180485FF5A
:1099000008C08091180480648093180480E38093D9
:10991000AB01809118048F778093180486E917C0F3
:10992000808191818E5C9F4FACF480919501863946
:1099300041F4809118048068809318048FE280932A
:10994000AB01809118048F7B8093180482E380938D
:10995000950105C0809118048F738093180480913D
:1099600019048F7E809319049091810882E3989F57
:10997000C00111249093F3048093F204E981FA81E9
:10998000B9978CF080915104882369F080911A0472
:1099900090911B04FFEF8F3F9F0729F00196909352
:1099A0001B0480931A0440911A0450911B044F3FEA
:1099B000510509F048F51092740410927504109244
:1099C0007604109277041092700410927104109231
:1099D0007204109273041092DE041092DF0410924D
:1099E000E0041092E10410927C0410927D04109225
:1099F0007E0410927F048091180480628093180482
:109A000084E68093950135C180911904826080932A
:109A100019048091180485FF98C080912F0599271B
:109A20009C012470307082FD04C08091180486FF70
:109A30002AC0809142018D3331F580911104882331
:109A400011F180E58093410484EF91E0A0E0B0E063
:109A50008093420490934304A0934404B09345043C
:109A60008093480490934904A0934A04B0934B0414
:109A700088EE93E09093940180939301232B19F047
:109A80008DE08093AB0180912E0390912F03A091E4
:109A90003003B091310387399105A105B1058CF4EC
:109AA00080914C0490914D04A0914E04B0914F04CC
:109AB000825A9E4FAF4FBF4F24F08091AE0A80FD77
:109AC00021C088EE93E0909394018093930180915C
:109AD000180486FF0FC0109241048CE291E0A0E0D0
:109AE000B0E08093480490934904A0934A04B09353
:109AF0004B0403C080E38093AB01809118048F7105
:109B000080931804109274041092750410927604D5
:109B100010927704109270041092710410927204E3
:109B20001092730410927C0410927D0410927E04B3
:109B300010927F04495E534008F49BC088EE93E086
:109B400090931B0480931A0494C08091180487FF9B
:109B50001AC080914201863711F08D33A1F48091B3
:109B60001104882381F08091C8088093410480EE1D
:109B700091EBAFEFBFEF8093420490934304A09327
:109B80004404B0934504209193013091940143E043
:109B9000283E340708F048C02F5F3F4F30939401B0
:109BA000209393011092740410927504109276041D
:109BB0001092770410927004109271041092720443
:109BC0001092730410927C0410927D0410927E0413
:109BD00010927F0480912E0390912F03A091300367
:109BE000B09131038C529140A040B0408093480422
:109BF00090934904A0934A04B0934B04285E3340E9
:109C0000C1F58091180487FF34C0809142018B32E6
:109C100081F1809118048F77809318048091180443
:109C200080628093180425C080911104882309F173
:109C300080914201863711F08D32D9F480914C0425
:109C400090914D04A0914E04B0914F04885E9340D2
:109C5000A040B04074F48091FB079091FC078D5AAE
:109C600093403CF010929401109293018EE0809307
:109C7000AB0180915E08E82FFF27EE0FFF1FE05336
:109C8000F64F80819181813591050CF454C120916A
:109C90005104222309F04FC180915F08E82FFF276C
:109CA000EE0FFF1FE053F64F808191818C349105B8
:109CB0000CF411C18091F4048F5F8093F404893C0B
:109CC00008F439C12093F40410921B0410921A0472
:109CD00030915C08E32FFF27EE0FFF1FE053F64F94
:109CE0008081918187349105B4F480915D08E82FDB
:109CF000FF27EE0FFF1FE053F64F80819181019007
:109D0000F081E02DF7FF03C0F095E195FF4FE734B8
:109D1000F1050CF478C041E020915D08A22FBB272B
:109D2000AA0FBB1FA053B64F8D919C9111978734FA
:109D3000910544F0E32FFF27EE0FFF1FE053F64F8E
:109D4000808191818D919C918734910574F08091EF
:109D50005C08E82FFF27EE0FFF1FE053F64F8081CE
:109D60009181873491050CF042E0E22FFF27EE0F3E
:109D7000FF1FE053F64F808191818634910574F482
:109D800080915C08E82FFF27EE0FFF1FE053F64F8E
:109D900080819181873491050CF043E0E22FFF2709
:109DA000EE0FFF1FE053F64F808191818A5B9F4F3A
:109DB00074F480915C08E82FFF27EE0FFF1FE0533B
:109DC000F64F80819181873491050CF044E0E22FB9
:109DD000FF27EE0FFF1FE053F64F808191818A5BD2
:109DE0009F4F74F480915C08E82FFF27EE0FFF1F50
:109DF000E053F64F80819181863491050CF445E063
:109E0000842F0E94453180915D08E82FFF27EE0FD7
:109E1000FF1FE053F64F808191810190F081E02D8A
:109E2000F7FF03C0F095E195FF4F7E97CCF480914A
:109E30005C08E82FFF27EE0FFF1FE053F64F8081ED
:109E400091818A5B9F4F64F481E08093EB051092CF
:109E50003D0488EE93E090932303809322036BC02C
:109E6000809101010E94F03080E00E94920A80916E
:109E700082080E94549B8091AE0A80FF10C080919E
:109E80001C0190911D01875B934038F480911C0167
:109E900090911D018E5E924010F40E94C61F81E0D9
:109EA0000E94D73C982F80933D0421E0209320030B
:109EB000579A8091D005882311F087E006C0992336
:109EC00019F42093AB0103C088E18093AB0185E0D6
:109ED0008093590527C080819181855B9F4F4CF508
:109EE0008091F4048F5F8093F404893C20F12093E7
:109EF00051042093F40410921B0410921A0482E07F
:109F00000E94D73C982F80933D048091D0058823F0
:109F100011F087E005C0992311F481E001C088E1C8
:109F20008093AB0168E770E0809101010E94FD3BE6
:109F300002C02093F40480915E08E82FFF27EE0F03
:109F4000FF1FE053F64F808191818C599F4F0CF099
:109F500037C22091BF08E22FFF27EF77F070EE0F96
:109F6000FF1FEA5EF54F80819181069714F084E629
:109F700006C0808191818B5F9F4F1CF48CE9809398
:109F8000F70480915104E0915F08882309F063C1D0
:109F9000FF27EE0FFF1FE053F64F808191818C5910
:109FA0009F4F9CF48091CF0883FD0BC0E22FFF27C9
:109FB000EE0FFF1FE053F64F80819181855B9F4F2D
:109FC000DCF08091BF088823B9F08091CF0883FF2F
:109FD0003FC18091BF08E82FFF27EE0FFF1FE0531E
:109FE000F64F80819181875F9F4F0CF431C1809142
:109FF000F704843609F02CC180913D04882329F0B0
:10A000008091190488608093190480911E019091B9
:10A010001F01A0912001B09121018093FD07909331
:10A02000FE07A093FF07B093000810922E03109232
:10A030002F03109230031092310310924C041092AF
:10A040004D0410924E0410924F0410923B03109254
:10A050003C0310923D0310923E0380915C08E82F70
:10A06000FF27EE0FFF1FE053F64F808191818D593E
:10A070009F4FACF480915D08E82FFF27EE0FFF1F84
:10A08000E053F64F808191810190F081E02DF7FF40
:10A0900003C0F095E195FF4FE436F10534F480916B
:10A0A000BF08882311F48093F5048091F5048F5F35
:10A0B0008093F5048E3F08F466C18091B70A9091B1
:10A0C000B80A97FF03C0909581959F4F8197B4F48C
:10A0D0008091740A9091750A97FF03C090958195BD
:10A0E0009F4F45975CF48091650A9091660A97FFAF
:10A0F00003C0909581959F4F459714F010923D04B1
:10A100001092F5048091D005882309F094C08091C5
:10A110003D04882309F48FC080913305882309F01A
:10A120008AC081E090E090931B0480931A0481E040
:10A13000809351041092DE041092DF041092E00428
:10A140001092E10410927C0410927D0410927E041F
:10A1500010927F04109278041092790410927A047D
:10A1600010927B0480917708E82EFF2400271127A6
:10A170008091B20A9091B30A9C01442737FD409523
:10A18000542FC801B7010E94B79FDC01CB01809317
:10A190008C0490938D04A0938E04B0938F048091CF
:10A1A000C20A9091C30A9C01442737FD4095542F61
:10A1B000C801B7010E94B79FDC01CB0180938404E2
:10A1C00090938504A0938604B09387048091AC0497
:10A1D0009091AD04A091AE04B091AF048093880437
:10A1E00090938904A0938A04B0938B048091A40473
:10A1F0009091A504A091A604B091A7048093800437
:10A2000090938104A0938204B09383041092740409
:10A2100010927504109276041092770410927004D4
:10A2200010927104109272041092730484E6809369
:10A230003C0484E39AC08CED95E0909323038093D3
:10A24000220380913D04882309F09DC081E08DC0E8
:10A250001092F50498C0FF27EE0FFF1FE053F64F52
:10A2600080819181853691059CF08091CF0883FD96
:10A270000BC0E22FFF27EE0FFF1FE053F64F808148
:10A280009181855B9F4FDCF08091BF088823B9F0F6
:10A290008091CF0883FF75C08091BF08E82FFF270A
:10A2A000EE0FFF1FE053F64F808191818E5C9F4F30
:10A2B0000CF067C08091F7048C3909F062C080917E
:10A2C0005C08E82FFF27EE0FFF1FE053F64F808159
:10A2D00091818D599F4FACF480915D08E82FFF2745
:10A2E000EE0FFF1FE053F64F808191810190F081C6
:10A2F000E02DF7FF03C0F095E195FF4FE436F1053F
:10A300003CF48091BF08882319F48093F60418C0A8
:10A3100010927404109275041092760410927704CF
:10A3200010927004109271041092720410927304CF
:10A3300010926304109262041092610410926004FF
:10A340008091F6048F5F8093F6048B3F88F0109223
:10A3500051041092F60410921B0410921A0480917A
:10A3600018048F718093180486E28093AB010BC0B0
:10A37000843649F48CEA9DE0909323038093220372
:10A3800002C01092F6042091140430911504F3E0F9
:10A39000283E3F0708F045C080913803909139036B
:10A3A0008B569F4F1CF02F5F3F4F05C02115310585
:10A3B000C1F121503040309315042093140431C072
:10A3C0001092F70410921504109214042AC02E5E05
:10A3D000324038F18091CD0A9091CE0A8059914057
:10A3E00000F580914C0490914D04A0914E04B091E1
:10A3F0004F048C5D9540A040B0409CF480E395E70D
:10A40000909315048093140480911A0490911B0476
:10A410008A5E934030F089EE93E090931B04809322
:10A420001A04809141018150809341018091410142
:10A430008F3F21F08091190484FFDFC30E942C48D4
:10A44000B090720880910005909101059C01220F47
:10A45000331F280F391FC0905C08AC2DBB27AA0FF3
:10A46000BB1FFD01E053F64F4B2D55278081918195
:10A47000849FB001859F700D949F700D1124260F4D
:10A48000371F37FF02C02D5F3F4FB90175956795A4
:10A4900075956795AA5EB54F80917308082F1127AF
:10A4A0008D919C91809FD001819FB00D909FB00DA8
:10A4B00011246A0F7B1F7093010560930005809142
:10A4C0000205909103059C01220F331F280F391FAD
:10A4D000D0905D08AD2DBB27AA0FBB1FFD01E05337
:10A4E000F64F80819181849FF001859FF00D949FAC
:10A4F000F00D11242E0F3F1F37FF02C02D5F3F4F7D
:10A50000A9015595479555954795AA5EB54F8D91EB
:10A510009C91809F7001819FF00C909FF00C112402
:10A520004E0D5F1D50930305409302058091260454
:10A53000882309F448C0CB0177FD0396DC01B5956B
:10A54000A795B595A795CA0157FD0396FC01F5950A
:10A55000E795F595E7958091A601682F772767FD28
:10A5600070956A9F90016B9F300D7A9F300D11247A
:10A5700080913505482F552747FD50954E9FC001C6
:10A580004F9F900D5E9F900D1124280F391F37FFAC
:10A5900002C0295F3F4F03E0359527950A95E1F703
:10A5A00030936304209362046E9F90016F9F300D7F
:10A5B0007E9F300D11244A9FC0014B9F900D5A9FE2
:10A5C000900D11243FC08091BD08E82FFF27E75B65
:10A5D000FE4F86818093A601908190933505A82F28
:10A5E000BB27A7FDB095A69F9001A79F300DB69FF2
:10A5F000300D1124E92FFF27E7FDF095E49FC001FE
:10A60000E59F900DF49F900D1124280F391F37FFFF
:10A6100002C0295F3F4F13E0359527951A95E1F762
:10A620003093630420936204A49F9001A59F300D92
:10A63000B49F300D1124E69FC001E79F900DF69F57
:10A64000900D1124281B390B37FF02C0295F3F4FA3
:10A6500043E0359527954A95E1F7309361042093BF
:10A66000600480915F08E82FFF27EE0FFF1FE05383
:10A67000F64F80819181909581959F4F90935F04D3
:10A6800080935E048530910514F0049705C00FEFA8
:10A690008C3F900734F4049690935F0480935E049B
:10A6A00004C010925F0410925E0480911404909193
:10A6B00015048150924078F1809162049091630476
:10A6C00097FD079623E0959587952A95E1F7909356
:10A6D000630480936204809160049091610497FD0B
:10A6E000079603E0959587950A95E1F790936104A5
:10A6F0008093600410927404109275041092760492
:10A7000010927704109270041092710410927204E7
:10A710001092730443C080912105882309F43EC040
:10A72000282F3327809162049091630497FD079648
:10A7300013E0959587951A95E1F7289FA001299F29
:10A74000500D389F500D1124CA0157FD0F96B4E0EB
:10A7500095958795BA95E1F7909363048093620489
:10A76000809160049091610497FD0796A3E0959510
:10A770008795AA95E1F7289FB001299F700D389F12
:10A78000700D1124CB0177FD0F96F4E09595879518
:10A79000FA95E1F7909361048093600480906204DD
:10A7A000909063048091240590912505881A990A58
:10A7B000909263048092620400916004109161049D
:10A7C0008091220590912305081B190B10936104B9
:10A7D0000093600480915E08E82FFF27EE0FFF1FB3
:10A7E000E053F64FE080F1808FE790E0E80EF91E2D
:10A7F000F0925D04E0925C04809177019927AA278A
:10A8000097FDA095BA2FBC01CD010E942B9FDC01C2
:10A81000CB0120E030E040E251E4BC01CD010E94D8
:10A82000999EDC01CB01BC01CD010E94FD9EDC01A3
:10A83000CB018093BC0A809176018093930A80912A
:10A8400075019927AA2797FDA095BA2FBC01CD01C4
:10A850000E942B9FDC01CB0120E030E040E251E47C
:10A86000BC01CD010E94999EDC01CB01BC01CD0150
:10A870000E94FD9EDC01CB0180936C0A80917401E3
:10A880008093820A8091F70580FF59C08091C50AA4
:10A89000813808F454C08091F005992787FD909580
:10A8A0002B2D3327829FD001839FB00D929FB00D37
:10A8B00011248A0E9B1E9092630480926204809100
:10A8C000F105992787FD9095829FF001839FF00DF8
:10A8D000929FF00D11240E0F1F1F1093610400931F
:10A8E00060048091F205282F332727FD3095809151
:10A8F0005E0490915F04820F931F90935F04809396
:10A900005E048091F405282F332727FD3095809130
:10A910006D089927289F8001299F100D389F100DE1
:10A92000112410934801009347018091F305992762
:10A930008E159F0524F490935D0480935C048091B0
:10A940005C0490915D0497FF04C010925D04109226
:10A950005C048091AE0A82FF02C01092930A40917B
:10A96000620450916304CA0157FD03969C0135951A
:10A9700027953595279537FF03C0309521953F4F93
:10A9800080911E0490911F0482179307B4F4CA01AA
:10A9900057FF03C0909581959F4F97FD039695951E
:10A9A00087959595879590931F0480931E0485360F
:10A9B000910544F084E690E001C0019790931F0454
:10A9C00080931E044091600450916104CA0157FDB8
:10A9D00003969C01359527953595279537FF03C03C
:10A9E000309521953F4F80911C0490911D04821752
:10A9F0009307B4F4CA0157FF03C0909581959F4F08
:10AA000097FD0396959587959595879590931D0449
:10AA100080931C048536910544F084E690E001C0E3
:10AA2000019790931D0480931C048091190484FF66
:10AA300008C010921F0410921E0410921D04109260
:10AA40001C04ED2DFF27EE0FFF1FE053F64F409142
:10AA50009708242F3327808191812817390744F4E0
:10AA60008091CC0882FF04C081E08093330413C03E
:10AA7000ED2DFF27EE0FFF1FE053F64F842F992790
:10AA800020919808821B910920813181281739076C
:10AA900014F41092330440915D08E42FFF27EE0F69
:10AAA000FF1FE053F64F50919708852F99272227D3
:10AAB0003327281B390B808191818217930744F437
:10AAC0008091CC0883FF04C081E08093320416C0DB
:10AAD00080913204882391F0E42FFF27EE0FFF1FAF
:10AAE000E053F64F809198089927851B91092081A2
:10AAF00031818217930714F410923204EC2DFF2752
:10AB0000EE0FFF1FE053F64F40919708242F332795
:10AB1000808191812817390744F48091CC0880FF07
:10AB200004C081E08093300417C0809130048823F2
:10AB300099F0EC2DFF27EE0FFF1FE053F64F842F07
:10AB4000992720919808821B91092081318128172B
:10AB5000390714F41092300440915C08E42FFF2769
:10AB6000EE0FFF1FE053F64F50919708852F99275E
:10AB700022273327281B390B808191818217930765
:10AB800044F48091CC0881FF04C081E080933104BB
:10AB900016C080913104882391F0E42FFF27EE0F37
:10ABA000FF1FE053F64F809198089927851B910964
:10ABB000208131818217930714F41092310480911F
:10ABC0003304882319F480913204811181E0809349
:10ABD000340480913004882321F480913104882347
:10ABE00051F081E0809335041092340410923304C4
:10ABF0001092320402C0809335048091340488237B
:10AC000021F480913504882369F080919608992772
:10AC100029813A818217930714F49A83898381E00A
:10AC2000809368048091180499279C0124703070E7
:10AC300082FF31C0809124059091250590958195E2
:10AC40009F4F9093630480936204809122059091BA
:10AC50002305909581959F4F9093610480936004A4
:10AC6000809183019091840190935D0480935C04B2
:10AC700010925F0410925E048091AE0A8B778B660F
:10AC80008093AE0A8091910A8C7B8093910A88EC24
:10AC900080932F041EC08091190484FF1AC0309342
:10ACA0005F0420935E043093630420936204309326
:10ACB0006104209360049AE59093BC0A88E780932E
:10ACC000930A90936C0A8093820A10923404109233
:10ACD00035048091850A9091860AA091870AB091E7
:10ACE000880A2091AC043091AD044091AE0450919B
:10ACF000AF04820F931FA41FB51F8093850A909302
:10AD0000860AA093870AB093880A80918D0A909151
:10AD10008E0AA0918F0AB091900AE090A404F0905E
:10AD2000A5040091A6041091A704EB82FC820D8378
:10AD30001E838E0D9F1DA01FB11F80938D0A9093BF
:10AD40008E0AA0938F0AB093900A80917A0A90910C
:10AD50007B0AA0917C0AB0917D0AE090A804F09053
:10AD6000A9040091AA041091AB04EF82F886098728
:10AD70001A878E0D9F1DA01FB11F80937A0A909392
:10AD80007B0AA0937C0AB0937D0A80916D0A909112
:10AD90006E0AA0916F0AB091700AE090A004F09042
:10ADA000A1040091A2041091A304EB86FC860D87F8
:10ADB0001E878E0D9F1DA01FB11F80936D0A90935B
:10ADC0006E0AA0936F0AB093700AF0903504FF8664
:10ADD000FF2029F480913404882309F460C0109284
:10ADE0009C0410929D0410929E0410929F04109255
:10ADF00098041092990410929A0410929B04109255
:10AE0000850A1092860A1092870A1092880A109278
:10AE10008D0A10928E0A10928F0A1092900A109248
:10AE20007A0A10927B0A10927C0A10927D0A109284
:10AE30006D0A10926E0A10926F0A1092700A809139
:10AE40008C0490918D04A0918E04B0918F04809316
:10AE5000880490938904A0938A04B0938B04809112
:10AE6000840490918504A0918604B0918704809316
:10AE7000800490938104A0938204B0938304109281
:10AE8000370310923603109239041092380410924E
:10AE90003B0410923A040F85002309F0D0C1809141
:10AEA0003404882309F0CBC18091FB079091FC0703
:10AEB000815092402CF480915104882309F4BFC141
:10AEC00090903E0BA09077082090B20A3090B30A81
:10AED0004090C20A5090C30A19140CF0BBC0BB24A6
:10AEE000CC24DD24CA01B901A60195010E942BA042
:10AEF00079018A018091070B9091080B281A390A71
:10AF0000C101AA2797FDA095BA2FE81AF90A0A0BE2
:10AF10001B0B6B817C818D819E81A60195010E9416
:10AF20002BA059016A018091090B90910A0B481AD4
:10AF3000590AC201AA2797FDA095BA2FA81AB90AE3
:10AF4000CA0ADB0A292C332427FC3094432C532CC7
:10AF5000C801B701A20191010E94B79F97FF04C0E9
:10AF600061507E4F8F4F9F4F3B014C0109E09594FC
:10AF70008794779467940A95D1F7C601B501A20129
:10AF800091010E94B79F97FF04C061507E4F8F4F81
:10AF90009F4F5B016C0119E0D594C794B794A794B7
:10AFA0001A95D1F780911E0490911F048134910568
:10AFB0003CF480911C0490911D0481349105D4F0DF
:10AFC000D401C30197FE03C00196A11DB11D3C0130
:10AFD0004D019594879477946794D601C501D7FE67
:10AFE00003C00196A11DB11D5C016D01D594C794EC
:10AFF000B794A7948091400B282F332727FD3095D5
:10B00000432F532F261537054805590514F43901E8
:10B010004A01992787FD9095909581959F4FAA2782
:10B0200097FDA095BA2F681679068A069B0614F438
:10B030003C014D012A153B054C055D0514F45901F1
:10B040006A01A816B906CA06DB060CF0D0C05C017E
:10B050006D01CDC0EA2CFF2400271127CA01B901D8
:10B06000A80197010E942BA039014A01C101AA271A
:10B0700097FDA095BA2F681A790A8A0A9B0A6B81F4
:10B080007C818D819E81A80197010E942BA059018E
:10B090006A01C201AA2797FDA095BA2FA81AB90A7A
:10B0A000CA0ADB0AD401C30197FE03C00F96A11D93
:10B0B000B11D3C014D01F4E0959487947794679419
:10B0C000FA95D1F7D601C501D7FE03C00F96A11D91
:10B0D000B11D5C016D01E4E0D594C794B794A794C9
:10B0E000EA95D1F780911E0490911F048134910557
:10B0F0003CF480911C0490911D0481349105A4F0CE
:10B10000C401B30123E030E040E050E00E942BA0F6
:10B1100039014A01C601B50123E030E040E050E0CA
:10B120000E942BA059016A0180915F08E82FFF2738
:10B13000EE0FFF1FE053F64F808191810190F08167
:10B14000E02DF7FF03C0F095E195FF4F7A97A4F04B
:10B15000C401B30123E030E040E050E00E942BA0A6
:10B1600039014A01C601B50123E030E040E050E07A
:10B170000E942BA059016A0189E180938F0121E28D
:10B1800062167104810491042CF070E2672E712C18
:10B19000812C912C30EE63163FEF73063FEF830650
:10B1A0003FEF930644F460EE662E6FEF762E6FEF5E
:10B1B000862E6FEF962E41E2A416B104C104D1048D
:10B1C0002CF050E2A52EB12CC12CD12C50EEA5169E
:10B1D0005FEFB5065FEFC5065FEFD50644F440EEBE
:10B1E000A42E4FEFB42E4FEFC42E4FEFD42E8091EC
:10B1F0008C0490918D04A0918E04B0918F048619D7
:10B200009709A809B90980938C0490938D04A093A1
:10B210008E04B0938F048091840490918504A09152
:10B220008604B09187048A199B09AC09BD098093F3
:10B23000840490938504A0938604B093870480913E
:10B240003603909137038F3F910509F008F4C4C588
:10B250006F85662309F04EC580913404882309F078
:10B2600049C580916804882309F044C570919F08FE
:10B27000788B772309F43EC58091850A9091860AE0
:10B28000A091870AB091880AB7FF04C081509F4FF0
:10B29000AF4FBF4FE92EFA2E0B2F112707FD1A953E
:10B2A000E092850AF092860A0093870A1093880A32
:10B2B00080918D0A90918E0AA0918F0AB091900A88
:10B2C000B7FF04C081509F4FAF4FBF4F892F9A2FB8
:10B2D000AB2FBB27A7FDBA95898B9A8BAB8BBC8B09
:10B2E00080938D0A90938E0AA0938F0AB093900A50
:10B2F00080917708A82EBB24CC24DD2420919C04C7
:10B3000030919D0440919E0450919F04C601B50167
:10B310000E94B79F97FF04C061507F4F8F4F9F4F90
:10B32000672E782E892E992487FC9A9460929C042B
:10B3300070929D0480929E0490929F0420919804A4
:10B340003091990440919A0450919B04C601B50133
:10B350000E94B79F97FF04C061507F4F8F4F9F4F50
:10B36000272E382E492E552447FC5A9420929804B3
:10B370003092990440929A0450929B0480919404D4
:10B3800090919504A0919604B0919704B7FF04C0E2
:10B3900081509F4FAF4FBF4F892F9A2FAB2FBB27A5
:10B3A000A7FDBA958093940490939504A093960476
:10B3B000B0939704D801C70186199709A809B9095C
:10B3C0008093EA049093EB04A093EC04B093ED0413
:10B3D00020919E08E22EFF2400271127BC01CD01F9
:10B3E000A80197010E942BA059016A012093F8043B
:10B3F0003093F9044093FA045093FB0489899A89A5
:10B40000AB89BC8982199309A409B5098093EE041C
:10B410009093EF04A093F004B093F104BC01CD012C
:10B42000A80197010E942BA02093FC043093FD04F7
:10B430004093FE045093FF04D601C501D7FE04C01B
:10B4400081509F4FAF4FBF4F892F9A2FAB2FBB27F4
:10B45000A7FDBA95909339048093380457FF04C030
:10B4600021503F4F4F4F5F4FBB2757FDBA95A52F38
:10B47000942F832F90933B0480933A0480911E0471
:10B4800090911F0481349105DCF480911C0490910B
:10B490001D0481349105A4F480915F08E82FFF27F3
:10B4A000EE0FFF1FE053F64F808191810190F081F4
:10B4B000E02DF7FF03C0F095E195FF4F7A97E4F098
:10B4C00080913E0B8F3FC1F48091380490913904F4
:10B4D00097FD01969595879590933904809338044C
:10B4E00080913A0490913B0497FD0196959587953C
:10B4F00090933B0480933A0480917A0A90917B0A5E
:10B50000A0917C0AB0917D0AB7FF04C081509F4F83
:10B51000AF4FBF4F892F9A2FAB2FBB27A7FDBA95EF
:10B5200080937A0A90937B0AA0937C0AB0937D0A59
:10B5300080916D0A90916E0AA0916F0AB091700A85
:10B54000B7FF04C081509F4FAF4FBF4F892F9A2F35
:10B55000AB2FBB27A7FDBA9580936D0A90936E0A17
:10B56000A0936F0AB093700A8091AC049091AD04DF
:10B57000A091AE04B091AF042F81388549855A85DA
:10B58000281B390B4A0B5B0B2093E2043093E30436
:10B590004093E4045093E5048091A4049091A504A1
:10B5A000A091A604B091A704EB84FC840D851E85B0
:10B5B000E81AF90A0A0B1B0BE092E604F092E70482
:10B5C0000093E8041093E9042093EA043093EB0419
:10B5D0004093EC045093ED04E092EE04F092EF04FB
:10B5E0000093F0041093F1048091880490918904F1
:10B5F000A0918A04B0918B04821B930BA40BB50B12
:10B600008093880490938904A0938A04B0938B0458
:10B610008091800490918104A0918204B091830470
:10B620008E199F09A00BB10B809380049093810425
:10B63000A0938204B093830488898823E1F0209149
:10B64000660430916704213831054CF08091BE04C6
:10B650009091BF0401969093BF048093BE0420583C
:10B660003F4F4CF48091BE049091BF04019790939A
:10B67000BF048093BE04109267041092660481E0B8
:10B6800090E09093050580930405E090EA04F09023
:10B69000EB040091EC041091ED04D801C70117FFF1
:10B6A00007C088279927DC018E199F09A00BB10BD1
:10B6B00081509240A040B04034F084E090E09093FC
:10B6C00005058093040580910A0590910B05A091D2
:10B6D0000C05B0910D052091850A3091860A4091A4
:10B6E000870A5091880A821B930BA40BB50B815ECD
:10B6F000914BAF4FBF4F8F539C49A040B04028F0B3
:10B7000080913F0B89310CF4FFC021E0E21620E16B
:10B71000F20620E0020720E012070CF473C08091CB
:10B720000605882309F46AC0D801C70117FF07C0BE
:10B7300088279927DC018E199F09A00BB10B9C016A
:10B74000AD01B7FF04C021503E4F4F4F5F4FF9E0AE
:10B750005595479537952795FA95D1F7809104052A
:10B7600090910505820F931F909305058093040522
:10B77000D801C70117FF03C00796A11DB11DE3E063
:10B78000B595A79597958795EA95D1F78093F80495
:10B790009093F904A093FA04B093FB048958934161
:10B7A000A040B04064F088E893E1A0E0B0E080936E
:10B7B000F8049093F904A093FA04B093FB04209149
:10B7C000F8043091F9044091FA045091FB0457FFBA
:10B7D00004C021503F4F4F4F5F4F232F342F452F31
:10B7E000552747FD5A958091380490913904820F6E
:10B7F000931F909339048093380406C081E08093AE
:10B80000060502C01092060540E0E41640EFF4067B
:10B810004FEF04074FEF14070CF073C0809107053A
:10B82000882309F46AC0D801C70117FF07C0882719
:10B830009927DC018E199F09A00BB10B9C01AD016A
:10B84000B7FF04C021503E4F4F4F5F4F69E0559501
:10B850004795379527956A95D1F780910405909182
:10B860000505820F931F9093050580930405D80169
:10B87000C70117FF03C00796A11DB11D23E0B595B1
:10B88000A795979587952A95D1F78093F80490937B
:10B89000F904A093FA04B093FB0488579C4EAF4F71
:10B8A000BF4F64F488E79CEEAFEFBFEF8093F804DE
:10B8B0009093F904A093FA04B093FB042091F80448
:10B8C0003091F9044091FA045091FB0457FF04C0F1
:10B8D00021503F4F4F4F5F4F232F342F452F552778
:10B8E00047FD5A958091380490913904820F931F37
:10B8F000909339048093380411C081E08093070548
:10B900000DC0109207050AC010920505109204059B
:10B9100084E690E090938E0180938D016889262FB4
:10B92000332780910405909105052817390724F4E1
:10B93000309305052093040510913F0B112379F0F6
:10B94000212F332727FD309580910405909105051F
:10B950002817390724F430930505209304054091F6
:10B96000EA045091EB046091EC047091ED044138CD
:10B9700051056105710574F08091C2049091C30472
:10B980002091040530910505820F931F9093C30405
:10B990008093C20440585F4F6F4F7F4F74F4809183
:10B9A000C2049091C3042091040530910505821BC7
:10B9B000930B9093C3048093C20481E090E0909332
:10B9C000050580930405C090EE04D090EF04E0904C
:10B9D000F004F090F104D701C601F7FE07C08827F4
:10B9E0009927DC018C199D09AE09BF09815092404D
:10B9F000A040B04034F084E090E09093050580933F
:10BA0000040580910E0590910F05A0911005B0914D
:10BA1000110520918D0A30918E0A40918F0A509124
:10BA2000900A821B930BA40BB50B815E914BAF4F19
:10BA3000BF4F8F539C49A040B04018F019310CF40F
:10BA4000FFC001E0C01600E1D00600E0E00600E023
:10BA5000F0060CF473C080910805882309F46AC0CD
:10BA6000D701C601F7FE07C088279927DC018C198A
:10BA70009D09AE09BF099C01AD01B7FF04C021506B
:10BA80003E4F4F4F5F4F09E05595479537952795A6
:10BA90000A95D1F78091040590910505820F931FB7
:10BAA0009093050580930405D701C601F7FE03C0F6
:10BAB0000796A11DB11D13E0B595A795979587959C
:10BAC0001A95D1F78093FC049093FD04A093FE0493
:10BAD000B093FF0489589341A040B04064F088E8D7
:10BAE00093E1A0E0B0E08093FC049093FD04A09368
:10BAF000FE04B093FF042091FC043091FD044091BA
:10BB0000FE045091FF0457FF04C021503F4F4F4F98
:10BB10005F4F232F342F452F552747FD5A9580918E
:10BB20003A0490913B04820F931F90933B048093BF
:10BB30003A0406C081E08093080502C0109208050F
:10BB400020E0C21620EFD2062FEFE2062FEFF2061A
:10BB50000CF073C080910905882309F46AC0D701ED
:10BB6000C601F7FE07C088279927DC018C199D09BB
:10BB7000AE09BF099C01AD01B7FF04C021503E4F83
:10BB80004F4F5F4FE9E05595479537952795EA95D3
:10BB9000D1F78091040590910505820F931F909332
:10BBA000050580930405D701C601F7FE03C007967B
:10BBB000A11DB11D73E0B595A795979587957A95C9
:10BBC000D1F78093FC049093FD04A093FE04B093FE
:10BBD000FF0488579C4EAF4FBF4F64F488E79CEE3C
:10BBE000AFEFBFEF8093FC049093FD04A093FE049D
:10BBF000B093FF042091FC043091FD044091FE04B9
:10BC00005091FF0457FF04C021503F4F4F4F5F4FEB
:10BC1000232F342F452F552747FD5A9580913A04FD
:10BC200090913B04820F931F90933B0480933A04BE
:10BC300011C081E0809309050DC0109209050AC06A
:10BC4000109205051092040584E690E090938E0111
:10BC500080938D014889242F33278091040590918A
:10BC600005052817390724F43093050520930405AA
:10BC700080913F0B882379F0282F332727FD3095BB
:10BC800080910405909105052817390724F4309315
:10BC90000505209304054091EE045091EF04609156
:10BCA000F0047091F104413851056105710574F09B
:10BCB0008091C0049091C104209104053091050544
:10BCC000820F931F9093C1048093C00440585F4F2C
:10BCD0006F4F7F4FCCF48091C0049091C1042091AC
:10BCE000040530910505821B930B9093C10480934A
:10BCF000C0040AC010923B0410923A041092390416
:10BD000010923804109268048091930A882341F4B9
:10BD100010923B0410923A041092390410923804A5
:10BD20008091850A9091860AA091870AB091880A2D
:10BD300080930A0590930B05A0930C05B0930D0515
:10BD400080918D0A90918E0AA0918F0AB091900AED
:10BD500080930E0590930F05A0931005B0931105E5
:10BD600010929C0410929D0410929E0410929F04C5
:10BD7000109298041092990410929A0410929B04C5
:10BD800010929404109295041092960410929704C5
:10BD90001092850A1092860A1092870A1092880AD9
:10BDA00010928D0A10928E0A10928F0A1092900AA9
:10BDB00010927A0A10927B0A10927C0A10927D0AE5
:10BDC00010926D0A10926E0A10926F0A1092700A09
:10BDD0001092370310923603E0905E04F0905F04F7
:10BDE000C701F7FE04C0882799278E199F09049779
:10BDF0003CF08091AE0A84FD03C082E380933C0452
:10BE000010917408A12EBB24CC24DD24B70188270F
:10BE100077FD8095982F9701F7FE04C022273327DE
:10BE20002E193F09442737FD4095542F0E94B79F94
:10BE30009B01AC01C601B5010E94B79F97FF04C0EA
:10BE400061507E4F8F4F9F4F59E09595879577951D
:10BE500067955A95D1F79B01812F99278E9DD00127
:10BE60008F9DB00D9E9DB00D1124CD01B7FD0396A1
:10BE70009595879595958795280F391F809114047E
:10BE8000909115048150924010F020E030E08091B4
:10BE90003E0490913F04280F391F442737FD4095F9
:10BEA000542F2093DE043093DF044093E00450933A
:10BEB000E10480917C0490917D04A0917E04B09176
:10BEC0007F04821B930BA40BB50B80937C0490938F
:10BED0007D04A0937E04B0937F048155934CA040D1
:10BEE000B04064F080E593ECA0E0B0E080937C0487
:10BEF00090937D04A0937E04B0937F0480917C0492
:10BF000090917D04A0917E04B0917F04805B9C435E
:10BF1000AF4FBF4F64F480EB9CE3AFEFBFEF809374
:10BF20007C0490937D04A0937E04B0937F040091E1
:10BF300091011091920117FDFCC08091AE0A83FF20
:10BF4000F8C080919001815080939001882309F07E
:10BF5000F4C08DE0809390018091AC049091AD0489
:10BF6000A091AE04B091AF04B7FF04C081509E4FC2
:10BF7000AF4FBF4F39E0B595A795979587953A95FF
:10BF8000D1F77C0197FF04C0F094E194F108F39499
:10BF90008091A4049091A504A091A604B091A70457
:10BFA000B7FF04C081509E4FAF4FBF4F29E0B595FA
:10BFB000A795979587952A95D1F79C0197FF03C080
:10BFC000309521953F4FE216F3060CF47901B70145
:10BFD000F7FE02C0695F7F4F2B0183E055944794C1
:10BFE0008A95E1F722E030E0420E531E6090BE0ACF
:10BFF0007090BF0A8090C00A9090C10A20914301BE
:10C00000309144014091450150914601C401B30172
:10C010000E942BA059016A0130936B0A20936A0A8F
:10C02000021B130BC801845E9D4F68E671E00E94FD
:10C03000F69F9C01245B304080918D0190918E0190
:10C04000009731F0019790938E0180938D011BC072
:10C0500049E1E416F104BCF4809166049091670410
:10C06000820F931F909367048093660480913C0431
:10C07000882349F0815080933C04882321F4B092B6
:10C080006B04A0926A0480918D0190918E01892B9E
:10C09000F9F480918F019927289FB001299F700D95
:10C0A000389F700D1124CB01B2010E94F69FCB0185
:10C0B000AA2797FDA095BA2F680E791E8A1E9B1E8F
:10C0C0006092BE0A7092BF0A8092C00A9092C10A22
:10C0D00080913C04882369F580916A0490916B04F7
:10C0E00020916A0A30916B0A821B930B845E9D4FEC
:10C0F00068E671E00E94F69F9C01245B30408091CD
:10C100007A0186959927289FD001299FB00D389FE5
:10C11000B00D11249D01B7FF02C0215F3F4F04E025
:10C12000359527950A95E1F730933F0420933E0417
:10C1300004C010923F0410923E048091680488234A
:10C1400081F0109270041092710410927204109297
:10C150007304109274041092750410927604109275
:10C160007704809135048823F1F48091930A282F75
:10C170003327442755278091AC049091AD04A091BA
:10C18000AE04B091AF04BC01CD010E94B79FDC01A9
:10C19000CB01BC01CD0128EF3AE240E050E00E9423
:10C1A0002BA0290102C04424552480913404882303
:10C1B000F1F48091930A282F332744275527809143
:10C1C000A4049091A504A091A604B091A704BC0179
:10C1D000CD010E94B79FDC01CB01BC01CD0128EF4E
:10C1E0003AE240E050E00E942BA0190102C0222454
:10C1F00033248091670A9091680A893C91051CF06C
:10C2000088EC90E005C088539F4F34F488E39FEF9B
:10C210009093680A8093670A8091720A9091730ADA
:10C22000893C91051CF088EC90E005C088539F4F35
:10C2300034F488E39FEF9093730A8093720A80919D
:10C24000740A9091750AAA2797FDA095BA2F20919C
:10C25000BC0AA22EBB24CC24DD24BC01CD01A60146
:10C2600095010E94B79F9B01AC018091670A909154
:10C27000680AAA2797FDA095BA2F17E0880F991F83
:10C28000AA1FBB1F1A95D1F7280F391F4A1F5B1F22
:10C2900057FF04C0215C3F4F4F4F5F4FA6E05595BD
:10C2A000479537952795AA95D1F78201020F131F5D
:10C2B0001093750A0093740A8091650A9091660A3A
:10C2C000AA2797FDA095BA2FBC01CD01A601950123
:10C2D0000E94B79F9B01AC018091720A9091730AF2
:10C2E000AA2797FDA095BA2FF7E0880F991FAA1FDC
:10C2F000BB1FFA95D1F7280F391F4A1F5B1F57FF45
:10C3000004C0215C3F4F4F4F5F4FE6E05595479586
:10C3100037952795EA95D1F77101E20EF31EF09259
:10C32000660AE092650A8091B70A9091B80A880F70
:10C33000991FAA2797FDA095BA2F20916C0A332741
:10C3400044275527BC01CD010E94B79F5B016C01BA
:10C3500097FF08C02FE330E040E050E0A20EB31E8C
:10C36000C41ED51E76E0D594C794B794A7947A9549
:10C37000D1F78091820A282F3327442755278091AF
:10C38000900490919104A0919204B0919304BC0107
:10C39000CD010E94B79FDC01CB01BC01CD0120EF94
:10C3A00035E540E050E00E942BA0B501620F731FFD
:10C3B0007093B80A6093B70A0150104134F080E0DE
:10C3C00090E19093750A8093740A8091740A909119
:10C3D000750A8050904F34F480E090EF9093750A86
:10C3E0008093740A51E0E51650E1F50634F080E0E0
:10C3F00090E19093660A8093650A8091650A909116
:10C40000660A8050904F34F480E090EF9093660A73
:10C410008093650A6150704134F080E090E1909320
:10C42000B80A8093B70A8091B70A9091B80A8050F1
:10C43000904F34F480E090EF9093B80A8093B70A5D
:10C440008091190485FD16C08091020199272091E1
:10C4500026013091270109811A81089F7001099FE7
:10C46000F00C189FF00C1124C701B9010E94E29F43
:10C470007A836983809112058150809312058F3FE2
:10C4800009F05EC08091130590911405892B41F449
:10C4900080912601909127019093140580931305B4
:10C4A0008091260190912701209113053091140568
:10C4B0002817390718F42F5F3F4F09C080912601D4
:10C4C000909127018217930730F421503040309328
:10C4D00014052093130584E6809312058091F202DF
:10C4E000282F332740911305509114054217530705
:10C4F00010F48AE00CC080910001280F311D241730
:10C50000350738F480911004882319F08150809306
:10C5100010048091F102282F33274217530710F49B
:10C5200089E10CC080910001280F311D24173507C7
:10C5300038F480910F04882319F0815080930F0400
:10C54000809110048823D1F080914204909143049B
:10C55000A0914404B0914504B7FD10C08091C80873
:10C560008093410480EE91EBAFEFBFEF80934204E4
:10C5700090934304A0934404B09345048091210315
:10C58000882311F40E94057129813A81220F331FFB
:10C59000220F331F3A8329838091AE0A80FD02C0A7
:10C5A0000C94DD6C80913404882311F00C94DD6CC4
:10C5B00020913504222311F00C94DD6C8091D0057C
:10C5C00099278F779070009711F00C94DD6C3C01E7
:10C5D0008091C4049091C504892B09F044C08091D6
:10C5E0001C0190911D018959934058F087B58A3FED
:10C5F00020F480913A03815011C081E0809320059E
:10C600005EC080911C0190911D018436910530F52A
:10C6100087B58630F8F080913A038F5F80933A03B4
:10C6200095E089029001112480910708821B87BD43
:10C6300087B5809588BD8CE291E090932303809329
:10C6400022038EE591E09093C5048093C4040E9478
:10C650008E1F35C081E080931F0531C020931F05D8
:10C66000209320052CC0709239036092380380918A
:10C670001104882321F081E00E948C9917C08091D9
:10C680004C0490914D04A0914E04B0914F0454E09D
:10C69000880F991FAA1FBB1F5A95D1F780933B03A0
:10C6A00090933C03A0933D03B0933E038091C40458
:10C6B0009091C50401979093C5048093C404809120
:10C6C000AE0A20912F0481FF3CC0223348F58091AF
:10C6D00096018150809396018F3F09F052C080915E
:10C6E000AB01882339F480916904882319F088E22A
:10C6F0008093AB011092690480914C0490914D0499
:10C70000A0914E04B0914F04809348049093490443
:10C71000A0934A04B0934B0481E08093960131C00A
:10C72000273478F18091AB01882339F48091690432
:10C73000882319F487E28093AB0188EC80939601FB
:10C740001DC08091470190914801820F911D209159
:10C750006D083327829FA001839F500D929F500D3B
:10C760001124CA01AA2797FDA095BA2F80934804E7
:10C7700090934904A0934A04B0934B0481E08093C2
:10C7800069048091AC049091AD04A091AE04B09185
:10C79000AF04E0904301F0904401009145011091F5
:10C7A0004601BC01CD01A80197010E942BA05901AF
:10C7B0006A018091A4049091A504A091A604B0916F
:10C7C000A704BC01CD01A80197010E942BA0B901CB
:10C7D000C5010E94799090937F0A80937E0ACC973E
:10C7E00034F08CE390E090937F0A80937E0A8091EE
:10C7F0007E0A90917F0A0E948A7A90937F0A8093A2
:10C800007E0A80E28093420110924704109246040F
:10C8100080916904882309F46EC7809119049927CF
:10C820009C012071307084FD66C78091180482607D
:10C83000809318047091910A872F992741E0842EE4
:10C84000912C8822992280FD04C08091AE0A81FD3E
:10C8500010C0E980FA8030931605209315053093B7
:10C8600047042093460480911904806C8093190436
:10C87000DDC28091190481FFACC200918301109147
:10C880008401C8010F96A0915C04B0915D04B88F3B
:10C89000AF8B8A179B0708F09AC080911F058823E9
:10C8A00009F095C08091190487FF15C08091190483
:10C8B0008F778093190480912E0390912F03A0917C
:10C8C0003003B09131038093480490934904A093BE
:10C8D0004A04B0934B04E090710AEE20D9F18091A4
:10C8E000480490914904A0914A04B0914B04BC01C2
:10C8F000CD0124E630E040E050E00E942BA0AE2CB9
:10C90000BB24CC24DD24A216B306C406D50614F538
:10C9100090924704809246048091AB018823C1F431
:10C9200080914C0490914D04A0914E04B0914F041D
:10C93000BC01CD012FE530E040E050E00E942BA08B
:10C94000A216B306C406D5061CF48AE18093AB0197
:10C950008DE338C08091170590911805459784F0B4
:10C9600080912E0390912F03A0913003B091310359
:10C970008093480490934904A0934A04B0934B04D5
:10C98000809119048064809319042F89388D201BAD
:10C99000310B2F50304037FF03C0309521953F4F6A
:10C9A000309347042093460480911004882349F073
:10C9B000C90163E070E00E94F69F709347046093A2
:10C9C00046048BE2809342011092400437C1C801B3
:10C9D0000F97EF89F88DE817F907C8F52091200522
:10C9E0002223A9F58091190486FF15C080911904AE
:10C9F0008F7B8093190480912E0390912F03A09137
:10CA00003003B09131038093480490934904A0937C
:10CA10004A04B0934B0480911904806880931904F0
:10CA20008F89988D801B910B0F9697FF03C090956F
:10CA300081959F4F909581959F4F90934704809348
:10CA400046048DE28093420120934004F7C08DE3B9
:10CA50008093420160914104662371F12091420468
:10CA6000309143044091440450914504809148041E
:10CA700090914904A0914A04B0914B048217930706
:10CA8000A407B507CCF4809119048064809319043D
:10CA9000862F992790934704809346048AE08093D9
:10CAA00040048EE5809342018091190487FFC6C03F
:10CAB000809119048F7733C0662309F443C0209115
:10CAC00042043091430440914404509145048091C4
:10CAD000480490914904A0914A04B0914B0428174E
:10CAE00039074A075B0774F58091190480688093C1
:10CAF0001904862F9927909581959F4F909347040D
:10CB00008093460486EF8093400486E78093420139
:10CB10008091190486FF92C0809119048F7B8093C5
:10CB2000190480912E0390912F03A0913003B091AE
:10CB300031038093480490934904A0934A04B0932E
:10CB40004B047CC080911904807C09F477C08091EB
:10CB50004004882309F04CC080912E0390912F034C
:10CB6000A0913003B0913103885C9040A040B04068
:10CB7000209148043091490440914A0450914B045B
:10CB800082179307A407B5076CF080912E0390914C
:10CB90002F03A0913003B0913103885C9040A040F6
:10CBA000B0401DC080912E0390912F03A0913003BF
:10CBB000B091310388539F4FAF4FBF4F28173907AC
:10CBC0004A075B07BCF080912E0390912F03A09140
:10CBD0003003B091310388539F4FAF4FBF4F8093C5
:10CBE000480490934904A0934A04B0934B0402C0B4
:10CBF00010924004809119048F738093190410924D
:10CC000016051092150571FF06C084EF91E0909310
:10CC100023038093220380915004882379F4809128
:10CC20004C0490914D04A0914E04B0914F04C397D1
:10CC3000A105B1051CF081E08093500460911505B9
:10CC4000709116058091460490914704680F791FF2
:10CC50007093160560931505CB0177FF04C08827F4
:10CC60009927861B970B855F91400CF49BC04091E0
:10CC70004004442389F1809142049091430420911F
:10CC8000480430914904821B930B0996439748F45A
:10CC90008091420490914304A0914404B0914504D2
:10CCA00012C0242F332727FD3095432F532F809117
:10CCB000480490914904A0914A04B0914B04820F1A
:10CCC000931FA41FB51F8093480490934904A09319
:10CCD0004A04B0934B0424C0209148043091490485
:10CCE00040914A0450914B0480916D081616170626
:10CCF00044F463E00E94D69F280F311D411D511D51
:10CD000007C063E00E94D69F281B310941095109E1
:10CD1000209348043093490440934A0450934B04B1
:10CD20001092160510921505E0904C04F0904D04F9
:10CD300000914E0410914F04D801C70180509440D7
:10CD4000A040B040209148043091490440914A04E9
:10CD500050914B0482179307A407B5075CF4D801E0
:10CD6000C70180509C4FAF4FBF4F281739074A0764
:10CD70005B0744F08093480490934904A0934A04CD
:10CD8000B0934B048091910A81FF06C084E690E045
:10CD9000909323038093220380914104882311F40C
:10CDA0000E94554B8091C4049091C504892BD1F108
:10CDB00080912E0390912F03A0913003B091310305
:10CDC0008093480490934904A0934A04B0934B0481
:10CDD00029C080914C0490914D04A0914E04B091D3
:10CDE0004F0480599140A040B040809348049093F4
:10CDF0004904A0934A04B0934B048091710888239E
:10CE000011F0992702C08FE790E0909384018093FE
:10CE10008301E980FA80F0923704E09236048EE2D2
:10CE200080934201E0903604F090370480912E0305
:10CE300090912F03A0913003B091310320914804C9
:10CE40003091490440914A0450914B042817390706
:10CE50004A075B0724F08091910A80FD5EC48091AF
:10CE600011046091C4047091C504882309F07CC248
:10CE7000672B49F0E0903604F090370410921805C3
:10CE800010921705E1C080912E0390912F03A0917D
:10CE90003003B0913103821B930BA40BB50B80932D
:10CEA000E2049093E304A093E404B093E504823099
:10CEB00000E890070FEFA0070FEFB0072CF481E018
:10CEC00090E8AFEFBFEF09C08F5F9F47A040B04031
:10CED00064F08FEF9FE7A0E0B0E08093E2049093CE
:10CEE000E304A093E404B093E5048091E2049091FC
:10CEF000E304909318058093170580917C01282FF7
:10CF00003327442755278091E2049091E304A091B0
:10CF1000E404B091E504BC01CD010E94B79F97FFE6
:10CF200004C0615E7F4F8F4F9F4F25E09595879599
:10CF3000779567952A95D1F76093E2047093E3049F
:10CF40008093E4049093E50465302EEF72072FEF91
:10CF500082072FEF92072CF484E09EEFAFEFBFEF34
:10CF600009C0605074408040904064F080E094E0DC
:10CF7000A0E0B0E08093E2049093E304A093E40483
:10CF8000B093E5046090E2047090E30420913803CC
:10CF90003091390337FF02C0295F3F4F03E03595D9
:10CFA00027950A95E1F74FEF223834071CF421E862
:10CFB0003FEF05C02038310514F020E830E0C9010A
:10CFC000AA2797FDA095BA2F20917D0133274427EA
:10CFD0005527BC01CD010E94B79F97FF04C06D5F2C
:10CFE0007F4F8F4F9F4F12E0959587957795679567
:10CFF0001A95D1F79B015FEF613075071CF420E0B3
:10D000003FEF06C06F3F710519F014F020E031E0EA
:10D0100080911904807C49F0C90137FD03969C0179
:10D0200035952795359527950DC08091910A80FFFC
:10D0300009C0C90137FD07969C01A3E035952795E6
:10D04000AA95E1F7620E731E20917B01222309F459
:10D0500054C060916C0470916D0480916E04909145
:10D060006F0497FF04C061587F4F8F4F9F4FF7E0C9
:10D070009595879577956795FA95D1F73327442746
:10D0800055270E94B79F97FF04C0615E7F4F8F4F67
:10D090009F4FE5E09595879577956795EA95D1F748
:10D0A0006093E2047093E3048093E4049093E504B6
:10D0B0006138AFEF7A07AFEF8A07AFEF9A072CF42A
:10D0C00080E89FEFAFEFBFEF0AC06F3F71058105AA
:10D0D000910569F064F080E091E0A0E0B0E0809319
:10D0E000E2049093E304A093E404B093E5048091F8
:10D0F000E2049091E304680E791E80917901282F53
:10D1000033278091420B992787FD9095289FF00146
:10D11000299FF00D389FF00D11249F01F7FF02C0E9
:10D1200021583F4F220F232F221F330BFFEF2138AF
:10D130003F071CF420E83FEF06C02F3F310519F0F0
:10D1400014F020E031E0260D371DC901AA2797FD14
:10D15000A095BA2F00913604109137049801442706
:10D1600037FD4095542FBC01CD010E94B79F97FF1A
:10D1700004C061507E4F8F4F9F4F59E09595879522
:10D18000779567955A95D1F7E61AF70A8091460484
:10D1900090914704892B09F064C0101611060CF019
:10D1A00060C02091170530911805C90137FF03C0F1
:10D1B000309521953F4F2D33310540F48091640423
:10D1C000909165048E159F0574F526C02C53304050
:10D1D00045E0369527954A95E1F72031310510F065
:10D1E0002FE030E040916404509165041816190650
:10D1F000E4F480E190E0821B930B489F9001499FEB
:10D20000300D589F300D1124B4E036952795BA950E
:10D21000E1F72E153F0520F5809181019091820163
:10D22000E816F906F4F07C011CC0205F3F4F8091A6
:10D23000810190918201829FB001839F700D929F26
:10D24000700D11249B01A4E036952795AA95E1F76E
:10D250004E155F0514F07A0104C0E216F30608F0DB
:10D260007901C701AA2797FDA095BA2FFDE0880F85
:10D27000991FAA1FBB1FFA95D1F720917E0A309102
:10D280007F0A442737FD4095542FBC01CD010E94F1
:10D290002BA02093E6043093E7044093E8045093D6
:10D2A000E904E090E604F090E7048091190590917C
:10D2B0001A059C01220F331F280F391F2E0D3F1D09
:10D2C00037FF02C02D5F3F4FA901559547955595F2
:10D2D000479550931A054093190580916908282FA6
:10D2E0003327220F331F220F331F241735076CF407
:10D2F0008091B60A282F3327220F331F220F331FA6
:10D30000205530404217530724F030931A052093DC
:10D3100019058091910A80FF14C0809119059091A0
:10D320001A05A981BA818A179B0724F0B0931A05C0
:10D33000A0931905E0911905F0911A05FA83E98384
:10D34000ECC129813A81201B310B37FF02C02D5FD0
:10D350003F4F3595279535952795E0901905F09025
:10D360001A05E20EF31EC1C1672B49F0E0903604A6
:10D37000F0903704109218051092170538C180916B
:10D380002E0390912F03A0913003B0913103821BA3
:10D39000930BA40BB50B8093E2049093E304A0934A
:10D3A000E404B093E504823000E890070FEFA00793
:10D3B0000FEFB0072CF481E090E8AFEFBFEF09C0AA
:10D3C0008F5F9F47A040B04064F08FEF9FE7A0E0E1
:10D3D000B0E08093E2049093E304A093E404B0935C
:10D3E000E5048091E2049091E30490931805809302
:10D3F000170580917C01282F3327442755278091DA
:10D40000E2049091E304A091E404B091E504BC012E
:10D41000CD010E94B79F97FF04C0615E7F4F8F4F81
:10D420009F4F05E095958795779567950A95D1F774
:10D430006093E2047093E3048093E4049093E50422
:10D44000653028EF72072FEF82072FEF92072CF439
:10D4500084E098EFAFEFBFEF09C0605078408040A4
:10D46000904064F080E098E0A0E0B0E08093E204B7
:10D470009093E304A093E404B093E5046090E20485
:10D480007090E30480917B01282F332780913F0324
:10D4900090914003829FA001839F500D929F500D59
:10D4A00011249A0157FF02C021503F4F232F330F01
:10D4B000330B8091380390913903820F931FAA2771
:10D4C00097FDA095BA2F8093E2049093E304A09374
:10D4D000E404B093E5048091400420914604309127
:10D4E0004704882331F0B3E0220F331FBA95E1F7E8
:10D4F0001BC080916D089927289FB001299F700D4E
:10D50000389F700D11249B01A3E0220F331FAA95B1
:10D51000E1F7260F371F37FF02C0215E3F4FF5E0CE
:10D5200035952795FA95E1F730931304209312046B
:10D5300080911204909113049C01442737FD40957B
:10D54000542F8091E2049091E304A091E404B091FF
:10D55000E504821B930BA40BB50B8093E20490931C
:10D56000E304A093E404B093E50420917D01332704
:10D5700044275527BC01CD010E94B79F97FF04C0E7
:10D58000615E7F4F8F4F9F4FE5E09595879577952B
:10D590006795EA95D1F76093E2047093E304809372
:10D5A000E4049093E5046530A8EF7A07AFEF8A07AB
:10D5B000AFEF9A072CF484E098EFAFEFBFEF09C00C
:10D5C000605078408040904064F080E098E0A0E0B7
:10D5D000B0E08093E2049093E304A093E404B0935A
:10D5E000E5048091E2049091E304680E791EE61848
:10D5F000F70880916404909165048E159F053CF4B2
:10D600008091810190918201E816F9060CF07C016D
:10D61000C701AA2797FDA095BA2F5DE0880F991F33
:10D62000AA1FBB1F5A95D1F720917E0A30917F0A1D
:10D63000442737FD4095542FBC01CD010E942BA0FB
:10D640002093E6043093E7044093E8045093E90400
:10D65000E090E604F090E7048091190590911A0596
:10D660009C01220F331F280F391F2E0D3F1D37FF3E
:10D6700002C02D5F3F4FA901559547955595479598
:10D6800050931A054093190580916908282F332774
:10D69000220F331F220F331F241735076CF480919C
:10D6A000B60A282F3327220F331F220F331F20558E
:10D6B00030404217530724F030931A052093190580
:10D6C0008091910A2091190530911A0580FF10C0B0
:10D6D000E981FA812E173F0724F0F0931A05E093B1
:10D6E0001905E0901905F0901A05FA82E98215C033
:10D6F0003A83298312C00E94554B09811A811093E5
:10D700001A050093190580911904806C80931904FF
:10D71000809118048D7F80931804809119049927B3
:10D720009C012270307081FF39C180911B0590915E
:10D730001C05A0911D05B0911E050097A105B1051E
:10D7400021F0809150048130B9F480913604909199
:10D750003704AA2797FDA095BA2F1EE0880F991FBE
:10D76000AA1FBB1F1A95D1F780931B0590931C0528
:10D77000A0931D05B0931E0580915004813019F4CB
:10D7800082E08093500429813A8179010027F7FCD7
:10D790000095102F80917E0A90917F0A9C0144276A
:10D7A00037FD4095542FC801B7010E94B79FDC0197
:10D7B000CB018093E6049093E704A093E804B09330
:10D7C000E904B7FF04C08150904EAF4FBF4F7C01BA
:10D7D0008D01FDE015950795F794E794FA95D1F73B
:10D7E000E092E604F092E7040093E8041093E90461
:10D7F00060911A0470911B043FE0603A730750F582
:10D8000080911B0590911C05A0911D05B0911E05EE
:10D810009C01AD01EAE05695479537952795EA9525
:10D82000D1F7821B930BA40BB50BA8019701F4E071
:10D83000220F331F441F551FFA95D1F7820F931FF4
:10D84000A41FB51F80931B0590931C05A0931D0575
:10D85000B0931E0560547F4118F580911B0590918F
:10D860001C05A0911D05B0911E059C01AD01ECE0C9
:10D870005695479537952795EA95D1F7821B930BD7
:10D88000A40BB50BA801970172E0220F331F441FB0
:10D89000551F7A95D1F7820F931FA41FB51F41C062
:10D8A0008091380390913903809138039091390326
:10D8B00097FF03C0909581959F4F84369105CCF5D5
:10D8C00080912E0390912F03A0913003B0913103EA
:10D8D0009C018091480490914904281B390B37FF23
:10D8E00003C0309521953F4F2F3F310509F00CF5CE
:10D8F00080911B0590911C05A0911D05B0911E05FE
:10D900009C01AD016EE056954795379527956A9530
:10D91000D1F7821B930BA40BB50B8E0D9F1DA01F7F
:10D92000B11F80931B0590931C05A0931D05B09318
:10D930001E0580911B0590911C05A0911D05B091BD
:10D940001E051EE0B695A795979587951A95D1F770
:10D95000909337048093360440916F08442399F0E4
:10D9600055279C01BA010E94F69FC901861B970B9F
:10D970009093650480936404260F371F30938201CF
:10D98000209381011FC010926504109264048FEFF0
:10D9900093E0909382018093810114C0109250040F
:10D9A00010921B0510921C0510921D0510921E0569
:10D9B000309337042093360405C080911904806C9D
:10D9C0008093190480912F0581FF37C089819A8146
:10D9D00097FD0396959587959595879520911604C3
:10D9E000309117042817390760F48091360490911C
:10D9F0003704892B31F0220F331F220F331F3A8354
:10DA0000298380912E0390912F03A0913003B09130
:10DA100031038093480490934904A0934A04B0933F
:10DA20004B0488E99AE3909323038093220380E0D8
:10DA30009EE090930C0180930B012091790A822F34
:10DA40009927880F991F880F991F889669817A8175
:10DA50008617970714F09A8389838091B60A9927CD
:10DA6000880F991F880F991F80559040A981BA810E
:10DA70008A179B0714F49A83898380917203882301
:10DA800041F48091540B8E3F20F080913305882320
:10DA900021F180911A0490911B040297C097E8F439
:10DAA000E981FA811E161F06C4F481E090E090938C
:10DAB0001B0480931A04E22EFF24EE0CFF1CEE0CD4
:10DAC000FF1C8701085D1F4F1A8309838091540B47
:10DAD000883218F489E08093AB0180912103882378
:10DAE00011F40E94057129813A813093C507209372
:10DAF000C4078091DE049091DF04A091E004B0910E
:10DB0000E10442E0880F991FAA1FBB1F4A95D1F775
:10DB10000091B70A1091B80A081B190B213A310578
:10DB20008CF0C90137FD019695958795801791076F
:10DB30000CF48C01909581959F4F081719076CF490
:10DB40008C010BC00135110514F000E510E03FEF2A
:10DB5000003B130714F400EB1FEF8091B60A282F47
:10DB60003327220F331F220F331FC90149815A81E6
:10DB7000841B950B801791070CF48C0169817A81C5
:10DB8000621B730B061717070CF48B018091740A44
:10DB90009091750A6091620470916304861B970BE3
:10DBA0009093840A8093830AD090930A20917404FE
:10DBB000309175044091760450917704DD2041F056
:10DBC000461A570AC201AA2797FDA095BA2F04C08A
:10DBD000AA2797FDA095BA2F280F391F4A1F5B1F50
:10DBE0002093740430937504409376045093770423
:10DBF0008091740490917504A0917604B09177049B
:10DC000081509A4FA040B04064F080E09AEFA0E0CD
:10DC1000B0E08093740490937504A0937604B0935D
:10DC200077048091740490917504A0917604B0916A
:10DC3000770480509640AF4FBF4F64F480E096E089
:10DC4000AFEFBFEF8093740490937504A0937604B4
:10DC5000B0937704C0907E082091830A3091840AA3
:10DC6000F8E0FC1598F08C2D9927829F7001839F16
:10DC7000F00C929FF00C1124C701F7FC07967C0171
:10DC8000B3E0F594E794BA95E1F712C08C2D869530
:10DC90009927829FA001839F500D929F500D1124C0
:10DCA000CA0157FD03967C01F594E794F594E79437
:10DCB000A0907E01B0907F019501442737FD4095EB
:10DCC000542F8091740490917504A0917604B091C2
:10DCD0007704BC01CD010E942BA0E20EF31E9090B0
:10DCE0006801692D772788279927980117FF04C0B5
:10DCF00022273327201B310B37FF02C02F5F3F4FF6
:10DD000035952795A981BA812A0F3B1F442737FDF6
:10DD10004095542F0E94B79F97FF04C0615C7F4FCE
:10DD20008F4F9F4FE6E09595879577956795EA9594
:10DD3000D1F79B016E157F050CF47B013095219581
:10DD40003F4FE216F3060CF479018091650A909139
:10DD5000660A6091600470916104861B970B909332
:10DD6000640A8093630A2091700430917104409199
:10DD7000720450917304DD2041F0261A370AC10164
:10DD8000AA2797FDA095BA2F04C0AA2797FDA095B2
:10DD9000BA2F280F391F4A1F5B1F2093700430933E
:10DDA00071044093720450937304809170049091B5
:10DDB0007104A0917204B091730481509A4FA040F5
:10DDC000B04064F080E09AEFA0E0B0E0809370048F
:10DDD00090937104A0937204B093730480917004C3
:10DDE00090917104A0917204B09173048050964098
:10DDF000AF4FBF4F64F480E096E0AFEFBFEF80938A
:10DE0000700490937104A0937204B09373042091F2
:10DE1000630A3091640A48E04C1598F08C2D9927DC
:10DE2000829FB001839F700D929F700D1124CB01D2
:10DE300077FD07966C0163E0D594C7946A95E1F786
:10DE400012C0C6948C2D9927829FD001839FB00D5C
:10DE5000929FB00D1124CD01B7FD03966C01D594AE
:10DE6000C794D594C7949501442737FD4095542F06
:10DE70008091700490917104A0917204B091730428
:10DE8000BC01CD010E942BA0C20ED31E692D7727A5
:10DE900088279927980117FF04C022273327201BC2
:10DEA000310B37FF02C02F5F3F4F35952795E98132
:10DEB000FA812E0F3F1F442737FD4095542F0E94B3
:10DEC000B79F97FF04C0615C7F4F8F4F9F4F36E035
:10DED00095958795779567953A95D1F79B016C1540
:10DEE0007D050CF46B01309521953F4FC216D3068A
:10DEF0000CF4690180912103882311F40E940571BB
:10DF00008091790A282F33273E8B2D8B8091B60A7A
:10DF1000282E33245090C0082FE6A22E29E0B22EDE
:10DF20009AEE892E98E0992E8BE0482EB4E96B2E5C
:10DF3000BAE07B2ED4012C9112160CF02FC12034A4
:10DF400029F4E981FA81F88FEF8B1FC049815A814A
:10DF5000CA01AA2797FDA095BA2F332727FD309530
:10DF6000432F532FBC01CD010E94B79F97FF04C0E0
:10DF7000615C7F4F8F4F9F4FA6E095958795779572
:10DF80006795AA95D1F7788F6F8BF40121812034A2
:10DF900039F42F89388D2E0D3F1D388F2F8B2AC0D5
:10DFA000203C39F44F89588D4E195F09588F4F8B9B
:10DFB00021C0C701AA2797FDA095BA2F332727FDB7
:10DFC0003095432F532FBC01CD010E94B79F97FF7F
:10DFD00004C0615C7F4F8F4F9F4FF6E0959587950A
:10DFE00077956795FA95D1F7AF89B88DA60FB71FCA
:10DFF000B88FAF8BF4012281203439F42F89388D0A
:10E000002C0D3D1D388F2F8B2AC0203C39F44F89B1
:10E01000588D4C195D09588F4F8B21C0C601AA2716
:10E0200097FDA095BA2F332727FD3095432F532F07
:10E03000BC01CD010E94B79F97FF04C0615C7F4F78
:10E040008F4F9F4FE6E09595879577956795EA9571
:10E05000D1F7AF89B88DA60FB71FB88FAF8BF4017A
:10E060002381203439F42F89388D200F311F388FC8
:10E070002F8B2AC0203C39F44F89588D401B510BFF
:10E08000588F4F8B21C0C801AA2797FDA095BA2FA2
:10E09000332727FD3095432F532FBC01CD010E941C
:10E0A000B79F97FF04C0615C7F4F8F4F9F4F56E033
:10E0B00095958795779567955A95D1F7AF89B88DDE
:10E0C000A60FB71FB88FAF8BF501808181FD08C007
:10E0D000D3018D919C91EF89F88D8E179F0774F471
:10E0E000D3018D919C91EF89F88D8E0F9F1F97FD25
:10E0F000019695958795988F8F8B1EC0552049F472
:10E100002F89388D220F331F281B390B388F2F8B07
:10E1100013C031E0351580F4252D33274F89588DF4
:10E12000841B950BB9010E94F69FCB016F89788DF6
:10E13000680F791F788F6F8B8D899E89880F991F43
:10E14000880F991FAF89B88D8A179B0754F4C101B6
:10E15000880F991F880F991FEF89F88DE817F90725
:10E1600014F0988F8F8B8F89988D97FD03969595D6
:10E17000879595958795F5018183880F991F880F5D
:10E18000991F2F89388D281B390BC901880F82836D
:10E19000EF89F88DD301ED93FC9303C0F501118253
:10E1A00012824A9422E030E0620E731E44E050E096
:10E1B000840E951E68E070E0A60EB71E47FEBACE2C
:10E1C000E2E1C85E0C9462A084B1806A84B93D9A91
:10E1D00082E58CBD1DBC459A81E08093C80A8AEA1D
:10E1E0008093D90A83E88093DA0A8AE08093DB0A75
:10E1F0001092DD0A1092DC0A1092DF0A1092DE0AF9
:10E200001092410B1092FD0A08953091C80A3323F1
:10E2100009F070C00DB407FE6DC085E08093210346
:10E22000459A2EB58091360599278130910589F060
:10E23000823091051CF4892B21F03EC00297B9F081
:10E240003BC03093FC0A209337052138A9F581E0C3
:10E2500008C0253549F480913705820F8093370532
:10E2600082E08093360528C03093360525C0809122
:10E27000FC0AE82FFF27E25EF44F20838F5F809334
:10E28000FC0A909137058032A0F0291769F480E2EA
:10E29000AEE1BBE0EEEFFAE00D9001928A95E1F776
:10E2A00081E08093FD0A02C03093FD0A109236058A
:10E2B00003C0920F909337052091D80A2232A0F420
:10E2C00045980000000000000000E091D10AF091A4
:10E2D000D20AE20FF11D80818EBD8091FA0A9081F1
:10E2E000890F8093FA0A03C081E08093C80A2F5FE8
:10E2F0002093D80A0895EF92FF920F931F93809175
:10E3000077089927880F991F880F991F7C0100278C
:10E31000F7FC0095102F8091AC049091AD04A09172
:10E32000AE04B091AF04BC01CD01A80197010E94D9
:10E330002BA03093DD0A2093DC0A8091A4049091F5
:10E34000A504A091A604B091A704BC01CD01A80129
:10E3500097010E942BA03093DF0A2093DE0A2091C0
:10E36000BE0A3091BF0A4091C00A5091C10ADA0139
:10E37000C90173E0880F991FAA1FBB1F7A95D1F7B7
:10E38000820F931FA41FB51F820F931FA41FB51FD9
:10E390002091430130914401409145015091460143
:10E3A000BC01CD010E942BA03093E50A2093E40A22
:10E3B0008091BE049091BF042091450330914603A3
:10E3C000821B930B9093EB0A8093EA0AE091B404CA
:10E3D000F091B50480918A0A90918B0ABF010E9446
:10E3E000F69FCB019B01220F331F220F331F280FF3
:10E3F000391F280F391F37FF02C02D5F3F4F35955A
:10E400002795359527953093E10A2093E00A80916E
:10E41000BA0A9091BB0ABF010E94F69F9B01220F8E
:10E42000331F220F331F260F371F260F371F37FFCB
:10E4300002C02D5F3F4F3595279535952795309331
:10E44000E30A2093E20A1092B5041092B4041092E9
:10E450008B0A10928A0A1092BB0A1092BA0A809113
:10E46000DB0A9927AA27BB27FC013A97E830F10578
:10E4700008F03BC2E559FF4F0C947DA080912E041B
:10E480008093EE0A80912D048093EF0A80912C04F2
:10E490008093F00A80912B048093F10A80912A04E2
:10E4A0008093F20A809129048093F30A80912804D2
:10E4B0008093F40A809127048093F50A80911904CF
:10E4C0008093F60A80911904837F809319048091C8
:10E4D00001018093F70A8091260190912701809392
:10E4E000F80A809118048093F90A4299FEC180913C
:10E4F0001804877F80931804F8C180914E0B909187
:10E500004F0B9093EF0A8093EE0A8091520B9091FB
:10E51000530B9093F10A8093F00A8091AC080E940B
:10E5200010488093F20A809142018093F30A9091FF
:10E5300038059093F40AE92FFF2713E0EE0FFF1F31
:10E540001A95E1F7E159F64F80818093F50A8681AB
:10E550008093F60A83818093F70A87818093F80A73
:10E5600085818093F90A9F5F90933805E92FFF27F3
:10E57000EE0FFF1FEE0FFF1FE352F74F85851816B2
:10E580000CF4B3C1992309F4B0C1892F99270196DE
:10E590006DE070E00E94F69F9C01982FE82FFF2706
:10E5A000EE0FFF1FEE0FFF1FE352F74F8585181682
:10E5B00014F0222351F72093380597C1809102016E
:10E5C0008093EE0A8091AD088093EF0A8091AE08A7
:10E5D0008093F00A8091AF088093F10A8091B0088F
:10E5E0008093F20A8091B4088093F30A8091B50871
:10E5F0008093F40A8091B6088093F50A8091B90857
:10E600008093F60A8091B7088093F70A8091B80842
:10E610008093F80A8091BA0866C18091AB08809314
:10E62000EE0A80918208863081F08091E90282347E
:10E6300051F00E94177CE82FFF27E95BFD4E849183
:10E640008093E90202C00E94177C80915A05809352
:10E65000EF0A8091C8088093F00A8091C1088093E6
:10E66000F10A80910F048093F20A809161058093F2
:10E67000F30A1092610539C1F89480915E08E82F81
:10E68000FF27EE0FFF1FE053F64F0190F081E02DC2
:10E69000E038F1051CF0EFE7F0E006C02FEFE138BD
:10E6A000F20714F4E1E8FFEFE093EE0A80915F08CF
:10E6B000E82FFF27EE0FFF1FE053F64F0190F08188
:10E6C000E02DE038F1051CF0EFE7F0E006C07FEF49
:10E6D000E138F70714F4E1E8FFEFE093EF0A8091E7
:10E6E0005D08E82FFF27EE0FFF1FE053F64F019064
:10E6F000F081E02DE038F1051CF0EFE7F0E006C016
:10E700008FEFE138F80714F4E1E8FFEFE093F00A47
:10E7100080915C08E82FFF27EE0FFF1FE053F64FB4
:10E720000190F081E02DE038F1051CF0EFE7F0E01A
:10E7300006C02FEFE138F20714F4E1E8FFEF789418
:10E74000E093F10A809153048093F20A809154047B
:10E750008093F30A809155048093F40A80915604C3
:10E760008093F50A809157048093F60A80915804AB
:10E770008093F70A809159048093F80A80915A0493
:10E78000B2C08091EB05853018F01092EB0585E062
:10E790008093EE0A8091BB088093EF0A80914C042D
:10E7A00090914D04A0914E04B0914F04BC01CD0155
:10E7B00025E030E040E050E00E942BA03093F10AC9
:10E7C0002093F00A8091480490914904A0914A0452
:10E7D000B0914B04BC01CD0125E030E040E050E0B9
:10E7E0000E942BA03093F30A2093F20A8091B10883
:10E7F0008093F40A8091B2088093F50A8091B3085F
:10E800008093F60A809152048093F70A809139052B
:10E810008093F80A8091C4079091C50797FD0396ED
:10E8200095958795959587955EC082E08093EE0AD1
:10E8300084E08093EF0A1092F00A8CE38093F10A4F
:10E84000809103018093F20A8091D0058093F30AAE
:10E850009091D1059093F40A8F778093D0059071B1
:10E860009093D1058091C9088093F50A8091AE0AF2
:10E870008093F60A8091910A8093F70A8091BD08EF
:10E880008093F80A8091CF082EC0809190088093E1
:10E89000EE0A8091CD088093EF0A809170018093F9
:10E8A000F00A809189088093F10A80918A08809308
:10E8B000F20A80918B088093F30A80916F01809314
:10E8C000F40A80918D088093F50A80918E088093D8
:10E8D000F60A80918F088093F70A8091540B8093F9
:10E8E000F80A8091EE078093F90A8091FD0A882347
:10E8F00009F47DC16091FE0A8091A701681719F0A3
:10E900008AEF8093A5016093A70181E08093900135
:10E910004091FF0A5091000BCA0181509E4F8F5FBA
:10E920009340B0F42091010B3091020BC90181504A
:10E930009E4F8F5F934060F48091680885FF08C008
:10E9400050932505409324053093230520932205F9
:10E950008091050B9091060B21E08936920724F4F3
:10E96000909392018093910120910F0B3091100BA5
:10E9700080912203909123038217930740F48091A2
:10E98000F302882321F43093230320932203862F5C
:10E9900099278936910509F4A5C08A36910544F472
:10E9A0008736910571F08836910509F462C027C158
:10E9B0008A36910509F418C18B36910509F4E2C035
:10E9C0001EC18091110B80933E0B8091120B80939E
:10E9D000400B8091130B80933F0B8091140B80931D
:10E9E0008F018091150B8093420B8091160B8093C1
:10E9F000A6018091170B809335058091180B8093A9
:10EA00002105809126048823F9F02091190B30917B
:10EA10001A0B37FD19C030936B0420936A04909150
:10EA20009208992389F08FE0989FC0011124281B38
:10EA3000390BC90188599E4F68E671E00E94F69F24
:10EA400090936B0480936A0420912C0530912D05DE
:10EA500080911B0B90911C0B280F391F37FF02C0B0
:10EA60002F5F3F4F3595279530932D0520932C052B
:10EA7000C6C08091110B8093D30A8091120B8093B2
:10EA8000D40A8091130B8093D50A8091140B809344
:10EA9000D60A8091150B8093D70A8091B407909184
:10EAA000160B892B8093B4079091B50793708091D2
:10EAB000170B8C70982B9093B5078091180B80934F
:10EAC00033058091190B8093970180911A0B8093E5
:10EAD000410B80911B0B80932F0580911C0B809321
:10EAE0002E058DC08091110B8093C90A8091120B65
:10EAF0008093CA0A8091130B8093CB0A8091140BE8
:10EB00008093CC0A8091150B9091160B9093CE0AAE
:10EB10008093CD0A8091170B9091180B9093D00A97
:10EB20008093CF0A8091190B992787FD9095909338
:10EB30000B0A80930A0A80911A0B809341048091FA
:10EB40001B0B90911C0B9C01442737FD4095542FC3
:10EB5000DA01C90163E0880F991FAA1FBB1F6A95DC
:10EB6000D1F7820F931FA41FB51F820F931FA41FFD
:10EB7000B51F8093420490934304A0934404B09340
:10EB800045043DC08091110B809332058091120B9A
:10EB9000809331058091130B809330059091140B75
:10EBA000992349F08091AB01882319F0815183307A
:10EBB00010F49093AB018091170B9091180B9093E8
:10EBC0005F0580935E058091150B809364058091AD
:10EBD000160B809363058091190B809362058091D9
:10EBE0001A0B809360050BC00E94847C08C01092B1
:10EBF00025051092240510922305109222051F91DD
:10EC00000F91FF90EF9008958091C80A882319F41E
:10EC100080E090E00895459889ED9AE09093D20ABB
:10EC20008093D10A90913405E92FFF27E856FE4FD3
:10EC30009F5F9093340580818093DB0A9D3010F0B4
:10EC4000109234051092C80A0E947B7181E0809373
:10EC5000D80A8091D90A8093FA0A8EBD81E090E0AB
:10EC6000089587B18C6087B94298439810923B050C
:10EC700080E88093A90110923A058093A801089535
:10EC800080910A0A90910B0A81589F4F39F0809128
:10EC90000A0A90910B0A815880934505809140059E
:10ECA0008150809340058F3F09F052C18091A508A3
:10ECB000809341058091A7088093420589E0809365
:10ECC000400580911904992780739070892B21F455
:10ECD0008091D10580FF1DC08091A908882351F043
:10ECE00080914305882319F484E080933B0581E0FB
:10ECF000809343058091AA08882379F08091440588
:10ED0000882319F484E080933A0581E080934405D8
:10ED100004C0109243051092440580914305882356
:10ED200009F082C08091CC08282F332724FF07C028
:10ED300080915104882319F425FD8FC090C09091D3
:10ED4000A608983F48F080918C0A8D3D28F080916C
:10ED5000410588236CF00AC0983F78F080918C0AB6
:10ED6000853059F48091410587FF02C0429A01C065
:10ED7000429881E08093A90154C080913B05815065
:10ED800080933B058F3F09F06BC08091CF0885FFD2
:10ED90002FC090914505892F869580933B05992337
:10EDA00061F4909339058091410587FF02C0429A32
:10EDB00001C042981092A90153C081E080933905A7
:10EDC0008091A90190914105882349F480934505DC
:10EDD00080E48093A90199230CF43FC040C098239C
:10EDE00011F0429A01C0429886958093A90138C0DB
:10EDF00080918C0A869580933B058091A901813092
:10EE000021F41092450580E401C086958093A90104
:10EE10008091A90190914105892311F0429A01C086
:10EE20004298109239051CC080913B058150809317
:10EE30003B058F3FA9F489E080933B058091A901B0
:10EE4000813011F480E801C086958093A9018091FA
:10EE5000A9019091A908892311F0429A01C0429812
:10EE600080914405882309F043C09091CC0897FF16
:10EE700007C080915104882319F496FD52C053C0F5
:10EE80009091A808983F48F08091B50A8D3D28F0F0
:10EE90008091420588236CF00AC0983F78F08091F9
:10EEA000B50A853059F48091420587FF02C0439A24
:10EEB00001C0439881E08093A80136C080913A0553
:10EEC000815080933A058F3F79F58091B50A8695F8
:10EED00080933A058091A801813011F480E401C04B
:10EEE00086958093A8018091A8019091420517C052
:10EEF00080913A05815080933A058F3FA9F489E0CB
:10EF000080933A058091A801813011F480E801C016
:10EF100086958093A8018091A8019091AA088923E1
:10EF200011F0439A01C04398429B05C08091180498
:10EF3000886080931804439B06C080911804806108
:10EF4000809318040895809118048F7E809318048C
:10EF500008950F931F93CF93DF93482FEB01809178
:10EF60005204E42FFF27843BD8F08F010E0F1F1FA0
:10EF7000F801E053F64F808191819B01281B390BEA
:10EF8000C90163E070E00E94F69FCB01880F991FD2
:10EF9000860F971F0A5E154FF8019183808306C084
:10EFA000EE0FFF1FEA5EF54F11821082E42FFF275C
:10EFB000EE0FFF1FE053F64FD183C083DF91CF9157
:10EFC0001F910F9108954FB724E130E0F89480919C
:10EFD000C9008F778093C9008091C9008F7B80938F
:10EFE000C9008091C9008F7D8093C900832F992724
:10EFF0008093CD002093CC008091C80082608093E4
:10F00000C80080E18093C9008091CA008F77809307
:10F01000CA008091CA008F7B8093CA008091CA0089
:10F020008F7D8093CA008091CA008F7E8093CA0032
:10F030008091CA00877F8093CA008091C9008B7F2E
:10F040008093C9008091CA0084608093CA00809137
:10F05000CA0082608093CA008091C80087FF03C005
:10F060008091CE00F9CF8091C90080688093C9005B
:10F070004FBF0895EF92FF920F931F93CF93DF93AB
:10F08000482F00E010E08091AA01813061F41092D5
:10F09000AA0184E48093480510924A05109249051C
:10F0A00010924B05E6C180914805882319F421E0B0
:10F0B00030E001C0980190914905992371F4232B08
:10F0C00011F081E010C084E48093480590934A05D4
:10F0D0009093490590934B05B5C1913069F4232B6A
:10F0E00009F0A6C182E08093490580914A058F5FAF
:10F0F00080934A0583E0A4C19230D1F4232B09F018
:10F1000097C183E08093480540934B0590914A0551
:10F11000923039F410924C0547FF03C081E0809390
:10F120004C0583E0809349059F5F90934A058AC10F
:10F13000933009F07DC1232B09F07AC190934805E3
:10F1400082E08093490580914A058F5F80934A054C
:10F1500020914B05822F9927782F6627842F992796
:10F16000682B792B80918208813051F47370CB0128
:10F170008050924063E070E00E94F69FEB0119C05E
:10F18000823069F47770CB018050944066E070E083
:10F190000E94F69FEB012695269526950CC0EB0163
:10F1A000D370C856D140CE01D7FD0196EC01D5955C
:10F1B000C79526952695022F11270F7010700F5FA7
:10F1C0001F4F0D30110508F02CC10230110519F444
:10F1D00004E010E005C00430110511F402E010E075
:10F1E000D801A00FB11FFD01E053F64F808191813E
:10F1F0009E01281B390BC90137FF03C090958195EB
:10F200009F4F069704F5E091C408EE2351F0FF27C5
:10F21000EE0FFF1FE053F64F8081918184369105F8
:10F2200094F480915204883C30F480915204865FBB
:10F230008093520408C088EC8093520480916F0040
:10F240008F7D80936F00A053B64F8D919C91BC0130
:10F25000660F771F680F791F6C0F7D1F77FF02C045
:10F260006D5F7F4F7B01F594E794F594E794CE01B1
:10F2700001968E159F0524F40894E108F10808C052
:10F28000CE010197E816F9061CF40894E11CF11C64
:10F290000630110509F0ABC0C536D1050CF482C0AB
:10F2A00090914705E92FFF27ED5BF44FE081ED37A3
:10F2B00029F480914605809580934605993009F0A0
:10F2C0006DC080914605882319F4E33821F066C0AB
:10F2D000ED3709F063C08091440B8D3739F480918C
:10F2E000450B833899F463E87FEF0DC0833871F4E0
:10F2F0008091450B833819F460E070E004C08D37CD
:10F3000029F46DE770E085E00E94A9778091460BB3
:10F310008D3739F48091490B833899F46DE770E0AB
:10F320000DC0833871F48091490B833819F460E083
:10F3300070E004C08D3729F463E87FEF86E00E9417
:10F34000A97780914A0B8D3739F480914B0B833824
:10F3500099F463E87FEF0DC0833871F480914B0B13
:10F36000833819F460E070E004C08D3729F46DE74C
:10F3700070E089E00E94A9778091480B992787FD6A
:10F380009095BC018AE00E94A9778091470B99274C
:10F3900087FD9095BC018CE00E94A97710924705EB
:10F3A00010924605CA30D1055CF4809147058F5F05
:10F3B00080934705E82FFF27ED5BF44F83E88083B8
:10F3C000809147058A3011F4109247053FEFCC3900
:10F3D000D3076CF480914705E82FFF27ED5BF44FCE
:10F3E0008DE78083809146058095809346050530A2
:10F3F000110518F4B701802F11C00730110519F459
:10F40000BE0187E00BC00530110519F4BE0188E08C
:10F4100005C008301105B1F4BE018BE00E94A97748
:10F4200011C00231110570F081E08093AA010AC079
:10F4300081E08093AA0110924A0510924C0584E461
:10F440008093480580914A05803198F080914C0561
:10F45000882331F48091AA01882311F4809341011B
:10F4600010924A0510924C051092490584E480934D
:10F470004805E6E0CDB7DEB70C946EA0CF93FC0153
:10F4800097FF05C0CFEFF095E195FF4F01C0C1E0B8
:10F4900028E631E0CF01B9010E94F69FFC018B35CF
:10F4A000910554F08B5590408A35910538F484EBE2
:10F4B00090E08E1B9F0BFC0141E00DC0CF01855BEE
:10F4C00090408A35910518F4E45BF04003C02E1B90
:10F4D0003F0BF9014FEFEE0FFF1FE35CF64F259155
:10F4E00034918C2F992787FD9095289FB001299FF3
:10F4F000700D389F700D1124842F992787FD9095EA
:10F50000689FA001699F500D789F500D1124CA017A
:10F51000CF9108952AE530E0281B390BC9010E94DC
:10F520003E7A0895089508950895089508950895D8
:10F5300008950895089580E090E0089510924F0B8B
:10F5400010924E0B1092530B1092520B1092510BC3
:10F550001092500B1092540B82E390E00E94631BB8
:10F5600090934E0580934D050895E82FFF2783E083
:10F57000EE0FFF1F8A95E1F7E159F64F95819F3F06
:10F5800019F480E090E00895993C18F4892F9927A8
:10F590000895808182FF07C08AE0989FC0011124EE
:10F5A000885097400895892F99270895A0E0B0E0EA
:10F5B000ECEDFAE70C944FA080914D0590914E052B
:10F5C0000E946C1B882309F4CFC080914D05909157
:10F5D0004E05C29690934E0580934D05C0E0D0E055
:10F5E0007E01BB247FEFC72E8091540B8E3F21F408
:10F5F00081E08093E80204C08F3F11F4B092E802EA
:10F60000DD240FE619E0F801838187FF17C0B3946A
:10F610008581893C30F08D2D0E94B57AC80FD91FA5
:10F6200002C0C80FD11DF8018181E80EF11C86814E
:10F63000C81610F0C82E02C01092E802D394085FDA
:10F640001F4FFBE0FD15F8F6C092540BEF2841F573
:10F650002091530530915405409155055091560520
:10F66000BB27A52F942F832F90935205809351058C
:10F67000AA27BB27281B390B4A0B5B0BCE01AA27F5
:10F68000BB27280F391F4A1F5B1F20935305309358
:10F6900054054093550550935605C5E0D0E013C07E
:10F6A00080915105909152058C179D0718F4C81B45
:10F6B000D90B02C0C0E0D0E08B2D9927880F991F8D
:10F6C000C80FD91F2596D0934F0BC0934E0BCF3F39
:10F6D000D10578F480912601909127018C9F9001AB
:10F6E0008D9F300D9C9F300D1124C90164E670E0A0
:10F6F00013C0CE0196958795969587952091260102
:10F7000030912701289FA001299F500D389F500D4F
:10F710001124CA0169E170E00E94E29F7093510BCD
:10F720006093500B80914F05909150058C0F9D1F59
:10F730009093500580934F0552E0813D9507A0F0CE
:10F740002091520B3091530B2F5F3F4F805D9240C1
:10F75000E2E0813D9E07C0F79093500580934F05EE
:10F760003093530B2093520BE9E0CDB7DEB70C94E6
:10F770006BA030916505E32FFF2783E0EE0FFF1F9D
:10F780008A95E1F7E159F64F2781422F552747FD2A
:10F790005095809166059927841795072CF420933E
:10F7A0006605309368050AC0222341F08091670501
:10F7B00099274817590714F420936705832F8F5F03
:10F7C000809365058C30D0F01092650580916705B7
:10F7D0008F3F19F080935C0502C010925C05809108
:10F7E000660580935D058091680580935B058FEFCA
:10F7F000809367051092660510926805089595E15B
:10F80000899F802D11240E94219885ED9CE09F9373
:10F810008F9383EF97E99F938F93E091B705F091D2
:10F82000B80509950F900F900F900F900895CF9302
:10F83000C0E09091AB0190935A058091190485FF27
:10F8400013C080911004882331F0809182088630A3
:10F8500011F4CEE001C0C0E1992301F18091690566
:10F860008031E1F4C92F1AC090913305892F81505E
:10F870008232B0F480915104882349F4E92FFF27A4
:10F88000EE0FFF1FEC50F64F8491882349F4E92FC7
:10F89000FF27EE0FFF1FED50F64FC491CC2351F41C
:10F8A0008091CF0886FD03C01092AB0105C0C091C6
:10F8B000AB0102C0C0935A05809169058C1771F4A1
:10F8C00080916A0590916B050E946C1B882319F446
:10F8D00080E090E017C080EA9FE002C080ED97E0F2
:10F8E0000E94631B90936B0580936A05CC2331F0D3
:10F8F0008091AB01C81711F41092AB01C093690558
:10F900008C2F9927CF91089520E030E050E080912E
:10F910001C0B992789389105E9F08A38910564F420
:10F920008230910539F1833091051CF40197F9F08B
:10F9300028C0039719F125C08D389105A1F08E38A4
:10F94000910524F48A38910541F01BC08E38910549
:10F9500039F017C027EB3BE008C02FE83CE005C0BA
:10F9600025E53BE002C021E83BE05CE20AC026EC72
:10F9700032E002C029ED32E054E003C02DEA3BE062
:10F9800059E09091110B40E08091120B481770F4F0
:10F99000951760F4D901A90FB11DE42FFF27E2509C
:10F9A000F54F85898C939F5F4F5FEECF089520E3DD
:10F9B00035E7809142018B3211F08D32F9F480915C
:10F9C0006D08282F33278091460490914704829F29
:10F9D000A001839F500D929F500D1124CA0163E036
:10F9E00070E00E94F69FCB019B01205D3A48C196D2
:10F9F000C19708F03FC02EEF34E73CC0803229F5B4
:10FA00008091190481FF36C0209157053091580527
:10FA1000205D3A4855E72133350748F085E724391A
:10FA2000380718F420E335E702C02456304045E794
:10FA300020333407F8F454E72D3C350718F020E361
:10FA400035E718C02C593F4F15C08E3549F49091B9
:10FA500041048AE0989F90011124205D3A480AC031
:10FA6000863741F4909141048AE0989FC0011124A7
:10FA7000281B390BC90108951F9399278A389105CE
:10FA800009F4ABC18B38910524F48938910551F004
:10FA900064C38D38910509F497C28E38910509F435
:10FAA000F0C15BC30E94177C182F8093910C80914A
:10FAB0004C0490914D04A0914E04B0914F04BC01B0
:10FAC000CD0124E630E040E050E00E942BA0DA01B6
:10FAD000C9018C509E4F9093BD0B8093BC0B11239A
:10FAE00019F40E94D77C02C080E395E79093C30B82
:10FAF0008093C20B8091C20B9091C30B9093C50B66
:10FB00008093C40B9093C70B8093C60B2091BC0BC2
:10FB10003091BD0B8091C00B9091C10B2817390714
:10FB200024F43093C10B2093C00B8091BE0B9091B5
:10FB3000BF0B8217930724F43093BF0B2093BE0BA7
:10FB40001092B90B87EB9BE090937F0580937E0525
:10FB5000809142018093DD0B8091180480FF02C0E8
:10FB600083E401C080E28093DE0B209133052223E1
:10FB700009F1822F6AE00E94D69F805D8093C80BB6
:10FB8000822F0E94D69F892F805D8093C90B8AE3C4
:10FB90008093CA0B81E1289FF0011124ABECBBE0FC
:10FBA000E75CF54F9FE084918D939150319697FFDC
:10FBB000FACFDEC080911004882361F0A8ECBBE08E
:10FBC000E3E9FCE094E184918D939150319697FFA5
:10FBD000FACFC0C28091190485FF0CC0A8ECBBE02D
:10FBE000E9EAFCE094E184918D939150319697FF7E
:10FBF000FACFB0C280915905882301F1A8ECBBE08F
:10FC0000ECE8FCE096E084918D939150319697FF5B
:10FC1000FACF80910101805D8093CC0BAFECBBE00B
:10FC2000E0EDF8E09BE081918D93915097FFFBCF41
:10FC300080E28093DA0B8093DB0BB8C030916305D0
:10FC4000332309F497C087E58093C80B80E5809340
:10FC5000C90B40E24093CA0B20916405822F6AE0F1
:10FC60000E94D69F805D8093CB0B822F0E94D69FEF
:10FC7000892F805D8093CC0B8FE28093CD0B832FF7
:10FC80000E94D69F805D8093CE0B832F0E94D69FCB
:10FC9000892F805D8093CF0B4093D00B20915E0520
:10FCA00030915F0583E0293E380780F0C90168EE96
:10FCB00073E00E94E29FCB01805D8093D10BC9016C
:10FCC00068EE73E00E94E29F9C0102C04093D10B5A
:10FCD0002536310580F0C90164E670E00E94E29F9C
:10FCE000CB01805D8093D20BC90164E670E00E9475
:10FCF000E29F9C0103C080E28093D20BC9016AE0BD
:10FD000070E00E94E29FCB01805D8093D30BC9011C
:10FD10006AE070E00E94E29F805D8093D40B8DE6E4
:10FD20008093D50B80E28093D60B20916205253617
:10FD300060F0822F64E60E94D69F805D8093D70B8F
:10FD4000822F0E94D69F292F02C08093D70B822F2B
:10FD50006AE00E94D69F805D8093D80B822F0E941C
:10FD6000D69F892F805D8093D90B83E78093DA0B30
:10FD700080E261CF80913D048823D9F4A8ECBBE0F8
:10FD8000E1ECFCE090E184918D939150319697FFE6
:10FD9000FACF82E38093D80B8EE28093D90B80E375
:10FDA0008093DA0B84E38093DB0B81E68093DC0B9A
:10FDB000D1C1A8ECBBE0EFEBFCE094E184918D9322
:10FDC0009150319697FFFACF8091E802882309F489
:10FDD000C1C182E58093C80BBDC180914C04909154
:10FDE0004D04A0914E04B0914F04BC01CD0124E616
:10FDF00030E040E050E00E942BA0DA01C9018C50B5
:10FE00009E4F9093A50C8093A40C8091910C882315
:10FE100019F40E94D77C02C080E395E79093A70C69
:10FE20008093A60C88E78093A80C8091CA0A8093DF
:10FE3000A90C8091C90A81FF02C084E407C08091A7
:10FE4000CB0A833011F480E201C081E28093AA0CD6
:10FE50008FE89CE090937F0580937E0580919701C9
:10FE60008093B60C8091AA0C8093B80C8091CF0A35
:10FE70009091D00A97FD0196959587958093AB0C4C
:10FE800069C10E94B97B80914C0490914D04A0916E
:10FE90004E04B0914F04BC01CD0124E630E040E0B7
:10FEA00050E00E942BA0DA01C9018C509E4F909324
:10FEB000700B80936F0B8091260190912701909396
:10FEC0006A0B8093690B8091260190912701909392
:10FED0006C0B80936B0B80916A0A90916B0A97FD73
:10FEE00001969595879580935B0B8093620B20918B
:10FEF000CF0A3091D00A37FF02C02F5F3F4F3595B0
:10FF000027952093600B8091CD0A9091CE0A64E1F1
:10FF100070E00E94E29F6093610B2093670B6093F7
:10FF2000680B8091910C882319F40E94D77C02C041
:10FF300080E395E79093780B8093770B88E7809325
:10FF4000790B80912601909127019093740B8093F7
:10FF5000730B80915C058C5E80936D0B80915D05C9
:10FF60008C5E80936E0B8091520B9091530B6AE0E4
:10FF700070E00E94E29F7093760B6093750B809106
:10FF8000910C8093570B80914E0B90914F0B909357
:10FF9000720B8093710B85E59BE090937F058093B6
:10FFA0007E052091EB023091EC02C9016CE370E018
:10FFB0000E94E29F60937C0BC9016CE370E00E9499
:10FFC000E29F80937D0BC6C00E94B97B8091CD0AD1
:10FFD0009091CE0A64E670E00E94E29F7093970BC6
:10FFE0006093960B80916A0A90916B0A97FD019637
:10FFF000959587958093870B8091910190919201BF
:020000021000EC
:1000000097FD0196959587958093880B8091EE07D3
:1000100080938B0B8091CF0A9091D00A97FD019627
:100020009595879580938C0B80910201482F5527D9
:100030009A012E5F3F4F809126019091270128174A
:10004000390784F48091260190912701841B950B38
:100050009C01220F331F280F391F822F8650809357
:10006000930B02C01092930B8091930B853618F07E
:1000700084E68093930B8091330599279093950B99
:100080008093940B80914C0490914D04A0914E0468
:10009000B0914F04BC01CD0124E630E040E050E0D7
:1000A0000E942BA0DA01C9018C509E4F9093990BAE
:1000B0008093980B809126019091270190938E0B4D
:1000C00080938D0B80912601909127019093900B46
:1000D00080938F0B8091910C882319F40E94D77C18
:1000E00002C080E395E790939B0B80939A0B8091DD
:1000F000910C885880939C0B809126019091270148
:100100009093A00B80939F0B80915C058C5E8093F5
:10011000910B80915D058C5E8093920B8091520BC8
:100120009091530B6AE070E00E94E29F7093A20BE3
:100130006093A10B1092830B80914E0B90914F0B0B
:1001400090939E0B80939D0B81E89BE090937F059D
:1001500080937E052CE230E002C020E030E0C9014F
:100160001F910895EF92FF920F931F93CF93DF9308
:1001700080915705909158059C0163E0220F331F31
:100180006A95E1F7281B390B809138039091390368
:10019000280F391F37FF02C0295F3F4F53E03595C5
:1001A00027955A95E1F7309358052093570580918C
:1001B0006F0599278230910509F443C78330910573
:1001C0003CF4009781F0019709F42EC30C94868DBE
:1001D0008330910511F40C94A98A049711F40C94BE
:1001E000118C0C94868D80916E05282F332744271F
:1001F00055278F5F80936E05F9012131310510F08D
:100200000C94838DED58FF4F0C947DA080911904C0
:1002100085FF2AC080E00E9421988091260190915C
:1002200027016AE070E00E94F69F9F938F93809170
:100230002601909127016AE070E00E94F69F7F936B
:100240006F938BEE9CE09F938F9384E198E99F934B
:100250008F93E091B705F091B80509952DB73EB79A
:10026000285F3F4F2DBF28C080E00E9421988091D9
:100270002601909127016AE070E00E94F69F9F930B
:100280008F9380912601909127016AE070E00E948F
:10029000F69F7F936F9388EF9CE09F938F9383EFFC
:1002A00097E99F938F93E091B705F091B805099571
:1002B0008DB79EB708968DBF8091AE0A80FF3FC074
:1002C000809169048823E9F08AE00E942198809156
:1002D000420199279F938F9380914C0490914D04F4
:1002E000A0914E04B0914F04BC01CD0124E630E052
:1002F00040E050E00E942BA03F932F9385E09DE0CB
:10030000C0C68AE00E94219880914C0490914D04CF
:10031000A0914E04B0914F04BC01CD0124E630E021
:1003200040E050E00E942BA03F932F9381E19DE09D
:100330009F938F9383EF97E99F938F9397C38AE05F
:100340000E9421988CE19DE09F938F9383EF97E922
:100350000C94868A8091190485FF2AC085E10E9449
:1003600021988091EB029091EC026CE370E00E9486
:10037000E29F9F938F938091EB029091EC026CE34C
:1003800070E00E94E29F7F936F9386E29DE09F93CF
:100390008F9384E198E99F938F93E091B705F09153
:1003A000B80509952DB73EB7285F3F4F2DBF28C030
:1003B00085E10E9421988091EB029091EC026CE320
:1003C00070E00E94E29F9F938F938091EB02909147
:1003D000EC026CE370E00E94E29F7F936F9383E3F3
:1003E0009DE09F938F9383EF97E99F938F93E09185
:1003F000B705F091B80509958DB79EB708968DBFE2
:100400008FE10E94219880E690E09F938F938091E6
:100410006A0A90916B0A9F938F9380E49DE09F936B
:100420008F93C3EFD7E9DF93CF93E091B705F091B6
:10043000B8050995809118042DB73EB7285F3F4F46
:100440002DBF80FF06C089E20E9421988BE49DE0C9
:1004500073C389E20E9421988DE49DE0DAC6809101
:10046000190485FF1BC08AE20E9421988091520BDB
:100470009091530B9F938F938FE49DE09F938F9365
:1004800084E198E99F938F93E091B705F091B805C7
:1004900009958DB79EB706968DBF1BC08AE20E9454
:1004A00021988091520B9091530B9F938F9387E5E6
:1004B0009DE09F938F9383EF97E99F938F93E091B4
:1004C000B705F091B80509952DB73EB72A5F3F4FA4
:1004D0002DBF86E30E94219880914E0B90914F0B87
:1004E0006AE070E00E94E29F9F938F9380914E0B91
:1004F00090914F0B6AE070E00E94E29F7F936F93B0
:100500008FE59DE09F938F9383EF97E99F938F9360
:100510000C94648C89E00E9421988BE69DE09F9367
:100520008F9303EF17E91F930F93E091B705F091B5
:10053000B80509958EE10E9421980F900F900F90B9
:100540000F908DE69DE09F938F931F930F93E09103
:10055000B705F091B805099583E30E9421980F90A3
:100560000F900F900F908FE69DE09F938F931F93B6
:100570000F93E091B705F091B80509958FE30E94BC
:1005800021980F900F900F900F9081E79DE09F931F
:100590008F931F930F93E091B705F091B8050995DC
:1005A0008EE70E9421980F900F900F900F9087E890
:1005B0009DE00C94448C8091A501882309F462C0CD
:1005C0008DE50E9421988DE99DE09F938F93C3EF65
:1005D000D7E9DF93CF93E091B705F091B80509957E
:1005E00084E50E9421980F900F900F900F908091BA
:1005F000CA0A99279F938F938FE99DE09F938F93CA
:10060000DF93CF93E091B705F091B80509958EE59A
:100610000E9421982DB73EB72A5F3F4F2DBF809192
:10062000CD0A9091CE0A6AE070E00E94E29F7F932B
:100630006F9388EA9DE09F938F93DF93CF93E09130
:10064000B705F091B80509958DB79EB706968DBF91
:100650008091CB0A833081F48091C90A81FF06C062
:100660008BE50E94219882EB9DE0D3C58BE50E942B
:10067000219885EB9DE0CDC58BE50E94219888EB04
:100680009DE040C784E00AC48091A501882309F455
:100690007BC08091710543EFE42E47E9F42E882357
:1006A00009F44BC089E60E94219880913205992770
:1006B0009F938F938BEB9DE09F938F93FF92EF928D
:1006C000E091B705F091B805099585E70E9421985A
:1006D0002DB73EB72A5F3F4F2DBF809197019927D5
:1006E0009F938F9300E610E01F930F938091CF0AA2
:1006F0009091D00A9F938F9386EC9DE09F938F9368
:10070000FF92EF92E091B705F091B805099582E765
:100710000E9421988DB79EB70A968DBF80913005B3
:1007200099279F938F931F930F938091310599275A
:100730009F938F9382ED9DE086C689E60E94219863
:100740008091970199279F938F9380E690E09F93E4
:100750008F938091CF0A9091D00A9F938F9380912D
:10076000CC0A99279F938F9382EE9DE09F938F935E
:10077000FF92EF92E091B705F091B80509958DB71A
:100780009EB70C960C946C8C85E088C390913305D1
:100790009923D1F080917B05882381F0933270F406
:1007A00087E00E94FF7B83E90E94219880913305B6
:1007B00099279F938F938BEF9DE0DAC383E90E9483
:1007C000219886E09EE0E9C38091190433EFE32E7F
:1007D00037E9F32E85FF07C084E90E9421988CE059
:1007E0009EE00C94738C83E90E9421988FE19EE037
:1007F0000C94738C8091F40C863069F480917105AF
:10080000882321F0109271050C94808D81E08093F3
:1008100071050C94808D883011F00C94808D0E94AD
:10082000269881E00C947C8D80916E05282F3327CB
:10083000442755278F5F80936E05F90121313105DB
:1008400010F00C94838DEC57FF4F0C947DA0809199
:10085000190485FF43C080E00E9421988091520BCB
:100860009091530B9F938F93809126019091270134
:100870006AE070E00E94F69F9F938F93809126011B
:10088000909127016AE070E00E94F69F7F936F933A
:100890008091EB029091EC026CE370E00E94E29F89
:1008A0009F938F938091EB029091EC026CE370E048
:1008B0000E94E29F7F936F9385E39EE09F938F93C7
:1008C00084E198E99F938F93E091B705F091B80583
:1008D00009952DB73EB7225F3F4FC2C580E00E9409
:1008E00021988091520B9091530B9F938F938091FD
:1008F0002601909127016AE070E00E94F69F9F9385
:100900008F9380912601909127016AE070E00E9408
:10091000F69F7F936F938091EB029091EC026CE3D2
:1009200070E00E94E29F9F938F938091EB029091E1
:10093000EC026CE370E00E94E29F7F936F9380E58E
:100940009EE0F7C285E10E94219880E690E09F93A7
:100950008F9380919101909192019F938F938BE659
:100960009EE09F938F93C3EFD7E9DF93CF93E091FE
:10097000B705F091B80509958091AE0A2DB73EB73D
:10098000285F3F4F2DBF80FF51C0809169048823AD
:1009900039F18FE10E94219880914C0490914D048F
:1009A000A0914E04B0914F04BC01CD0124E630E08B
:1009B00040E050E00E942BA03F932F9385E79EE0FC
:1009C0009F938F9383E098E99F938F93E091B7056E
:1009D000F091B80509958DB79EB706968DBF38C0C2
:1009E0008FE10E94219880914C0490914D04A09138
:1009F0004E04B0914F04BC01CD0124E630E040E04C
:100A000050E00E942BA03F932F938EE79EE09F9390
:100A10008F93DF93CF93E091B705F091B8050995D7
:100A20002DB73EB72A5F3F4F2DBF12C08FE10E9406
:100A3000219887E89EE09F938F93DF93CF93E09177
:100A4000B705F091B80509950F900F900F900F9092
:100A500089E20E9421988091420199279F938F9368
:100A600081E99EE09F938F93DF93CF93E091B70549
:100A7000F091B80509958DB79EB706962DC7809160
:100A8000A5018823F9F08BE20E94219880919701BB
:100A900099279F938F938091CD0A9091CE0A6AE017
:100AA00070E00E94E29F7F936F9380E690E09F93B7
:100AB0008F938091CF0A9091D00A9F938F9384E96E
:100AC0009EE068C182E0EAC18FE30E942198809194
:100AD000500B9091510B9F938F9380914E0B90915F
:100AE0004F0B6AE070E00E94E29F9F938F9380918A
:100AF0004E0B90914F0B6AE070E00E94E29F7F9353
:100B00006F938BEA9EE09F938F93C3EFD7E9DF93B8
:100B1000CF93E091B705F091B8050995809118043D
:100B20002DB73EB7265F3F4F2DBF80FF0AC082E53D
:100B30000E9421988FEB9EE09F938F9383E098E92A
:100B4000E5C482E50E94219882EC9EE062C3809118
:100B5000A50123EFE22E27E9F22E882309F449C0EC
:100B600084E50E9421988091CA0A99279F938F93C8
:100B70008091CC0A99279F938F9385EC9EE09F9359
:100B80008F93E701FF92EF92E091B705F091B805DE
:100B900009958DB79EB708968DBF8091CB0A83309B
:100BA00051F484E60E94219888ED9EE09F938F93F4
:100BB000FF92EF920BC084E60E9421988EED9EE09A
:100BC0009F938F9384E198E99F938F93E091B7056A
:100BD000F091B80509950F900F900F900F908091AC
:100BE000C90A81FF95C784E60E94219884EE9EE0A1
:100BF00010C384E50E9421988AEE9EE074C680911D
:100C0000700593EFE92E97E9F92E882309F45BC06C
:100C100089E60E94219883E00E94B57A6AE070E03C
:100C20000E94E29F9F938F9383E00E94B57A6AE0CF
:100C300070E00E94E29F7F936F9382E00E94B57AFA
:100C40006AE070E00E94E29F9F938F9382E00E948F
:100C5000B57A6AE070E00E94E29F7F936F9381E033
:100C60000E94B57A6AE070E00E94E29F9F938F93A2
:100C700081E00E94B57A6AE070E00E94E29F7F9373
:100C80006F9380E00E94B57A6AE070E00E94E29F74
:100C90009F938F9380E00E94B57A6AE070E00E9493
:100CA000E29F7F936F9380E09FE09F938F93FF92EB
:100CB000EF92E091B705F091B80509952DB73EB7D1
:100CC0002C5E3F4FCDC389E60E94219880E690E0DC
:100CD0009F938F9380918E09992787FD90959F937D
:100CE0008F9380918609992787FD90959F938F9385
:100CF00080917E09992787FD90959F938F9380918E
:100D00007609992787FD90959F938F938DE19FE0BA
:100D10009F938F93FF92EF92E091B705F091B80502
:100D200009958DB79EB70E96D7C5809170059091A5
:100D30005A08882309F4AFC0943009F4AEC0963045
:100D4000C9F58EE70E94219885E00E94B57A6AE095
:100D500070E00E94E29F9F938F9385E00E94B57A96
:100D60006AE070E00E94E29F7F936F9384E00E94AC
:100D7000B57A6AE070E00E94E29F9F938F9384E0CF
:100D80000E94B57A6AE070E00E94E29F7F936F93C1
:100D900080E39FE09F938F9383EF97E99F938F93D7
:100DA000E091B705F091B80509952DB73EB7245FDE
:100DB0003F4F56C3973008F4ABC68EE70E94219888
:100DC00088E00E94B57A6AE070E00E94E29F9F93FB
:100DD0008F9388E00E94B57A6AE070E00E94E29FFB
:100DE0007F936F9387E00E94B57A6AE070E00E947B
:100DF000E29F9F938F9387E00E94B57A6AE070E04C
:100E00000E94E29F7F936F9386E00E94B57A6AE02A
:100E100070E00E94E29F9F938F9386E00E94B57AD4
:100E20006AE070E00E94E29F7F936F9385E00E94EA
:100E3000B57A6AE070E00E94E29F9F938F9385E00D
:100E40000E94B57A6AE070E00E94E29F7F936F9300
:100E500084E00E94B57A6AE070E00E94E29F9F936E
:100E60008F9384E00E94B57A6AE070E00E94E29F6E
:100E70007F936F938FE39FE09F938F9383EF97E927
:100E80009F938F93E091B705F091B80509958DB7C1
:100E90009EB7489621C5943021F486E00E94FF7BDE
:100EA00037C69630F1F48EE70E94219880E690E0F4
:100EB0009F938F9380919E09992787FD90959F938B
:100EC0008F9380919609992787FD90959F938F9393
:100ED0008CE59FE09F938F9383EF97E99F938F9388
:100EE000B6C2973008F414C68EE70E94219880E6B7
:100EF00090E09F938F938091AE09992787FD9095FD
:100F00009F938F938091A609992787FD90959F9332
:100F10008F9380919E09992787FD90959F938F933A
:100F200080919609992787FD90959F938F938FE6DF
:100F30009FE09F938F9383EF97E99F938F93ECCEDE
:100F400090913305992309F44AC080917B05882349
:100F5000F9F09332E8F487E00E94FF7B83E90E9476
:100F600021988091330599279F938F9382E89FE082
:100F70009F938F9383E098E99F938F93E091B705B8
:100F8000F091B80509952DB73EB72A5F3F4F68C26B
:100F900083E90E9421988DE89FE09F938F9303EF50
:100FA00017E91F930F93E091B705F091B8050995E4
:100FB0001F921F929091330581E1989FC0011124E7
:100FC000875C954F9F938F931F930F93E091B70585
:100FD000F091B80509958DB79EB70A967DC48091AA
:100FE000190403EFE02E07E9F02E85FF06C084E91F
:100FF0000E94219883E99FE076C483E90E942198AA
:1010000086EA9FE070C48091F40C863079F4809178
:101010007005882319F01092700503C081E0809359
:10102000700585E00E94FF7B86E085C2883009F468
:10103000F4C3813009F064C50E94269810926F05B0
:101040005DC580916E05282F3327442755278F5F74
:1010500080936E05F9012131310508F054C5EB5636
:10106000FF4F0C947DA080E00E94219880ED98E0D5
:101070009F938F938091010199279F938F938CEB7E
:101080009FE09F938F9383E098E99F938F93E091E4
:10109000B705F091B80509952DB73EB7285F3F4FCA
:1010A000DFC185E10E9421988EED98E09F938F9398
:1010B000809102016AE00E94D69F892F99279F9311
:1010C0008F93809102010E94D69F99279F938F93BF
:1010D0008BEC9FE09F938F9383EF97E99F938F9380
:1010E000E091B705F091B805099575CF8AE20E94A5
:1010F00021988CED9FE09F938F93C3EFD7E9DF9307
:10110000CF93E091B705F091B80509958091AE0AAB
:101110000F900F900F900F9080FF41C08091680852
:1011200090912F0481FD0BC0892F99279F938F9356
:1011300081EE9FE09F938F93DF93CF931FCFE0913A
:10114000B705F091B805933318F08BEE9FE002C01D
:1011500082EF9FE09F938F93DF93CF9309950F903A
:101160000F900F900F908091910AE091B705F09148
:10117000B80590912F0480FF0BC0892F99279F936A
:101180008F9389EF9FE09F938F93DF93CF9372CCE0
:10119000892F99279F938F938FEF9FE0B7C085E0AA
:1011A00090E137C08FE30E9421988EE090E19F93F9
:1011B0008F93C3EFD7E9DF93CF93E091B705F09119
:1011C000B80509950F900F900F900F908091BE0871
:1011D000882319F482E190E11CC080912604E091FB
:1011E000B705F091B805882319F08BE190E102C0B2
:1011F00082E290E19F938F93DF93CF9309950F90B5
:101200000F900F900F908091CE0886FF81C489E2E5
:1012100090E19F938F93DF93CF9369C384E50E94FE
:10122000219880E390E19F938F93C3EFD7E9DF93F9
:10123000CF93E091B705F091B80509958091AE0A7A
:101240000F900F900F900F9085FD03C085E390E104
:1012500008C08091AC080E941048823358F48EE395
:1012600090E19F938F93DF93CF93E091B705F09137
:10127000B80516C0843B18F085E490E1F2CF809168
:10128000CE08E091B705F091B80585FF03C08CE466
:1012900090E102C083E590E19F938F93DF93CF931A
:1012A00009950F900F900F900F908091C20888239E
:1012B00009F42EC48EE50E9421988091C2089927D6
:1012C0009F938F938AE590E1CDCB89E60E94219888
:1012D00085E690E19F938F93C3EFD7E9DF93CF9398
:1012E000E091B705F091B80509950F900F900F9018
:1012F0000F908091C108E091B705F091B80588235F
:1013000051F099279F938F938FE690E19F938F934E
:10131000DF93CF9337CE83E790E19F938F93DF9353
:10132000CF93E9C28091720513EFE12E17E9F12EF8
:10133000882309F053C08EE70E94219880917001A4
:1013400099279F938F9380915D08E82FFF27EE0FD9
:10135000FF1FE053F64F808191819F938F9380917F
:101360005C08E82FFF27EE0FFF1FE053F64F808148
:1013700091819F938F9389E790E19F938F93FF9241
:10138000EF92E091B705F091B805099583E90E94C5
:1013900021988DB79EB70A968DBF80915F08E82F80
:1013A000FF27EE0FFF1FE053F64F808191819F933F
:1013B0008F9380915E08E82FFF27EE0FFF1FE05309
:1013C000F64F8081918181589F4F9F938F938DE835
:1013D00090E19F938F93FF92EF9259CE8EE70E94F8
:1013E00021988091550499279F938F93809154045D
:1013F00099279F938F938091530499279F938F935D
:101400008CE990E19F938F93FF92EF92E091B70563
:10141000F091B805099583E90E9421988DB79EB790
:101420000A968DBF8091580499279F938F9380913E
:10143000570499279F938F938091560499279F93E0
:101440008F9380EB90E19F938F93FF92EF92E091C7
:10145000B705F091B80509952DB73EB7265F3F4F08
:101460002DBF56C380917B05882309F451C38EE7B5
:101470000E9421988091AE0A86FD11C084EC90E113
:101480009F938F9384E198E99F938F93E091B705A1
:10149000F091B80509950F900F900F900F908091E3
:1014A000CC0899278F709070892B89F083ED90E19B
:1014B0009F938F9384E198E99F938F93E091B70571
:1014C000F091B80509950F900F900F900F908091B3
:1014D000AE0A82FF11C08DED90E19F938F9384E15E
:1014E00098E99F938F93E091B705F091B80509951E
:1014F0000F900F900F900F908091AE0A83FD08C35C
:1015000082EE90E19F938F9384E198E99F938F936C
:10151000EEC10091F40C063089F4809172058823A5
:1015200019F01092720503C081E08093720586E085
:101530000E94FF7B87E00E94FF7BE2C2083009F433
:10154000D8C2013009F0DCC20E94269800936F05D2
:10155000D5C280916E05282F33278F5F80936E054B
:101560002230310509F447C0233031053CF4211500
:10157000310549F02130310501F1C5C22630310570
:101580000CF0C1C277C080E00E94219880EF90E10A
:101590009F938F9303EF17E91F930F93E091B70584
:1015A000F091B805099585E10E9421980F900F9060
:1015B0000F900F908FEF90E167C180916305C3EFAB
:1015C000EC2EC7E9FC2E882381F08EE70E9421983B
:1015D0008091630599279F938F9380916405992744
:1015E0009F938F9384E191E16BC18EE70E942198D4
:1015F00086E291E178C183E90E94219880912601D9
:10160000909127016AE070E00E94F69F9F938F936C
:1016100080912601909127016AE070E00E94F69F78
:101620007F936F9389E391E19F938F9303EF17E982
:101630001F930F93E091B705F091B80509958EE9D6
:101640000E9421982DB73EB7285F3F4F2DBF8DEAEE
:101650009BE09F938F9383E491E19F938F931F93DC
:101660000F93E091B705F091B80509958DB79EB736
:1016700006968DBF8091AC018823E9F180916D05BC
:101680008823C9F080917B058823A9F089E40E9412
:10169000219886E491E19F938F9383EF97E99F933D
:1016A0008F93E091B705F091B80509950F900F90D1
:1016B0000F900F901AC089E40E9421988091AC018C
:1016C00099279F938F938AE491E19F938F9383EF60
:1016D00097E99F938F93E091B705F091B80509952D
:1016E0002DB73EB72A5F3F4F2DBF8FE30E94219851
:1016F00081E591E105C08FE30E9421988CE591E19D
:101700009F938F9383EF97E99F938F93E091B70512
:10171000F091B80509950F900F900F900F90809160
:101720006005882331F484E50E9421988BE691E1DD
:1017300039C08091CB0A833081F580916D05882373
:1017400051F08091AC01882331F084E50E9421980A
:1017500089E791E105C084E50E94219887E891E13D
:101760009F938F9383EF97E99F938F93E091B705B2
:10177000F091B80509950F900F900F900F90809100
:10178000F40C8630F1F48091AC01882319F0806864
:101790008093610510926D0514C084E50E94219824
:1017A00085E991E19F938F9383EF97E99F938F93BF
:1017B000E091B705F091B80509950F900F900F9043
:1017C0000F908091F40C843059F49091AC01809189
:1017D00060059817E8F481E080936D05980F0AC0C2
:1017E000823069F49091AC01923090F081E0809366
:1017F0006D0591509093AC0110927B0509C0883023
:1018000039F40E94269884E080936F0510926E054B
:101810008091F40C813009F073C10E94269882E017
:101820006BC180916E05282F33278F5F80936E05E3
:101830002230310509F465C0233031053CF421150F
:10184000310549F02130310521F15DC126303105E6
:101850000CF059C195C080E00E94219883EA91E183
:101860009F938F9303EF17E91F930F93E091B705B1
:10187000F091B805099585E10E9421980F900F908D
:101880000F900F9082EB91E19F938F931F930F9393
:101890002EC080916305B3EFEB2EB7E9FB2E8823B2
:1018A000E9F08EE70E9421988091630599279F9324
:1018B0008F938091640599279F938F9384EC91E196
:1018C0009F938F93FF92EF92E091B705F091B80547
:1018D00009958DB79EB708968DBF1AC18EE70E94F5
:1018E000219886ED91E19F938F93FF92EF92E09183
:1018F000B705F091B80509950F900F900F900F90D4
:1019000007C183E90E9421988091260190912701C7
:101910006AE070E00E94F69F9F938F93809126016A
:10192000909127016AE070E00E94F69F7F936F9389
:1019300088EE91E19F938F9303EF17E91F930F9325
:10194000E091B705F091B80509958EE90E942198BC
:101950002DB73EB7285F3F4F2DBF8DEA9BE09F9389
:101960008F9382EF91E19F938F931F930F93E09159
:10197000B705F091B80509958DB79EB706968DBF4E
:101980008091F40C882349F08091D8079091D90771
:1019900001969093D9078093D8078091AD01882351
:1019A000E9F180916C058823C9F080917B0588233B
:1019B000A9F089E40E94219885EF91E19F938F938C
:1019C00083EF97E99F938F93E091B705F091B80566
:1019D00009950F900F900F900F901AC089E40E9404
:1019E00021988091AD0199279F938F9389EF91E181
:1019F0009F938F9383EF97E99F938F93E091B70520
:101A0000F091B80509952DB73EB72A5F3F4F2DBF1E
:101A10008FE30E94219883E092E105C08FE30E944A
:101A200021988EE092E19F938F9383EF97E99F93A4
:101A30008F93E091B705F091B80509950F900F903D
:101A40000F900F9080916005882331F484E50E9407
:101A500021988DE192E113C080916C05882351F0AB
:101A60008091AD01882331F084E50E9421988BE2BA
:101A700092E105C084E50E94219889E392E19F9359
:101A80008F9383EF97E99F938F93E091B705F09140
:101A9000B80509950F900F900F900F908091F40C5E
:101AA000843059F49091AD0180916005981740F50C
:101AB00081E080936C05980F0AC0823069F49091A0
:101AC000AD019230E8F081E080936C0591509093E5
:101AD000AD0110927B0514C0863049F48091AD01B0
:101AE000882311F08093610510926C0509C0813044
:101AF00039F40E94269883E080936F0510926E055A
:101B00001092F40C05C010926E0502C010926F0581
:101B1000E6E0CDB7DEB70C946EA04FB728E130E019
:101B2000F8948091C9008F778093C9008091C90093
:101B30008F7B8093C9008091C9008F7D8093C900FD
:101B4000832F99278093CD002093CC008091C800EB
:101B500082608093C80080E18093C9008091CA00B0
:101B60008F778093CA008091CA008F7B8093CA00D0
:101B70008091CA008091CA008F7E8093CA008091B4
:101B8000CA0088608093CA008091C9008B7F8093CF
:101B9000C9008091CA0084608093CA008091CA0005
:101BA00082608093CA008091C80087FF03C0809143
:101BB000CE00F9CF8091C90080688093C9008091E0
:101BC000D20C84608093D20C4FBF08959091480549
:101BD000992341F48F3031F49093740580E580931C
:101BE00048050895E0917405EF5FE0937405E831CE
:101BF00021F481E0809373050895E93120F089E1B3
:101C0000809374050895FF27E554F34F808308956A
